:020000040000FA
:1000000000040020E508000079050000C508000094
:10001000830500008D05000097050000000000002A
:1000200000000000000000000000000009090000BE
:10003000A105000000000000AB050000B5050000B0
:10004000BF050000C9050000D3050000DD05000064
:10005000E7050000F1050000FB05000005060000B3
:100060000F06000019060000230600002D06000000
:1000700037060000410600004B0600005506000050
:100080005F06000069060000730600007D060000A0
:1000900087060000910600009B060000A5060000F0
:1000A000AF060000B9060000C3060000CD06000040
:1000B000D7060000E1060000EB060000F506000090
:1000C000FF06000009070000130700001D070000DD
:1000D00027070000310700003B070000450700002C
:1000E0004F07000059070000630700006D0700007C
:1000F00077070000810700008B07000095070000CC
:100100009F0700001FB500F003F88DE80F001FBD2A
:1001100000F0DEBB1FB56FF00100009040100390AF
:10012000029001904FF010208069000B420900F00E
:100130001F045DF822300120A04083434DF8223097
:10014000684600F044F91FBDF0B54FF6FF734FF459
:10015000B4751A466E1E11E0A94201D3344600E080
:100160000C46091B30F8027B641E3B441A44F9D14B
:100170009CB204EB134394B204EB12420029EBD17E
:1001800098B200EB134002EB124140EA0140F0BD8F
:10019000DD4992B00446D1E90001CDE91001FF220A
:1001A0004021684600F03AFB94E80F008DE80F000C
:1001B000684610A902E004C841F8042D8842FAD12B
:1001C00010216846FFF7C0FF1090AA208DF8440068
:1001D000FFF7A0FF00F0F2F84FF01024A069102202
:1001E0006946803000F001F9A069082210A900F0EA
:1001F000FCF800F0D7F84FF080510A6949690068AF
:100200004A43824201D8102070470020704710B541
:10021000D0E900214FF0805002EB8103026944696C
:100220006243934209D84FF01022536903EB8103D4
:100230000169406941438B4201D9092010BD5069D1
:10024000401C01D0002010BD0F2010BD70B501680A
:100250000446AE4D4FF01020062951D2DFE801F0E0
:10026000320318283B1DD4E90265646829463046EC
:1002700000F0CDF82A462146304600F0B6F8AA0034
:100280002146304600F09EFA002800D0032070BDC1
:1002900000F050FB4FF4805007E0201DFFF7ABFF4C
:1002A0000028F4D100F046FB60682860002070BD93
:1002B000241D94E80700920000F084FA0028F6D08C
:1002C0000E2070BD8069401C12D0201DFFF79FFFDB
:1002D0000028F6D109E08069401C09D0201DFFF7F5
:1002E0008AFF0028EDD1606820B12046FFF750FF5B
:1002F000042070BDFFF70EFF00F060F800F052F828
:10030000072070BD10B50C46182802D001200860E7
:1003100010BD2068FFF79AFF206010BD4FF0102439
:10032000A069401C05D0A569A66980353079AA2846
:1003300008D06069401C2DD060690068401C29D03D
:1003400060692CE010212846FFF7FEFE31688142EB
:100350001CD1A16901F18002C03105E030B108CAA9
:1003600051F8040D984201D1012000E000208A429A
:10037000F4D158B1286810B1042803D0FEE728460C
:1003800000F057F861496868086008E000F016F866
:1003900000F008F84FF480500168491C01D000F0CB
:1003A000A3FAFEE7BFF34F8F59480168594A01F499
:1003B000E06111430160BFF34F8FFEE74FF0102063
:1003C0008169491C02D0806900F0ADB87047524A7B
:1003D00001681160121D416811604F4A8168103236
:1003E0001160111DC068086070472DE9F041174683
:1003F0000D460646002406E03046296800F0A6F8BF
:10040000641C2D1D361DBC42F6D3BDE8F08170B5CD
:100410000C4605464FF4806608E0284600F083F855
:10042000B44205D3A4F5806405F58055002CF4D1C1
:1004300070BD4168044609B1012500E000254FF078
:1004400010267069A268920000F0BCF9C8B120467D
:1004500000F01AF89DB17669A56864684FF4002031
:1004600084420AD2854208D229463046FFF7CFFFA0
:100470002A4621463046FFF7B8FFFFF79FFFFFF7F8
:1004800091FFFFF747FEF8E72DE9FF414FF01024F9
:10049000616980680D0B01EB800000F6FF70010BB5
:1004A00000200090019002900246039068460123CC
:1004B0000BE0560902F01F0C50F8267003FA0CFCF2
:1004C00047EA0C0740F82670521CAA42F1D30AE012
:1004D0004A0901F01F0650F8225003FA06F6354388
:1004E00040F82250491C8029F2D3A169090B4A091E
:1004F00001F01F0150F822408B409C4340F82240FD
:10050000FFF765FFBDE8FF815809000000000020EB
:100510000CED00E00400FA050006004014480168F4
:100520000029FCD07047134A0221116010490B6862
:10053000002BFCD00F4B1B1D186008680028FCD056
:100540000020106008680028FCD07047094B10B5E7
:1005500001221A60064A1468002CFCD00160106861
:100560000028FCD00020186010680028FCD010BDC6
:1005700000E4014004E5014008208F49096809585A
:10058000084710208C4909680958084714208A49EF
:100590000968095808471820874909680958084711
:1005A0003020854909680958084738208249096878
:1005B000095808473C2080490968095808474020E5
:1005C0007D4909680958084744207B49096809584A
:1005D0000847482078490968095808474C20764957
:1005E000096809580847502073490968095808479D
:1005F0005420714909680958084758206E4909680C
:10060000095808475C206C49096809580847602068
:100610006949096809580847642067490968095801
:100620000847682064490968095808476C206249EE
:1006300009680958084770205F4909680958084740
:1006400074205D4909680958084778205A490968A3
:10065000095808477C2058490968095808478020EC
:1006600055490968095808478420534909680958B9
:100670000847882050490968095808478C204E4986
:1006800009680958084790204B49096809580847E4
:10069000942049490968095808479820464909683B
:1006A000095808479C204449096809580847A02070
:1006B0004149096809580847A4203F490968095871
:1006C0000847A8203C49096809580847AC203A491E
:1006D000096809580847B020374909680958084788
:1006E000B4203549096809580847B82032490968D3
:1006F00009580847BC203049096809580847C020F4
:100700002D49096809580847C4202B490968095828
:100710000847C8202849096809580847CC202649B5
:10072000096809580847D02023490968095808472B
:10073000D4202149096809580847D8201E4909686A
:1007400009580847DC201C49096809580847E02077
:100750001949096809580847E420174909680958E0
:100760000847E8201449096809580847EC2012494D
:10077000096809580847F0200F49096809580847CF
:10078000F4200D49096809580847F8200A49096802
:1007900009580847FC2008490968095808475FF4C8
:1007A0008070054909680958084700000348044952
:1007B000024A034B70470000000000206809000057
:1007C0006809000040EA010310B59B070FD1042A15
:1007D0000DD310C808C9121F9C42F8D020BA19BA0C
:1007E000884201D9012010BD4FF0FF3010BD1AB171
:1007F000D30703D0521C07E0002010BD10F8013BC6
:1008000011F8014B1B1B07D110F8013B11F8014BEC
:100810001B1B01D1921EF1D1184610BD02F0FF033F
:1008200043EA032242EA024200F005B870477047EB
:1008300070474FF000020429C0F0128010F0030C42
:1008400000F01B80CCF1040CBCF1020F18BF00F8C3
:10085000012BA8BF20F8022BA1EB0C0100F00DB872
:100860005FEAC17C24BF00F8012B00F8012B48BFD0
:1008700000F8012B70474FF0000200B51346944674
:100880009646203922BFA0E80C50A0E80C50B1F1E8
:100890002001BFF4F7AF090728BFA0E80C5048BFFC
:1008A0000CC05DF804EB890028BF40F8042B08BF9A
:1008B000704748BF20F8022B11F0804F18BF00F896
:1008C000012B7047014B1B68DB68184700000020B4
:1008D00009480A497047FFF7FBFFFFF713FC00BD0B
:1008E00020BFFDE7064B1847064A1060016881F3F8
:1008F0000888406800470000680900006809000097
:100900001D030000000000201EF0040F0CBFEFF3D9
:100910000881EFF30981886902380078182803D12B
:1009200000E00000074A1047074A12682C3212689C
:100930001047000000B5054B1B68054A9B589847B7
:1009400000BD000005030000000000205409000065
:1009500004000000001000000000000000FFFFFF86
:040960000090D00330
:1010000048120020D1E001006D9F000041E0010086
:101010006D9F00006D9F00006D9F000000000000AC
:1010200000000000000000000000000029E10100B5
:101030006D9F0000000000006D9F00006D9F00008C
:1010400091E1010097E101006D9F00006D9F00009C
:101050006D9F00006D9F00006D9F00006D9F000060
:101060009DE101006D9F00006D9F0000A3E1010064
:101070006D9F0000A9E10100AFE10100B5E10100B1
:101080006D9F00006D9F00006D9F00006D9F000030
:101090006D9F00006D9F00006D9F00006D9F000020
:1010A000BBE10100C1E101006D9F00006D9F0000E8
:1010B0006D9F00006D9F00006D9F00006D9F000000
:1010C000C7E101006D9F00006D9F00006D9F000053
:1010D0006D9F00006D9F00006D9F00006D9F0000E0
:1010E0006D9F00006D9F00006D9F00006D9F0000D0
:1010F0006D9F00006D9F00006D9F00006D9F0000C0
:101100006D9F00006D9F000000F002F81CF0CDFF05
:101110000AA090E8000C82448344AAF10107DA4552
:1011200001D11CF0C2FFAFF2090EBAE80F0013F0B4
:10113000010F18BFFB1A43F001031847BCD501008B
:10114000DCD501000A4410F8014B14F00F0508BF6C
:1011500010F8015B240908BF10F8014B6D1E05D083
:1011600010F8013B6D1E01F8013BF9D1641E03D05C
:10117000641E01F8015BFBD19142E4D3704700008B
:101180000023002400250026103A28BF78C1FBD890
:10119000520728BF30C148BF0B6070471FB500F031
:1011A0003DF88DE80F001FBD1EF0040F0CBFEFF3DC
:1011B0000880EFF30980014A10470000BF9D00003E
:1011C0008269034981614FF00100104470470000BB
:1011D000D511000001B41EB400B511F043F901B4FB
:1011E0000198864601BC01B01EBD0000F0B4404627
:1011F000494652465B460FB402A0013001B506488D
:10120000004700BF01BC86460FBC80468946924617
:101210009B46F0BC70470000091100001CF042BF63
:1012200070B51C4C054608202070A01C00F065F825
:101230005920A08029462046BDE8704007F01CB820
:1012400010B507F024F813490020891E087010BD5E
:1012500070B50C460F49891E097829B1A0F16001CB
:10126000532906D3012011E0602802D043F2010087
:101270000CE020CC084E94E80E0006EB8000A0F5B0
:101280008050241FD0F8806E2846B047206070BD83
:10129000012070470A00002014E2010010B5044646
:1012A0000021012000F03FF80021182000F03BF859
:1012B00000210B2000F037F80421192000F033F84A
:1012C00004210D2000F02FF804210E2000F02BF84F
:1012D00004210F2000F027F80421C84300F023F870
:1012E0000721162000F01FF80721152000F01BF839
:1012F0002046FFF795FF002010BD8C21018070472C
:10130000FFF79EBF10487047104A10B514680F4B86
:101310000F4A08331A60FFF79BFF0C48001D04605A
:1013200010BD704770474907090E002806DA00F023
:101330000F0000F1E02080F8141D704700F1E0205C
:1013400080F800147047000003F9004310050240C4
:101350000100000130B5F74D044610280AD0112CC9
:1013600006D02846122C817806D0132C08D0FFDF37
:10137000AC7030BDFFDFFBE71129F9D0FFDFF7E7E5
:101380001129F5D0FFDFF3E770B50FF05AFA0446E4
:1013900010F030FE201AC4B206200DF02DFC0546D8
:1013A00006200DF031FC2E1A07200DF025FC054615
:1013B00007200DF029FCDF49281A321888781228F6
:1013C0000DD000231A4413280BD0002002440878C3
:1013D000022808D000201044201AC0B270BD01239A
:1013E000F0E70120F2E70120F5E7D24800B50079E7
:1013F000D049420897B051F8050F89880CD01722C0
:101400008DF80020CDF80200ADF806100BA9684653
:101410000AF02BFF17B000BD4022F1E702210DF0CA
:1014200040BC2DE9F04196B01D4690460E46074659
:10143000FFF7F4FF04000BD02078222804D3A07F0C
:10144000C0F34010A84206D1082016B0BDE8F081D4
:1014500043F20200F9E745208DF80000ADF8027074
:101460003DB101208DF804008DF805608DF80680EF
:1014700002E000208DF804000BA968460AF0F5FE92
:10148000A07F65F34510A0770020DEE730B5044665
:10149000A1F120000D460A284AD2DFE800F0050736
:1014A0000C1C2328353A3F44FFDF42E020782028F7
:1014B0003FD1FFDF3DE09F480178032939D0807894
:1014C000132836D02078242833D0252831D023285B
:1014D0002FD0FFDF2DE0207822282AD0232828D8FB
:1014E000FFDF26E02078222823D0FFDF21E02078CC
:1014F00022281ED024281CD026281AD0272818D00D
:10150000292816D0FFDF14E02078252811D0FFDF2E
:101510000FE0207825280CD0FFDF0AE0207825286E
:1015200007D0FFDF05E02078282802D0FFDF00E0A9
:10153000FFDF257030BD30B50B8840F67B444FF699
:10154000FF72022801D0934204D09D1FA54224D2ED
:10155000022802D04D88954203D04D88AD1FA54288
:101560001BD24C88A34218D88B88B3F5FA7F14D2CB
:10157000022802D0C888904205D0C88840F6774536
:101580000A38A84209D2C888904208D0944206D0AE
:101590005B1C6343B3EB800F01DB072030BD0020F1
:1015A00030BD70B514460D46064611F0C9F960B954
:1015B0000DB1A54201D90C2070BD002409E000BF87
:1015C00056F8240011F0BCF908B1102070BD641C5D
:1015D000E4B2AC42F4D3002070BDF0B50024059D08
:1015E00010B1A94203D851E009B90020F0BD09208B
:1015F000F0BD055D8DB107197E78112E3FD00FDC4F
:101600000A2E3CD2DFE806F03B1624242A2A2C2C92
:101610003333025D72BB641CE4B28C42F9D3E4E75D
:101620001D2E2CDAA6F11206042E28D2DFE806F0D1
:1016300027271018022DDAD1BD781D70072D01D291
:101640006D0701D40A20F0BD157845F0010515E0BD
:10165000EE43F60707E0012D07D010E00620F0BDAD
:101660002E07A6F18056002EF5D06046F0BD157805
:10167000AE0701D50B20F0BD45F002051570055DE4
:10168000641C2C44E4B28C4202D9B0E74FF4485CAD
:101690008C42AED3A9E710B50278540809D00122D4
:1016A00043F20223012C07D0022C0DD0032C13D1BE
:1016B0000FE00020087005E080790324B4EB901F50
:1016C0000AD10A70002010BD8079B2EB901F03D1BF
:1016D000F7E780798009F4D0184610BD154A917B50
:1016E00039B1D17B022908D0032908D043F2022066
:1016F00070470146101D01F03FBB032100E00121AE
:1017000001700020704738B50C460546694601F067
:1017100033FB00280DD19DF80010207861F34700BD
:10172000207055F8010FC4F80100A888A4F805003E
:10173000002038BDB401002038B51378C0B10228AC
:1017400016D0F6A46D46246800944C7905EB9414E9
:10175000247864F34703137003280ED003F0FE00CF
:1017600010700868C2F801008888A2F8050038BD2A
:1017700023F0FE0313700228EED1D8B240F001002E
:10178000EEE730B50C46097897B0222902D208203E
:1017900017B030BD28218DF80010ADF80200132AD3
:1017A00003D03B2A01D00720F2E78DF804200BA9D3
:1017B00068460AF05AFD050003D121212046FFF7B3
:1017C00065FE2846E4E700B597B023218DF80010A8
:1017D000ADF802001088ADF804005088ADF806009E
:1017E000D088ADF80A009088ADF808000020ADF868
:1017F0000C00ADF80E000BA968460AF036FD09E6AC
:101800002DE9FF470220C64E8DF804000027708A9C
:10181000ADF80600B84643F202094DE001A80DF00C
:10182000AAF9050006D0708AA8B3A6F81280ADF810
:1018300006803FE0039CA07F01072DD504F1240022
:101840000090A28EBDF80800214604F1360301F095
:10185000A2FF050005D04D452BD0112D3DD0FFDF57
:101860003BE0A07F20F00800A077E07F810861F3D3
:101870000000C10861F34100E07794F8210000F016
:101880001F0084F820002078282827D1292120460D
:10189000FFF7FCFD22E015E040070BD5BDF808007E
:1018A000214604F10E02FFF78EFF05000DD04D45D5
:1018B00010D100257F1CFFB202200DF09DF9401CC5
:1018C000B842ABD8052D12D008E0A07F20F004006C
:1018D000A07703E0112D00D0FFDF0025BDF8060042
:1018E0007082052D05D0284604B0BDE8F087A6F823
:1018F00012800020F8E72DE9F047040000D1FFDF57
:101900002078874E20F00F00801C20F0F00070300F
:10191000207060680178091F1429E6D2DFE801F021
:10192000F00A0B4FEF0B0CEFEF36F00B0BF074F0EF
:101930000B0BF0F0FFDFD8E787883846FFF76EFD26
:10194000050000D1FFDF6078212140F008006070C1
:10195000707C40F0040070742846FFF797FD38460D
:1019600007F0C2FA384603F092FF384605F01DF83A
:101970003946022010F0A1FFA87F20F01000A877C0
:10198000FFF73EFF0028B0D0FFDFAEE7858828468E
:10199000FFF744FD00B9FFDF60688078012800D0C0
:1019A000FFDF60688179284607F00EFC00289CD094
:1019B000617841F0080161706168C88095E78688A8
:1019C0003046FFF72BFD050000D1FFDF6078314680
:1019D00040F0080060706068C088288160680089F5
:1019E000688160684089A881022010F066FF0020AD
:1019F000A875A87F00F0030002289CD1FFF700FF24
:101A0000002898D0FFDF70E780783C2803D00025BD
:101A100002280AD000E00125002720B13C2802D08E
:101A2000022800D0FFDF17B1A3E00127F5E76078B7
:101A3000002D40F008006070707C40F00800707469
:101A40006BD165680221B5F80480AD1C4746384665
:101A50000DF01EF90446032138460DF019F98246AF
:101A6000052138460DF014F98146042138460DF061
:101A70000FF9074604B9FFDFBAF1000F00D1FFDF0D
:101A8000B9F1000F00D1FFDF07B9FFDF22212046A7
:101A9000FFF7FCFC2879012833D00227A07F06211C
:101AA00067F30100A077288B2081688B6081A88B69
:101AB000A08105F1120001F096F920B36879800742
:101AC00000D5FFDF6979E07D61F34700E075D5F867
:101AD0000600A0616889A083062105F10C0001F0D1
:101AE00082F9F8B130794108607861F3470060709D
:101AF000D6F80500C4F80200B6F809001BE045E07E
:101B000049E00127CAE7E07D20F0FE00801CE07577
:101B1000D5F81200A061E88ADDE71DE00302FF01AD
:101B2000B4010020607820F0FE00801C6070E8683E
:101B3000C4F80200288AE080FE48007884F8220079
:101B4000A07F00F00301404607F0C0F9012F03D049
:101B5000022F0ED0FFDFC8E63078032800D0FFDF69
:101B60000021084610F0A9FEBDE8F047012001F071
:101B7000DDB8B078132800D0FFDF0021072010F077
:101B80009CFEBDE8F0471120FFF7E4BB2046BDE80E
:101B9000F04702F0D3B8607840F008006070A4E627
:101BA0002DE9F04705460078914600270209DFF845
:101BB00088A30C463E46012A75D000214FF6FF70DF
:101BC000022A71D0072A0AD00A2A6ED0FFDF00BF8E
:101BD000A9F800600CB127806680002085E6D5F862
:101BE00004C004F1080204F118089CF80060361FD4
:101BF000142E5AD2DFE806F09859594559590A5916
:101C0000593C5A5959C263FA59594DE811270926C6
:101C1000002C7CD0BCF80480A4F80480686880792B
:101C200020729AF81110404621F004018AF8111030
:101C300004210DF048F8052140460DF044F800213C
:101C400040460DF040F8012140460DF03CF80321DC
:101C500040460DF038F8022140460DF034F80621D8
:101C600040460DF030F8072140460DF02CF8AFE764
:101C700001270926F4B3BCF80400A08068688079C5
:101C80000FE012271026BCF80400214601F08CF862
:101C90009EE71C2709266CB3BCF80200A080686888
:101CA0000079207294E7B5E0DFE004E11B27092604
:101CB00004B30420207268684088A08088E79CF8FC
:101CC00002003C2826D0102718260CF1020C8CB1FB
:101CD000BCF80200A080BCF818006082BCF81800B4
:101CE0002082BCF81A00A082BCF81C00E0829CF89C
:101CF000050000E00BE00CF10601FFF71DFD9CF86C
:101D0000040010B10120E07309E00220FBE7A9F80C
:101D1000006062E71B270926002CF8D021729AF890
:101D2000111021F00801B2E01D273726002CEED05B
:101D3000A08069680879491DFFF7FEFC686890F883
:101D40002B00A0756868C0780428E07D13D020F0CF
:101D50000100E07569681F22C97861F34200E075EF
:101D60006968C97A61F3C700E075696840460C315B
:101D70001CF09AF82CE740F00100EAE71D2737260F
:101D8000002CC4D0A0806968481D0B790146184614
:101D9000FFF7D2FC696804F10F0201F10C00CB7A65
:101DA00001461846FFF7C8FC6868807CA075686823
:101DB000C178E07D61F3420020F0F900E0751F2159
:101DC00040461CF00AF903E720271026002C9ED07D
:101DD000A080686804F10902407A20726968CB1C0F
:101DE00088781946FFF7A8FCF2E6FFE704271026DB
:101DF000002C8CD0BCF80200A0806868808820810C
:101E00006868C088608168680089A08168684089C6
:101E1000E081DDE6287A012803D0022814D0FFDF14
:101E2000D6E61F271026002CABD06888A0806889D2
:101E30002081A8896081E889A081288AE0819AF8B8
:101E4000111021F0200122E012271026688800F0EE
:101E5000ABFF002C95D0687800F00700032889D1EB
:101E60009AF8111021F0020111E02A7A062A29D2EB
:101E7000DFE802F00310102121211B270926002C86
:101E8000A5D0A08021729AF8111021F001018AF8E2
:101E900011109DE61B270926002C98D0A080287AD7
:101EA000012806D0032020729AF8111021F01001A9
:101EB000EDE70220F7E74A4621462846BDE8F0470D
:101EC00002F0B7B8FFDF83E610B51B4896B0807804
:101ED000132802D0082016B010BD22208DF8000073
:101EE0000BA968460AF0C1F904460021072010F04A
:101EF000E4FC2046EFE700B50F4897B08078122841
:101F000001D008207BE41E208DF8000000208DF811
:101F100002008DF803000BA968460AF0A6F9002814
:101F2000F0D10021072010F0C8FC1120FFF712FAB1
:101F3000002064E410000020B401002000B5F9483E
:101F400097B00078012814D01B208DF800000020E5
:101F50008DF802000BA968460AF087F9002807D11E
:101F60000021084610F0A9FC012000F0DFFE00204F
:101F700045E4082043E42DE9F041EA4C002740B154
:101F800002281DD0072842D0082800D0FFDFBDE876
:101F9000F081FFF7D3FF0028F9D106F0B4F800284C
:101FA000F5D0017821F00F01891C21F0F0012031DA
:101FB0000170077206F087F8607C40F001001DE0B8
:101FC0008EB23046FFF72AFA050000D1FFDF2878ED
:101FD0002128DCD006F097F890B1017821F00F01AC
:101FE000891C21F0F001103101700221017246803C
:101FF000AF7506F068F8607C40F002006074C6E7D8
:1020000029463046BDE8F0411322FFF7BABBA57858
:10201000122D03D0132D04D0FFDFB8E7FFF76BFFBD
:1020200001E0FFF751FF0028B1D106F06CF800285D
:10203000ADD0017821F00F01891C21F0F001203191
:102040000170122D07D00221017206F03CF8607C6D
:1020500040F01000D2E70121F6E72DE9F0411446E7
:102060000D00074600D1FFDF2878012803D00228A1
:1020700021D0FFDF8BE73846FFF7D0F9060000D10B
:10208000FFDF0220B075207820F00F00801C20F0C8
:10209000F00010302070607840F008006070286810
:1020A000A0606868E060288920829E48417C41F0F9
:1020B000200141746BE73846FFF7B0F9060000D104
:1020C000FFDF69884FF6FF70814209D1AA888242FA
:1020D00006D131463846BDE8F0411322FFF751BB27
:1020E000814201D1A88898B1207820F00F00801C8F
:1020F00020F0F00010302070607840F00800607030
:102100002868A0606868E06028892082002006E0D6
:10211000782300223946022010F032FB0120B075EE
:1021200035E730B5054697B00C46084610F008FC78
:1021300080BB00200121203D072D6ED2DFE805F095
:1021400004264145515D67000021082010F08EFBF8
:1021500010B1112017B030BD24208DF80000D4F844
:102160000200CDF80200A0798DF806000BA96846A0
:102170000AF07BF8050056D10823002211461846C4
:1021800010F0FEFA08284ED0FFDF4CE0606810F037
:1021900019FC08B11020DDE748208DF800002088E8
:1021A000ADF802006088ADF804000BA968460AF09B
:1021B0005CF8050037D1606880B3BDF8301001804D
:1021C00031E0206802F0D6F909E049220AE000BFB8
:1021D0008DF802100CE000BF8DF8020008E0054603
:1021E00021E042228DF800202278D207F4D0EFE7D8
:1021F0000BA968460AF039F8F1E738208DF800009D
:102200002088ADF802006088ADF80400F0E720787F
:1022100028B1A0F11B01E12902D3072503E01B200F
:10222000414900250870284694E730B5054697B027
:102230000C46084610F0A8FB08B110208AE7202DB4
:1022400007D0212D25D0222D23D0232D21D00720CA
:1022500080E72088FFF7E2F820B10078222804D236
:10226000082077E743F2020074E725208DF800008C
:102270002088ADF802000BA9684609F0F6FF002897
:10228000DCD1DDF83210C4F802109DF83610A171CF
:1022900060E706205EE72348001D70472149087467
:1022A00070472048007C00F00100704738B51421C9
:1022B0001C481BF070FE012000F038FD1120FFF7D4
:1022C00049F81949FB20174C0870611D684605F054
:1022D000E2FF9DF80010207961F3470020F0010033
:1022E00020710020A0734FF46170A0810220E07380
:1022F000FFF77BF800B1FFDF00F08EFE01F0D9FCA4
:1023000038BD10B50C463E2120461BF044FEA07F90
:1023100020F00300A077202020700020A07584F812
:10232000230010BDB40100201000002070477CB5D0
:10233000054610F005FB08B110207CBDFE4C211DA8
:1023400060680090A06801902846FFF7DCF900283B
:10235000F3D1FFF74AF80028EFD000996160BDF88B
:10236000041021819DF80610A1727CBD10B50446B1
:1023700010F00AFB08B11020D3E7EF492246087994
:10238000491D4008FFF7D8F90020CAE72DE9F047BA
:102390009CB00D4604004FF0000812D00822FFF751
:1023A00000F900281CD1002609E000BF54F82600DF
:1023B00004A9FFF770F9002812D1761CF6B2AE42DC
:1023C000F4D32F460A2006AD0DF1440A8DF818000B
:1023D00026465146284609F048FF20B143F2032023
:1023E0001CB0BDE8F0874046DFF84C8388F8030056
:1023F0002EB300244FF00B091DE000BF56F8240057
:1024000005A9FFF748F900B1FFDF9DF81400A87097
:1024100056F8240050F8011FC5F803108088A5F86D
:10242000070085F800905146284609F01EFF00B1CC
:10243000FFDF641CE4B2BC42E0D388F803700020E4
:10244000CEE72DE9F0479EB01546894604001ED020
:102450000F4608222946FFF7A4F8002811D10026CC
:1024600013E000BF54F8260005A9103000F084FCEA
:10247000002806D13FB157F8260010F061FA10B1DC
:1024800010201EB0ADE7761CF6B2AE42EAD30026AD
:10249000A5F101081CE000BF06F1010A0AF0FF07E0
:1024A00012E000BF54F82600017C4A0854F82710B7
:1024B0000B7CB2EB530F05D10622113011311BF00A
:1024C000C7FCC0B17F1CFFB2AF42EBD30AF0FF06DE
:1024D0004645E1DBC8462F46342007AD0DF14809DB
:1024E0008DF81C0026464946284609F0BEFE28B154
:1024F00043F20420C5E743F20520C2E796B3002467
:102500002CE000BF56F82400A91C103000F034FC69
:1025100000B1FFDF56F82400102250F8111FC5F853
:1025200003108088A5F8070056F8241005F109006B
:102530001BF0BAFCB8F1000F15D058F82410102287
:1025400005F119001BF0B0FC3220287049462846DE
:1025500009F08BFE00B1FFDF641CE4B2BC42D1D3B2
:10256000012206E004E005F1190001F0F7FFEBE7B6
:1025700000224946284600F02AFC002081E770B579
:1025800096B0044610F0DCF918B9606810F023FA30
:1025900010B1102016B070BD60884AF2B8118842A0
:1025A00005D82078644D6E4618B1012804D0072064
:1025B000F0E7FEF71AFF1AE06078022804D003283B
:1025C00002D043F20220E5E7E87317208DF80000FF
:1025D000E97B0020CDF80200ADF80600022932D0D8
:1025E00003292DD0FFDF0BA9684609F03EFE002825
:1025F000D0D1606801F0A5FF207870B101208DF87E
:102600000200F01C01F0AAFF4B208DF800000BA97E
:10261000684609F02AFE00B1FFDF6088A8B1A881F2
:1026200080B2ADF8020030208DF800000BA968469A
:1026300009F01BFE00B1FFDF2078A8730020A9E796
:102640008DF80700CFE74020FAE74FF46170E6E726
:1026500010B5044610F098F920B9606838B110F050
:10266000B1F908B110205CE6606801F077FF3248EC
:1026700081896180C17B6170807B2070002050E681
:102680002DE9F0419CB0054600208DF864008DF8DE
:1026900060008DF830008DF868001E4614468846AC
:1026A000284610F098F918B9204610F094F910B1A6
:1026B00010201CB06BE455EA040018D01F270CABA7
:1026C00019AA414628460097FEF787FF0028F0D157
:1026D0001AAB18AA314620460097FEF77EFF002865
:1026E000E7D19DF86000C00703D00A20E1E707208A
:1026F000DFE701AF7DB11A208DF804008DF8068068
:1027000042462946F81C1BF0CFFB0DA901A809F091
:10271000ACFD0028CDD194B120208DF804008DF8B7
:10272000066032462146F81C1BF0BEFB0DA901A82D
:1027300009F09BFD002801E0B4010020B9D1FF4958
:102740009DF8300048700020B3E72DE9F0439BB0BE
:102750004FF00008FAA104468DF83480D1E9000159
:10276000CDE91901204610F0EBF890B92078012846
:1027700003D1606810F0E4F858B9F04D4FF001094A
:10278000A87B50B1E87B022807D1606810F023F9DC
:1027900018B110201BB0BDE8F0832878012801D0C3
:1027A0000820F7E707200CF02FFA18B9207848B175
:1027B000012807D0FEF7E8FD30B1687C10F00C0F5F
:1027C00008D103E01220E5E71320E3E7C10701D1B8
:1027D000800701D51120DDE7608943F6E172A0F1A1
:1027E00020019142217807D301297CD100287AD198
:1027F000A189002977D10FE0022901D0032901D155
:10280000A02870D3012907D06978C90704D0A1890D
:10281000002968D0B42966D8217831B1012908D0BF
:10282000022904D003295ED10AE0002609E002262D
:1028300007E008B9A08908B1042609E0012607E0ED
:102840000326A87B50B1E87B022807D1606828B135
:102850000DA96068FEF71FFF00289BD1207A30B1D8
:10286000012806D0022806D003286DD105E00027F4
:1028700004E0012702E0022700E003270EB1022E48
:102880000ED16FB1E87870B36878800702D043F258
:1028900001207FE7022E03D1022F55D0032F53D002
:1028A00018208DF838006089ADF83A006089ADF8DD
:1028B0003C008DF83E600DF13F00FEF70FFF00B1C8
:1028C000FFDF9DF834008DF840002078012806D005
:1028D000A87B68B1E87B02280AD1606840B16068D3
:1028E00050F8011F00E02FE0CDF84110808802E091
:1028F0004046CDF84180ADF845008DF84870A07B8A
:10290000C0F34002014662F35F01C0F3800041EA78
:10291000800019A9085C8DF84700A8B169460EA887
:1029200009F0A3FC0028B4D11B208DF838008DF8E5
:102930003A9069460EA809F098FC0028A9D19DF8A4
:1029400001001B2819D101E0072023E7052E09D239
:10295000DFE806F0030305050300032000E0022082
:1029600000F0E4F9012E0AD0A08940B100228300D2
:10297000114610460FF004FF08B103200AE70020BB
:1029800008E72DE9FC4107460D460326084610F0EE
:1029900022F8002864D13846FEF740FD040005D037
:1029A0002078222805D20820BDE8FC8143F20200ED
:1029B000FAE7A07F00F0030C2DB129466046FEF730
:1029C000BAFD0600F0D15D48BCF1010F05D0BCF1A5
:1029D000020F17D0FFDF3046E6E7A27D2946012A25
:1029E00002D0407C800701D51120DDE729B9684677
:1029F00000F01FFC0028D7D16946384606F067FB77
:102A00000646E8E7A17D022914D1407C800611D456
:102A100025B1A07F40070BD4002100E001213846FA
:102A200006F09DFB0600D6D1A075002DD3D002E0A4
:102A30001126D0E7A5B12A4621463846FEF7C3FE47
:102A400006461128C7D1A07F4107C4D4296844F89D
:102A50000E1F6968616040F0040020740026BAE728
:102A60001020A1E770B50C460546FEF7D7FC010023
:102A700005D022462846BDE87040FEF782BE43F2EC
:102A8000020070BD00B597B03F218DF800108DF8A1
:102A900002000BA9684609F0E8FB17B000BD01234E
:102AA000FEF7BFBC00231A461946FEF7BABC30B584
:102AB00097B004460FF044FF10B1102017B030BD9E
:102AC000204600F047F90028F8D11C4DA8781128BD
:102AD00001D00820F2E7FEF757FC20B1687CC00661
:102AE00003D51120EAE71320E8E72078800701D515
:102AF000E87848B31D208DF800002078022200F00D
:102B000001008DF802006088ADF80400A088ADF8DF
:102B100006002078C0F3400102EA500001438DF81E
:102B2000091002A8FEF7DAFD00B1FFDF0BA9684625
:102B300009F09BFB0028C1D11E2006E0B401002053
:102B4000070605040302010017E08DF800000120CC
:102B50008DF8020000208DF803000BA9684609F0EB
:102B600084FB0028AAD1E08800F010F90400A5D168
:102B70001220FEF7EFFB2046A0E707209EE7F0B506
:102B800097B015460C4607460FF025FF38B920468A
:102B90000FF0D6FE18B928460FF0D2FE10B1102063
:102BA00017B0F0BD974E707C10F0180F01D14007A0
:102BB00001D51120F4E7204600F0CCF80028EFD131
:102BC00029460220FEF7B7FC0028E9D1B078112889
:102BD00003D0122801D00820E2E72078C0F340019A
:102BE000394311D0800700D577B906200CF00CF8D6
:102BF00040B12078800701D5F07828B1B07812284C
:102C000004D007E01220CBE70720C9E7FFF773F9EC
:102C10000028C5D1FEF7B8FB022801D21320BFE778
:102C200021208DF800006088ADF80200A088ADF882
:102C300004002078C0F340008DF80600207880075B
:102C400016D43878420808D0012A18D043F202215D
:102C5000022A18D0032A18D115E0C00700D002209C
:102C60008DF8070057F8010F0290B888ADF80C00F6
:102C70000DF10E00FEF732FD58B1032090E7C007BA
:102C800005D00320ECE7C00701D0084688E7012003
:102C9000E6E72888ADF810006888ADF81200A8882B
:102CA000ADF81400E888ADF816000020ADF8180063
:102CB000ADF81A000BA9684609F0D7FA00288BD1A5
:102CC000E08800F063F8040086D11320FEF742FB91
:102CD000204665E730B5054697B00C4608460FF02C
:102CE00053FE08B11020E9E62846FEF797FB38B1FD
:102CF0000178222902D3807F800604D40820DDE6F3
:102D000043F20200DAE613208DF80000ADF802501D
:102D10000BA9684609F0A9FA0028E4D19DF9321000
:102D20007F2901D02170C9E60520C7E630B5354DB1
:102D3000040008D0012C04D0022C06D0032C04D0AF
:102D4000FFDF2C7030BDFFDFFBE728780128F8D0CB
:102D5000FFDFF6E7418843F6FD730A1F9A4209D266
:102D60008088042806D3B0F5804F03D8884201D864
:102D700000207047072070470278520804D0012ACB
:102D800002D043F202207047FEF785BC10B548B16F
:102D900083000022114607200FF0F2FC072801D023
:102DA000032060E400205EE470B50C0006460DD000
:102DB000FEF734FB050000D1FFDFA68028892081C3
:102DC000288960816889A081A889E08170BD10B5DB
:102DD00002F0010282703122027009F046FA0028E6
:102DE00000D0FFDF3FE410B500231A4603E0845C07
:102DF0002343521CD2B28A42F9D30BB1002032E4F1
:102E0000012030E4B40100204FF0E0224FF40041F3
:102E10000020C2F880112049087020499002086003
:102E2000704730B51C4D04462878A04218BF002CCE
:102E300002D0002818BFFFDF2878A04208BF30BDAD
:102E40002C701749154A0020ECB1164DDFF858C018
:102E5000131F012C0DD0022C1CBFFFDF30BD0860FA
:102E600003200860CCF800504FF400001060186098
:102E700030BD086002200860CCF800504FF0407070
:102E80001060186030BD086008604FF0607010601E
:102E900030BD00B5FFDF00BD1A00002008F501407D
:102EA00000F500401C03002014F50040094810B54F
:102EB00004680A49084808600EF0FDF908480460F3
:102EC00010BD0849002008604FF0E0210220C1F841
:102ED0008002704710050240010000011805024001
:102EE00014050240FC1F004010B50D2000F06FF8E3
:102EF000C4B26FF0040000F06AF8C0B2844200D09F
:102F0000FFDF3A490120086010BD70B50D2000F0C8
:102F100048F8374C0020C4F800010125C4F80453D8
:102F20000D2000F049F825604FF0E0216014C1F851
:102F3000000170BD10B50D2000F033F82C480121C0
:102F400041600021C0F80011BDE810400D2000F0E4
:102F500033B8284810B50468264927480831086066
:102F60002349D1F80001012804D0FFDF2148001DCA
:102F7000046010BD1D48001D00680022C0B2C1F8E9
:102F800000210FF0A8F9F1E710B51948D0F80011A9
:102F90000029FBD0FFF7DDFFBDE810400D2000F059
:102FA0000BB800F01F02012191404009800000F1A0
:102FB000E020C0F88011704700F01F02012191400D
:102FC0004009800000F1E020C0F88012704700281E
:102FD00006DA00F00F0000F1E02090F8140D03E095
:102FE00000F1E02090F800044009704704D500404B
:102FF00000D00040100502400100000170477047FA
:1030000018FFFFFFDBE5B15100F001008C00FFFF6E
:1030100084000000C0C62D00FE4800210160416010
:1030200070472DE9F743044692B091460120FFF71F
:1030300035F960680FF0C6FC58B160680FF0CBFC42
:1030400038B9607800F00300022802D10020FFF7B1
:1030500025F94D4648460FF073FC18B1102015B005
:10306000BDE8F08329460120FEF765FA0028F6D175
:1030700001258DF842504FF4C050ADF840000022B9
:1030800010A9284603F035FF0028E8D18DF84250FA
:103090004FF42850ADF8400000261C2168460796E2
:1030A0001AF09BFF9DF81C0007AF20F00F00401C9A
:1030B00020F0F00010308DF81C0020788DF81D00F5
:1030C00061789DF81E000DF1400861F3420040F068
:1030D00001008DF81E009DF8000008AA40F00200D3
:1030E0008DF800002089ADF83000ADF832606089BD
:1030F000ADF834000B9760680E900AA9CDF82880CF
:10310000684603F0F5FC0028A9D1C24CBDF82000A8
:1031100008AA20808DF8425042F60120ADF8400008
:103120009DF81E000AA920F00600801C20F0010076
:103130008DF81E000220ADF83000ADF8340013A861
:103140000E90684603F0D4FC002888D1BDF820001A
:103150006080211D484600F032F9002887D18DF8A3
:10316000425042F6A620ADF840001C216846079662
:103170001AF033FF9DF81C00ADF8345020F00F001A
:10318000401C20F0F00010308DF81C009DF81D0050
:1031900008AA20F0FF008DF81D009DF81E000AA966
:1031A00020F0060040F00100801C8DF81E009DF804
:1031B00000008DF8445040F002008DF80000CDE989
:1031C0000A8711A80E90ADF83050684603F090FCC5
:1031D000002899D1BDF82000E08000203FE73EB5EF
:1031E00004460820ADF8000020460FF0A9FB08B106
:1031F00010203EBD21460120FEF79DF90028F8D1A0
:103200002088ADF804006088ADF80600A088ADF80D
:103210000800E088ADF80A007E4801AB6A46808865
:10322000002104F061F8BDF800100829E1D0032066
:103230003EBD1FB50446002002900820ADF80800EE
:10324000CDF80CD020460FF07BFB10B1102004B05D
:1032500010BD704802AA81884FF6FF7004F029FA69
:103260000028F4D1BDF80810082901D00320EEE7AA
:10327000BDF800102180BDF802106180BDF8041077
:10328000A180BDF80610E180E1E701B582B002201F
:10329000ADF800005F4802AB6A464088002104F0A8
:1032A00023F8BDF80010022900D003200EBD1CB584
:1032B000002100910221ADF8001001900FF064FB95
:1032C00008B110201CBD53486A4641884FF6FF7074
:1032D00004F0EFF9BDF800100229F3D003201CBD63
:1032E000FEB514460E460746FEF7DBFF28B1304612
:1032F0000FF026FB18B11020FEBD0F20FEBDF82CEC
:1033000001D90C20FEBD38460FF01AFB414D18BB09
:10331000288801A903F05BF90028F3D138788DF8EB
:103320000500288801A903F0C1FF0028EAD1009018
:103330009DF800009DF8051040F002008DF8000097
:10334000090703D040F008008DF80000288869467E
:1033500003F04AFF0028D5D1ADF80840288833464D
:1033600002AA002103F0C0FFBDF80810A142C9D095
:103370000320FEBD7CB50546002000900190088822
:10338000ADF800000C46284601950FF01BFB18B95C
:1033900020460FF0F9FA08B110207CBD15B1BDF838
:1033A000000050B11B486A4601884FF6FF7004F0D8
:1033B00080F9BDF8001021807CBD0C207CBD30B5AB
:1033C00093B0044600200D460090142101A81AF085
:1033D00004FE1C2108A81AF000FE9DF80000CDF89C
:1033E00008D020F00F00401C20F0F00010308DF8C5
:1033F00000009DF8010020F0FF008DF801009DF80D
:10340000200040F002008DF8200001208DF84600D9
:1034100002E000001200002042F60420ADF8440053
:1034200011A801902088ADF83C006088ADF83E00FE
:10343000A088ADF84000E088ADF842009DF8020099
:1034400006AA20F00600801C20F001008DF8020082
:103450000820ADF80C00ADF810000FA8059001A9E8
:1034600008A803F045FB002803D1BDF81800288008
:10347000002013B030BD000010B504460FF060FA14
:1034800008B1102010BD2078C0F30210042807D81E
:103490006078072804D3A178102901D8814201D28D
:1034A000072010BDE078410706D421794A0703D4EC
:1034B000000701D4080701D5062010BD002010BD6B
:1034C00010B513785C08C37F64F30003C3771478E6
:1034D000A40864F34103C3771078C309887863F3C1
:1034E0004100887013781C094B7864F347134B70C4
:1034F0001378DB0863F3000088705078487110BDC2
:1035000010B5C4780B7864F300030B70C4786408BA
:1035100064F341030B70C478A40864F382030B7056
:10352000C478E40864F3C3030B700379117863F380
:103530000001117003795B0863F341011170037995
:103540009B0863F3820111700079C00860F3C30126
:10355000117010BD70B514460D46064604F0D3FD3B
:1035600080B10178142221F00F01891C21F0F001B3
:10357000A03100F8081B21461AF0DBFCBDE87040C2
:1035800004F0A1BD29463046BDE870401322FEF785
:10359000F8B870B514460E46054604F0B4FD70B197
:1035A000017821F00F01891C21F0F0012031017018
:1035B000458021688160BDE8704004F084BD3146DB
:1035C0002846BDE870401322FEF7DBB810B5FE4C6C
:1035D00094F8300000280CD104F120014FF6FF725E
:1035E000A1F110000CF0A3FF00B1FFDF012084F86F
:1035F000300010BD2DE9F047064608A8894690E83E
:1036000030041F469046142128461AF0E6FC00219B
:10361000CAF80010B8F1000F03D0B9F1000F03D1C0
:1036200014E03878C00711D020680FF0ADF9E8BB7E
:10363000B8F1000F07D120681230286020681430DC
:1036400068602068A8602168CAF800103878800790
:1036500028D560680FF0B6F940BBB9F1000F2DD046
:10366000FEF719FE0168C6F8B4118188A6F8B811F2
:10367000807986F8BA01FFF7A9FFDFF84C8308F1DB
:103680002008C5F80C80626862B196F8B40106F2B1
:10369000B51140081032FEF74FF81022414660681D
:1036A0001AF002FC3878400712D500E003E0A06869
:1036B0000FF06AF950B11020BDE8F087606800286B
:1036C000F9D0E8606068C6F8B001EBE7A06828614F
:1036D0000020F1E730B5054608780C4620F00F00D1
:1036E000401C20F0F001103121700020607095F82E
:1036F000230030B104280FD0052811D0062814D09B
:10370000FFDF20780121B1EB101F04D295F82000D3
:1037100000F01F00607030BD21F0F000203002E0AA
:1037200021F0F00030302070EBE721F0F000403065
:10373000F9E710B510B190F8A94044B1A24890F84B
:10374000354000205CB108601060186010BD00F1C9
:10375000A8040C6000F1D001F8301160F5E79A4C34
:1037600034340C60F0E700B58BB00723CDE90212CA
:103770008DF801300191944900236431059109933A
:1037800001468DF8103068460CF0A9FE002800D0E4
:10379000FFDF0BB000BD30B597B00C462C251A9951
:1037A0008DF80050ADF80200B3B118680190586868
:1037B0000290ADF80C2010220DF10E001AF074FBEF
:1037C0000BA9684608F051FD002803D1A17F41F004
:1037D0001001A17717B030BD00200190E8E72DE976
:1037E000F0470646008A8CB080B20D468146FDF750
:1037F00015FE0446744F3078283FDFF8CC814FF037
:10380000000A122873D2DFE800F072E93509367732
:103810007E98A8F3E7E6E5E4E35BE3E3A07F00F04E
:103820000300012806D0002148460BF03AFA0500B3
:1038300003D101E00121F7E7FFDF98F85C100906EA
:1038400002D5D8F860000BE0032105F121000EF04D
:1038500023FDD5F821005D49B0FBF1F201FB120018
:10386000C5F8210070686866B068A86620782528C9
:1038700000D0FFDFECE0A07F00F00300012806D0BD
:10388000002148460BF00DFA060003D101E00121AA
:10389000F7E7FFDF7078810702D52178252904D06A
:1038A00040F0010070700CB006E70220287096F816
:1038B0002000287106F121003136C5E90206F2E741
:1038C000A07F00F00300012806D0002148460BF03D
:1038D000E8F9040003D101E00121F7E7FFDF607898
:1038E000C10605D51320287041346C60DBE7DEE1AA
:1038F00040F008006070D6E73348082128380EF001
:10390000CBFC032016E02A208DF8000010220DF1D8
:10391000020071681AF0C8FA10220DF11200B168A5
:103920001AF0C2FA284968462C3908F09EFC00B10A
:10393000FFDF042028706F60B5E7E07FC00600D588
:10394000FFDFB0680090B38806220321484605F0E7
:1039500024FB0028A7D0FFDFA5E704B9FFDF7168CB
:1039600021B1102204F124001AF09EFA28212046E9
:10397000FDF78CFDA07F00F0030002280ED104F1BA
:103980002400002300901A4621464846FFF703FF13
:10399000112807D029212046FDF778FD307A84F8D8
:1039A000200080E7A07F000700D5FFDF14F81E0F7E
:1039B00040F008002070A4F816A0C4F818A0C4F8BD
:1039C0001CA0617808460AE01402002040420F0063
:1039D00030E068E196E08CE062E009E03FE061F30E
:1039E0008200410861F3C3006070307AE0705AE7EA
:1039F000A07F00F00300012806D0002148460BF00C
:103A000050F9040003D101E00121F7E7FFDF0221B3
:103A100004F175000EF040FC1020287004F5DA70F7
:103A20006860B4F875002882FA486C346C61C5E9A6
:103A3000028038E7A07F00F00300012805D00021B4
:103A400048460BF02EF918B901E00121F8E7FFDF35
:103A50000CB0324621464846BDE8F0477AE504B945
:103A6000FFDF207821289CD93079012802D0022854
:103A70000AD103E0E07F40F01000E07798F85C1096
:103A800041F0010188F85C10324621464846FFF7B4
:103A900061FD0CB02046BDE8F0472321FDF7F6BCE0
:103AA000327901230321484605F086F878B11120C8
:103AB0002870327905F10800AA80031D00900321C7
:103AC000484605F0F6F8002891D0FFDFEBE6A07F2E
:103AD00000F00300012806D0002148460BF0E1F871
:103AE000040003D101E00121F7E7FFDF3079207006
:103AF000D9E60321484605F0FDFB002899D11220A4
:103B00002870D0E6A07F00F00300012806D0002135
:103B100048460BF0C6F8050003D101E00121F7E7A4
:103B2000FFDF95F8740000F00300012878D1A07F32
:103B300000F00307E07FC0F3400616B1012F04D068
:103B40002BE095F89000C0072AD0D5F8AC1119B336
:103B500095F87320087C62F387000874E27FD5F83B
:103B6000AC1162F341000874D5F8AC1166F30000A3
:103B70000874AEB1D5F8AC01102204F124017835F7
:103B80001AF092F9287E40F001002876287820F07B
:103B9000010005F8780900E016B1022F04D02CE0EE
:103BA00095F87800C00726D0D5F8A81119B395F874
:103BB0007320087C62F387000874E27FD5F8A811AF
:103BC00062F341000874D5F8A81166F30000087488
:103BD0008EB1D5F8A801102204F1240178351AF02D
:103BE00063F9287840F0010005F8180B287820F0D8
:103BF000010005F89009022F51D0002000EB400091
:103C000005EBC00090F87800800709D595F86C00A6
:103C1000D5F8B021400805F16D011032FDF78CFD9B
:103C2000052060F3070815F8740F00F0030060F337
:103C30000F28287960F31748287F60F31F687548BC
:103C40005C38027822F00F02921C22F0F00220323F
:103C50000270427822F00702D21C4270A0F8029053
:103C6000C0F8088004F0B7FB2078252805D021286B
:103C700007D0FFDF2078222803D922212046FDF734
:103C800005FCA07F00F0030001280AD0002148466F
:103C90000BF019F800283FF412AEFFDF03E6012015
:103CA000ACE70121F3E7716881F801A0FBE5FFDFD4
:103CB000F9E570B5574C0025103C14F85C0F20F066
:103CC0008000207065600CF0D2FB5249A1F1100019
:103CD00004F013FB04F82C5C062060724D487C3025
:103CE00020615030A0611030E06170BD70B50D46AC
:103CF000FDF794FB040000D1FFDF4FF4DE7128468E
:103D00001AF06BF943485430686104F124002861CB
:103D1000A07F00F00300012808D0022105F5907073
:103D20000CF0A6FB002800D0FFDF70BD0121F5E7F5
:103D30000A46014602F590700CF0BABB70B5054614
:103D400040689CB0017808290DD00B2903D00C29BC
:103D500036D101218171686886883046FDF75EFBA7
:103D6000040035D133E046883046FDF757FB0400A8
:103D700000D1FFDF2078212822D0282822D16868AE
:103D800002210C3001F0B8F9E0B168680821001D8B
:103D900001F0B2F9B0B12D208DF80000ADF802604D
:103DA000102204F1240101A81AF07EF80BA968463C
:103DB00008F05BFA00B1FFDF29212046FDF766FB22
:103DC0001CB070BD687840F008006870F8E7FFDF4D
:103DD000A07F00F00301022902D120F01000A0779B
:103DE000207821280AD06868817909B1807898B153
:103DF000A07F00F0030002285BD0FFDFA07F00F06F
:103E000003000228DCD1FDF7FBFC0028D8D0FFDF3F
:103E1000D6E7000024020020687840F008006870AF
:103E2000E07FC10720D0800701D5062000E00520F3
:103E300084F823002078292818D02428DED13146A0
:103E400006200EF03AFD22212046FDF71FFBA07F41
:103E500000F0030001282AD0002130460AF033FF89
:103E60000028CBD0FFDFC9E70420E1E7A07F00F006
:103E70000300012806D0002130460AF012FF050099
:103E800003D101E00121F7E7FFDF25212046FDF7FF
:103E9000FDFA0F208DF8580016A905F590700CF06A
:103EA000FEFA0228AAD00028A8D0FFDFA6E7012149
:103EB000D3E7687840F0080068709FE72DE9F04389
:103EC0008BB09946154688460646FDF7A7FA0400CA
:103ED0004ED0207822284BD3232849D0E07FC0063B
:103EE00046D4A07F00F00300012806D00021304610
:103EF0000AF0D7FE070002D00BE00121F7E7A07F10
:103F000000F00300012804D1012130460AF0C0FE70
:103F1000074601AB02AA03A93846FFF70AFC03983B
:103F200000B9FFDF4FB1039807F5907787612078DC
:103F3000222806D0242804D007E0039900208861B5
:103F400003E025212046FDF7A1FA03980B214170DB
:103F500046628580C0E90289029901610199416147
:103F600004A90CF0BCFA022802D0002800D0FFDF20
:103F70000BB0BDE8F08330B587B00546FDF74EFACB
:103F8000017822292FD9807F00F00300012806D074
:103F9000002128460AF085FE040003D101E001213A
:103FA000F7E7FFDF227801230321284604F004FE0F
:103FB000002818D011208DF80400227803A8009062
:103FC000ADF8082004AB0321284604F072FE00B1CE
:103FD000FFDF01A904F590700CF061FA022802D00D
:103FE000002800D0FFDF07B030BD10B586B0044612
:103FF000FDF714FA0178222919D9807F00F0030017
:10400000012806D0002120460AF04BFE040003D10F
:1040100001E00121F7E7FFDF12208DF8000069467B
:1040200004F590700CF03BFA002800D0FFDF06B0DA
:1040300010BD2DE9F05F05460C460027007890463C
:1040400001093E46BB4604F1080A02297ED0072931
:1040500002D00A2909D142E068680178082905D010
:104060000B292CD00C292AD0FFDFC6E114271C26EF
:10407000002C6CD04088A080FDF7D0F95FEA0009E1
:1040800000D1FFDF99F817005246400809F11801E6
:10409000FDF752FB68688089208268684168C4F82F
:1040A00012108068C4F81600A07E20F0060040F0D0
:1040B0000100A07699F81E0040F040014DE01A275B
:1040C0000A26002CD5D08088A080FDF7A7F905002E
:1040D00000D1FFDF51462846FFF7FCFA8DE10CB115
:1040E000288BA080287A0E287ED006DC01287CD080
:1040F000022808D0032804D135E0102876D01128F2
:1041000075D0FFDF79E11E270926002CB1D0A088E9
:10411000FDF784F95FEA000900D1FFDF287B00F09A
:1041200003000128207A1BD020F001002072297B97
:10413000890861F341002072297BC90861F382007C
:104140002072297B090961F3C30001E04AE117E10C
:10415000207299F81E0040F0800189F81E104CE191
:1041600040F00100E2E713270D26002CAAD0A0881A
:10417000FDF754F98146807F00F00300012806D046
:104180000021A0880AF08DFD050003D101E0012186
:10419000F7E7FFDF99F81E0000F00302012A59D06B
:1041A000A86E817801F003010129217A54D021F011
:1041B0000101217283789B0863F3410121728378A6
:1041C000DB0863F38201217283781B0963F3C30167
:1041D0002172037863F306112172437863F3C711E8
:1041E000217284F809B003E05EE0A4E08CE09CE07A
:1041F000C178A172012A32D04279E17A62F30001DA
:10420000E1724279520862F34101E1724279920807
:1042100062F38201E1724279D20862F3C301E17272
:104220000279217B62F3000121730279520862F363
:10423000410121730279920862F3820121730079AE
:10424000C00860F3C301217399F8000023285AD9EC
:10425000262168E0686EA4E741F00101A9E7027930
:10426000E17A62F30001E1720279520862F34101DE
:10427000E1720279920862F38201E1720279D20856
:1042800062F3C301E1724279217B62F30001217381
:104290004279520862F3410121734279920862F334
:1042A000820121734079CBE718271026002C67D0B4
:1042B000A088FDF7B3F88246807F00F00300012854
:1042C00007D00021A0880AF0ECFC5FEA000903D1C6
:1042D00001E00121F6E7FFDFE868A06099F801003E
:1042E00040F0040189F8011099F80200800708D510
:1042F000012020739AF8000023287ED927215046F8
:1043000063E084F80CB078E015270F26C4B3A088CA
:10431000FDF784F8814606225146E86808F00DF85A
:104320000120A073AEE048464FE0162709263CB3B3
:10433000287B207261E0297BFE4802290CD01927D6
:104340000E26ECB101290DD003291AD004291BD067
:10435000052919D0FFDF23E01B270926BCB3012163
:10436000217205E001212172617A21F0030161725D
:1043700010F85C1F4A08520062F3060101700FE05A
:104380002BE00220207207E0687B052900F00F0077
:1043900040F0800020721BD0607A20F00300607231
:1043A000A088FDF73BF805460078212825D0232872
:1043B00000D0FFDFA87F00F00300012810D000210B
:1043C000A0880AF080FC22212846FDF75FF814E05F
:1043D000607A20F00300401CE1E7A8F8006011E0DB
:1043E0000121EDE70CB16888A080287A03282BD042
:1043F00004280AD005284BD0FFDFA8F800600CB1D4
:10440000278066800020BDE8F09F15270F26002C2E
:10441000E3D0A088FDF702F8807F00F003000128B8
:1044200006D00021A0880AF03CFC050003D101E081
:104430000121F7E7FFDFD5F821000622514607F0FA
:104440007CFF84F80EB0D8E717270926002CC4D0CB
:10445000A088FCF7E3FF8146807F00F0030001287D
:1044600006D00021A0880AF01CFC050003D101E061
:104470000121F7E7FFDFA878800701D5022000E0DF
:104480000120207299F800002328B6D927214AE795
:1044900019270E26002CA0D0A088FCF7BFFF5FEAEA
:1044A000000900D1FFDFC4F808B0A4F80CB084F80C
:1044B00008B0A07A40F00300A07299F81F1061F3D1
:1044C0008200A07299F81F1001EA510161F3C30044
:1044D000A072687A00F0030001288ED1607A40F063
:1044E0000400607299F81E00E97A00F003000128C8
:1044F00013D0607B61F300006073AA7A217B62F3C2
:1045000000012173EA7A520862F341006073A87ACD
:10451000400860F3410121736FE7207B61F30000E5
:104520002073AA7A617B62F300016173EA7A520810
:1045300062F341002073A87A400860F3410161737F
:104540005BE710B57B4C30B10146102204F120002E
:1045500019F0AAFC012084F8300010BD10B5044603
:10456000FFF734F8734920461022BDE8104020318F
:1045700019F09ABC70B56F4C06004FF0000514D0CE
:104580000EF0DEF908B110250DE00621304607F0E7
:10459000BBFE411C06D0206614F85C0F40F0800082
:1045A000207000E00725284670BD14F85C0F20F04D
:1045B0008000F5E7007810F00F0204D0012A05D042
:1045C000022A0CD110E0000909D10AE000090128F3
:1045D00007D0022805D0032803D0042801D00720E3
:1045E00070470870002070470620704705282AD2BF
:1045F000DFE800F003070F171F00087820F0FF0026
:104600001EE0087820F00F00401C20F0F000103071
:1046100016E0087820F00F00401C20F0F000203059
:104620000EE0087820F00F00401C20F0F000303041
:1046300006E0087820F00F00401C20F0F000403029
:10464000087000207047072070472DE9F041804630
:1046500088B00D46002708460EF0BDF9A8B94046BF
:10466000FCF7DCFE040003D02078222815D104E0FA
:1046700043F2020008B0BDE8F08145B9A07F010611
:1046800003D500F00300022801D01020F2E7A07F3C
:10469000C10601D4010702D50DB10820EAE725497A
:1046A00091F85C10C90701D01120E3E7E17FC9064A
:1046B00001D50D20DEE700F00300022805D125B169
:1046C0002846FEF7D9FE0700D4D1A07F00F00300F2
:1046D000012806D0002140460AF0E3FA060002D085
:1046E0000CE00121F7E7A07F00F0030001280BD0C8
:1046F000002140460AF0CCFA060007D0A07F00F067
:104700000300022804D009E00121F2E70420B1E708
:1047100025B12A4631462046FEF7D2FE07AB1A469F
:1047200069463046FFF705F8009800B9FFDF0C2016
:10473000009901E014020020487006F59070C1F85D
:104740002480486100200881A07F00F00300012838
:1047500028D0EDB302200871301D886170784009BF
:104760000877B078C0F340004877287800F001025D
:10477000887F62F301008877E27F62F382008877A6
:10478000E27F520862F3C3008877B27862F30410C4
:104790008877A878C87701F1210228462031FEF7F2
:1047A000AFFE22E001200871287800F00102087EA7
:1047B00062F3010008762A78520862F382000876D4
:1047C0002A78920862F3C30008762A78D20800E0BB
:1047D00007E062F30410087624212046FCF756FE19
:1047E0000BE0032008710520087625212046FCF700
:1047F0004DFEA07F20F08000A07701A900980BF06B
:104800006EFE022801D000B1FFDF384632E72DE905
:10481000FF4FF94A0D4699B09A4607CA14AB0027D4
:1048200083E807001998FCF7F9FD060006D03078F8
:10483000262806D008201DB0BDE8F08F43F2020004
:10484000F9E7B07F00F00309B9F1010F03D0B9F126
:10485000020F07D008E03DB91B98FEF70DFE0028B7
:10486000E9D101E01B9878BBB07F00F0030001287C
:1048700006D0002119980AF014FA040003D101E0CF
:104880000121F7E7FFDF852D25D007DCD5B1812D8C
:104890001BD0822D1BD0832D08D11AE0862D1CD071
:1048A000882D1CD0892D1CD08A2D1CD00F20207162
:1048B0000F281AD001208DF83400201D0E90207989
:1048C000A8B158E10020F2E70FE00120EFE7022055
:1048D000EDE70320EBE70520E9E70620E7E70820FE
:1048E000E5E70920E3E70A20E1E70720A3E7B9F1BC
:1048F000010F17D0D4E91950804602200190012001
:104900000090A87898F80210C0F3C000C1F3C0016D
:1049100008405FEA000B5DD050460EF011F8002809
:104920006CD12DE0D4E9198501200190022000907E
:10493000214630461B9AFEF7C3FD1B98007800F015
:104940000101A87861F30100A870F17F61F3820092
:10495000A870F17F490861F3C300A870A17861F3E2
:104960000410A870607840092870A078C0F3400057
:1049700068701B988078E870002068712871C0E723
:10498000DAF80C000DF0DCFFC0BBDAF81C000DF00B
:10499000D7FF98BBDAF80C00A060DAF81C00E060E2
:1049A00098F80100A17800F0010041EA4000A070F1
:1049B00098F80210C0B2C1F30011891E0840A0701F
:1049C000002084F82000009906F1170002290BD07E
:1049D00001210AE098F80110A07801F00101FD2200
:1049E00042EA41010840E2E7002104EB81018861CD
:1049F0000199701C022902D0012101E028E0002168
:104A000004EB81018861A87800F00300012849D1F6
:104A100098F8020000F00300012843D1B9F1010F1A
:104A200004D12A1D691D1B98FEF76AFD297998F8A3
:104A3000040001408DF82C10687998F8052010408A
:104A40008DF8300001432DD050460DF079FF08B1AC
:104A50001020F0E60AF1100004F5D47104F17C0294
:104A60000490B9F1020F3CD00090CDE90121002162
:104A70000BAB5A462046FEF7BDFD0028E9D104F5F0
:104A8000D67104F19402B9F1010F30D0049800906E
:104A9000CDE9012100210CAB5A462046FEF7AAFDC4
:104AA0000028D6D1A078800740D4A87898F80210C2
:104AB000C0F38000C1F38001084337D0297898F80B
:104AC000000014AAB9F1010F17D032F810204B00E2
:104AD000DA4012F0030718D0012F1ED0022F12D196
:104AE0001DE0CDF800A0CDE901210121C0E7CDF8FE
:104AF00000A0CDE901210121CDE732F811204300CA
:104B0000DA4002F00307032F07D0BBF1000F0DD0EE
:104B1000012906D0042904D008E00227F5E701277F
:104B2000F3E7012801D0042800D10427F07F40F0EA
:104B300001006BF34100F077A07881074FF003008C
:104B40000CD5A071BBF1000F15D100BF8DF85C0032
:104B500017AA31461998FEF71CFD0CE00221022F1E
:104B600018D0012F18D0042F22D00020A071F07F80
:104B700020F00100F07725213046FCF787FC0DA9D5
:104B800004F590700BF08BFC10B1022800D0FFDF11
:104B9000002050E6A171D9E7A1710D2104F1240094
:104BA00019F01BFA607840F0020060700420CDE735
:104BB0000120A071DFE72DE9F04387B091468846D8
:104BC0000446FCF72BFC070006D03878272806D0CF
:104BD000082007B0BDE8F08343F20200F9E7B87F90
:104BE00000F00300012809D0002120460AF059F8FE
:104BF000040006D104E0000060E301000121F4E7B5
:104C0000FFDFA679012E08D0B8F1000F0FD048467B
:104C10000DF096FEB8B11020DBE7B9F1000F25D1F9
:104C2000B8F1000F09D0B8F1010F1FD120E0022E1A
:104C300005D0032E05D0FFDF28E00C2526E0012556
:104C400024E0022522E0B8F1020F03D0B8F1010FF1
:104C50000AD00BE0032E09D100251022494604F1A9
:104C6000210019F021F911E0022E01D00720B0E750
:104C70000025102104F1210019F08DF95FEA0900E7
:104C800004D0062107F040FBC4F8210060782521FC
:104C900040F0020060703846FCF7F8FB6078C1070E
:104CA00013D020F00100607002208DF8000004F1A4
:104CB000210002908DF804506946FF300BF0EFFBA5
:104CC000022804D018B1FFDF01E084F82050002052
:104CD0007FE730B587B00D460446FCF79FFB88B1EF
:104CE000807F00F0030001280FD00021204609F04A
:104CF000D8FF04000ED028460DF022FE38B1102057
:104D000007B030BD43F20200FAE70121EEE7607818
:104D1000400701D40820F3E7294604F1410020228E
:104D2000054619F0C1F8607840F010006070010786
:104D30000FD520F00800607013208DF80000694640
:104D400004F5907001950BF0AAFB022801D000B188
:104D5000FFDF0020D4E770B592B00D460646FCF7A1
:104D60005DFB18B10178272940D103E043F202002E
:104D700012B070BD807F00F00300012806D0002132
:104D8000304609F08EFF040003D101E00121F7E76E
:104D9000FFDFA079022829D1A078C00726D0002300
:104DA00002220321304603F007FF08B30C208DF8E0
:104DB00005000A9604A804F5907402220090069457
:104DC000ADF80C2005AB0321304603F072FF00B1B3
:104DD000FFDF04208DF808008DF81C500BA901A8F6
:104DE0000BF07DFB00B1FFDF0020C1E70820BFE72B
:104DF0001120BDE770B5064686B014460D4608463C
:104E00000DF09EFD18B920460DF0BEFD10B110202A
:104E100006B070BDA6F57F40FF380ED03046FCF7D7
:104E2000FDFA38B1417822464B08811C1846FCF740
:104E300083FC07E043F20200EAE72046FDF796FA1A
:104E40000028E5D11021E01D0DF026FAE21D2946CB
:104E50006846FEF788FC102204F11700019919F04A
:104E600023F80020D4E72DE9F041044690B0154620
:104E70008846002708460DF0AEFD18B928460DF00B
:104E8000AAFD18B1102010B0BDE8F0812046FCF753
:104E9000C5FA060003D03078272818D102E043F283
:104EA0000200F0E7B07F00F00300012806D00021E7
:104EB000204609F0F6FE040003D101E00121F7E7E6
:104EC000FFDF6078400702D5A078800701D4082072
:104ED000D9E7B07F00F00300012818D0D4E9190108
:104EE000407800B1B5B1487810B1B8F1000F11D0D9
:104EF000C5B1EA1D02A8E168FEF735FC102205F1F4
:104F00001700039918F0A4FF30B104270AE0D4E990
:104F10001910E5E70720B6E71022E91D04F131007A
:104F200018F0C2FFB8F1000F06D0102208F10701F7
:104F300004F1210018F0B8FF6078252140F002004C
:104F400060703046FCF7A2FA6078C10715D020F0F7
:104F50000100607002208DF8200004F121000A9009
:104F600010300B908DF8247008A9EF300BF097FAF1
:104F7000022804D018B1FFDF01E084F8207000207F
:104F800081E7F8B515460E460746FCF747FA0400D8
:104F900004D02078222804D00820F8BD43F2020073
:104FA000F8BDA07F00F00300022802D043F2050004
:104FB000F8BD30460DF0C4FC18B928460DF0C0FC11
:104FC00008B11020F8BD00953288B31C2146384640
:104FD000FEF7E1FB112814D00028F3D1297C4A0800
:104FE000E17F62F30001E1772A7C62F34101E1771E
:104FF000297C890884F82010A17F21F08001A17705
:10500000F8BDA17F0907FBD4D6F80200C4F836002A
:10501000D6F80600C4F83A003088A0861022294647
:1050200004F1240018F040FF287C4108E07F61F380
:105030008200E077297C61F3C300E077287C800858
:1050400084F82100A07F40F00800A0770020D3E77B
:1050500070B596B00D46064613B1072016B070BD68
:10506000FCF7DCF9040007D02078222802D3A07FC7
:10507000400604D40820F1E743F20200EEE7C5B190
:105080002D208DF80000ADF802601022294601A8FD
:1050900018F00AFF287C4108E07F61F30000E07708
:1050A000297C61F34100E077287C800884F82000A7
:1050B00004E02E208DF80000ADF802600BA96846D0
:1050C00007F0D3F8A17F21F04001A177C6E770B5C2
:1050D0000D46FCF7A3F9040005D028460DF054FC5A
:1050E00020B1102070BD43F2020070BD2946204659
:1050F000FEF7F0FA002070BD05E000BF10F8012BAC
:105100000AB100207047491E89B2F7D201207047CA
:10511000F0B50078059F1E4614460D46012800D0C4
:10512000FFDF0C2030803A203880002C08D0287A0D
:10513000052806D0287B012800D0FFDF17206081DA
:10514000F0BDA889FBE72DE9F04786B0144691F839
:105150000C900E9A0D46B9F1010F0BD0102100787A
:105160002E8A8846052807D0062833D0FFDF06B0F0
:10517000BDE8F0870221F2E7E8890C2100EB40004E
:1051800001EB4000188033201080002CEFD0E8891C
:10519000608100271AE00096688808F1020301AADE
:1051A000696900F092FE06EB0800801C07EB4701DE
:1051B00086B204EB4102BDF8040090810DF10601B6
:1051C00040460E320BF02CFA7F1CBFB26089B84209
:1051D000E1D8CCE734201080E889B9F1010F11D073
:1051E000122148430E301880002CC0D0E88960811D
:1051F0004846B9F1010F00D00220207300270DF1BD
:10520000040A1FE00621ECE70096688808F1020313
:1052100001AA696900F059FE06EB0800801C86B2FD
:10522000B9F1010F12D007EBC70004EB4000BDF845
:105230000410C18110220AF10201103018F034FE6E
:105240007F1CBFB26089B842DED890E707EB470108
:1052500004EB4102BDF80400D0810AF1020140468E
:1052600010320BF0DDF9EBE72DE9F0470E4688B080
:1052700090F800C096F80C80378AF5890C201099B8
:1052800002F10C044FF0000ABCF1030F08D0BCF18E
:10529000040F3ED0BCF1070F7DD0FFDF08B067E7F9
:1052A00005EB850C00EB4C00188031200880002AAB
:1052B000F4D0A8F1060000F0FF09558125E018217F
:1052C00001A818F08AFE00977088434601AA716908
:1052D00000F0FBFDBDF804002080BDF80600E08072
:1052E000BDF808002081A21C0DF10A0148460BF010
:1052F00097F9B9F1000F00D018B184F804A0A4F810
:1053000002A007EB080087B20A346D1EADB2D6D2F8
:10531000C4E705EB850C00EB4C00188032200880B8
:10532000002ABBD0A8F1050000F0FF09558137E045
:1053300000977088434601AA716900F0C6FD9DF888
:105340000600BDF80410E1802179420860F30001F5
:1053500062F34101820862F38201C20862F3C30171
:10536000020962F30411420962F34511820962F3F2
:1053700086112171C0096071BDF8070020812246A5
:105380000DF1090148460BF04BF918B184F802A061
:10539000A4F800A000E007E007EB080087B20A3499
:1053A0006D1EADB2C4D279E7A8F1020084B205FB4C
:1053B00008F000F10E0CA3F800C035230B80002A82
:1053C000A6D055819481009783B270880E3271699E
:1053D00000F07BFD62E72DE9F84F1E460A9D0C4662
:1053E00081462AB1607A00F58070D080E089108112
:1053F00099F800000C274FF000084FF00E0A0D2816
:1054000073D2DFE800F09E070E1C28303846556A3C
:1054100073737300214648460095FFF779FEBDE897
:10542000F88F207B9146082802D0032800D0FFDFA8
:10543000378030200AE000BFA9F80A80EFE7207B20
:105440009146042800D0FFDF378031202880B9F151
:10545000000FF1D1E3E7207B9146042800D0FFDF65
:1054600037803220F2E7207B9146022800D0FFDF10
:1054700037803320EAE7207B1746022800D0FFDF81
:105480003420A6F800A02880002FC8D0A7F80A80F2
:10549000C5E7207B1746042800D0FFDF3520A6F89B
:1054A00000A02880002FBAD04046A7F80A8012E05A
:1054B000207B1746052802D0062800D0FFDF1020E9
:1054C000308036202880002FA9D0E0897881A7F885
:1054D0000E80B9F80200B881A1E7207B9146072829
:1054E00000D0FFDF37803720B0E72AE04FF012000E
:1054F00018804FF038001700288090D0E08978811C
:10550000A7F80E80A7F8108099F800000A2805D0A7
:105510000B2809D00C280DD0FFDF80E7207B0C285A
:1055200000D0FFDF01200AE0207B0D2800D0FFDF44
:10553000042004E0207B0E2800D0FFDF0520387314
:105540006DE7FFDF6BE770B50C460546FBF766FFBE
:1055500020B10078222804D2082070BD43F2020056
:1055600070BD0521284609F09CFB206008B1002091
:1055700070BD032070BDFFB585B00746089814467E
:105580000D46022628B908A93846FFF7DCFF002897
:1055900040D108980121801D04F074FDADF8080089
:1055A00002464DB100233146384603F005FB98B35F
:1055B0000898007880BB05E02078092820D00F28C3
:1055C0002BD0FFDF03A8009004ABBDF808203146C4
:1055D000384603F06EFB00281CD1089802A9801DF4
:1055E000C4E90107DDE90332204604F058FD40B369
:1055F000072824D2DFE800F01A182323211C1E00FC
:10560000072600233146384603F0D6FA0028D9D1C0
:1056100043F2040009B0F0BD06E0002331463846ED
:1056200003F0CAFA0028CDD11120F3E70020F1E7FA
:105630000820EFE743F20300ECE70720EAE7032046
:10564000E8E703980090BDF8083004223146384658
:1056500003F0A3FC0028DDD1002DDBD008990D70EC
:10566000D8E710B588B01C46AAB104238DF80030E5
:105670001388ADF80C305288ADF80E208A788DF87A
:1056800012200988ADF8101000236A462146FFF762
:1056900072FF08B010BD1020FBE770B50D46052164
:1056A00009F0FFFA040000D1FFDF2946A01DBDE884
:1056B000704004F0D0BC70B596B00C460646FFF7BB
:1056C000ECFF05462146304601F036FE012130460A
:1056D00001F050FE002D25D13046FBF79FFE05005E
:1056E00000D1FFDF95F822001B281BD9172C19D9F0
:1056F0003A208DF80000ADF8026095F82200211DD7
:10570000884201D9241D00E00446ADF8044040F66B
:105710004800ADF806000BA9684606F0A6FD002873
:1057200000D0FFDF16B070BD2DE9F84305460078C4
:1057300000260C4612287BD2DFE800F0896464431F
:105740003B663737133737370937373737372879D5
:10575000001FC0B2022801D010281FD104BBFFDFF8
:105760001EE004B9FFDF6088052109F09AFA00788D
:10577000032805D004280AD0072811D0FFDF0DE048
:105780002879801FC0B202280AD048B106E02879E3
:10579000401FC0B2022803D0102801D0072657E0CE
:1057A000607840F00800607052E0002CF8D1FFDF14
:1057B000F6E704B9FFDF28790128F1D160881721C5
:1057C00042E0A888052180B2804609F06AFA0746BF
:1057D00004B1FFDF07B9FFDF4146B81D04F015FC37
:1057E00002F091FC040008D0607840F0080060707E
:1057F000A4F8028002F067FC2BE013214046FDF77D
:1058000031F937E0FFDF23E004B9FFDF60880521CD
:1058100009F047FA070000D1FFDF6946B81D04F020
:10582000FBFB00B1FFDFA988172902D2172201E094
:105830000DE00A46BDF80000824201D9014602E0AF
:10584000172900D217216088FFF735FFA8E7FFDF8F
:1058500084B1607800070DD52078182220F00F0061
:10586000C01C20F0F00090302070294604F10800A0
:1058700018F05FFB3046BDE8F88300200870881DF3
:1058800004F0B7BB0A460146901D04F0C4BB70B5D6
:105890000546052109F005FA040000D1FFDF29467D
:1058A000A01DBDE8704004F0B0BB2DE9F74F90B0EB
:1058B0004FF0000AADF830A0ADF804A047880C46C0
:1058C00005460521384609F0ECF9060000D1FFDF56
:1058D00024B1A780A4F806A0A4F808A0297A04F1AE
:1058E00010003827C91E4FF00C0B4FF001084FF085
:1058F000120902900F297DD2DFE801F0F1F0EF7F6D
:1059000008D2888D9F3DDBF2EDB6B60030780228D4
:1059100000D0FFDFA8890BEBC001ADF804103021E7
:10592000ADF83010002C25D06081B5F80E8000272E
:105930001DE004EBC709317989F80E107188A9F8C8
:105940000C10CDF800806888042305AA296900F0AE
:10595000BCFABDF81410A9F8101008F10400BDF845
:1059600016107F1C1FFA80F8A9F81210BFB26089C8
:10597000B842DED808E13078022800D0FFDFE9899C
:105980000BEBC100ADF804003020ADF8300095F805
:105990000CB0002CABF10400C0B20F90EAD06181D2
:1059A000B5F81090002722E0CDF8009068885B469B
:1059B00003AA696900F089FA09EB0B001FFA80F964
:1059C00004EBC70808F10C0204A90F980AF028FE9E
:1059D00018B188F80EA0A8F80CA0BDF80C10A8F813
:1059E0001010BDF80E107F1CA8F81210BFB260890D
:1059F000B84200E0C7E0D7D8C6E00CA8009001ABE1
:105A0000224629463046FFF79EFBBDE03078082845
:105A100005D0FFDF03E03078082800D0FFDFE889F9
:105A20001030ADF804003620ADF83000002C3FD027
:105A3000A98961817188A18127E03078092800D087
:105A4000FFDFA88900F10C01ADF804103721ADF893
:105A50003010002C2CD06081E8890090AB896888D8
:105A600004F10C02296955E0E8893921103080B22F
:105A7000ADF80400ADF83010002C72D0A989618116
:105A8000287A10280AD002212173E989E181288A25
:105A90000090EB8968886969029A3BE00121F3E78D
:105AA0000CA8009001AB224629463046FFF7DCFBEC
:105AB0006AE030780A2800D0FFDFADF80490ADF836
:105AC00030704CB3A9896181A4F810A0A4F80EA08D
:105AD00084F80C8058E020E002E030E038E041E05B
:105AE00030780B2800D0FFDF288AADF830701230F4
:105AF000ADF8040084B104212173A9896181E98989
:105B0000E181298A2182688A00902B8A688804F1C1
:105B10001202696900F0D9F936E030780C2800D01B
:105B2000FFDFADF80490ADF8307044B30521217368
:105B3000A4F80AA0A4F80EA0A4F810A024E00CA8D1
:105B4000009001AB224629463046FFF7E1FA1BE000
:105B50000CA8009001AB224629463046FFF73BFCDB
:105B600012E00DE00B203B21ADF80400ADF8301041
:105B700034B1A4F80680A4F808A084F80AA003E0D1
:105B80001299088014E0FFDF1299BDF80400088024
:105B900074B1BDF830002080BDF804006080287A20
:105BA000032805D0102803D0112801D086F800A0C2
:105BB00013B00020BDE8F08F2DE9FC4156880F4658
:105BC000804615460521304609F06BF8040000D1E7
:105BD000FFDFA41DCDE900642B463A4640466968C4
:105BE00004F011FCBDE8FC8170B50D46052109F0FB
:105BF00058F8040000D1FFDF2946A01DBDE8704021
:105C000004F015BA70B50D46052109F04AF80400F4
:105C100000D1FFDF2946A01DBDE8704004F03ABA6C
:105C20002DE9F0438DB00D461446814607A9FFF7D4
:105C30008AFC002814D14FF6FF7601274FF4205834
:105C40008CB103208DF800001020ADF8140008A8D6
:105C5000069008AA204605A90AF001FD78B10720A0
:105C60000DB0BDE8F0830820ADF80C508DF812702F
:105C70008DF80000ADF80E60ADF810800CE00798CC
:105C8000A1780171218841808DF81270ADF80C5017
:105C9000ADF81080ADF80E606A4602214846079BB9
:105CA000FFF769FCDCE708B501228DF8022042F617
:105CB0000202ADF800200A4603236946FFF7D1FC33
:105CC00008BD08B501228DF8022042F60302ADF8A6
:105CD00000200A4604236946FFF7C3FC08BD00B54F
:105CE00087B079B102228DF800200A88ADF80C2027
:105CF0004988ADF80E1000236A460521FFF73BFCEA
:105D000007B000BD1020FBE709B10723A9E4072075
:105D1000704770B588B00D461446064607A9FFF7D0
:105D200012FC00280ED17CB10620ADF80C508DF885
:105D30000000ADF80E40079B6A4608215C803046A3
:105D4000FFF719FC08B070BD05208DF80000ADF814
:105D50000C50F0E700B587B059B107238DF800303B
:105D6000ADF80C20049100236A460921FFF703FCDB
:105D7000C6E71020C4E770B588B00C46064600257B
:105D800007A9FFF7E0FB0028DCD107980121801D5F
:105D900004F078F99CB12178062921D2DFE801F0DE
:105DA000200505160318801E80B2C01EE28880B24E
:105DB0000AB1A3681BB1824203D90C20C2E71020AC
:105DC000C0E7042904D0A08850B901E00620B9E753
:105DD000012913D0022905D004291CD005292AD075
:105DE0000720AFE709208DF800006088ADF80C00AF
:105DF000E088ADF80E00A068049023E00C208DF838
:105E000000006088ADF80C00E088ADF80E00A068D6
:105E10000A25049016E00D208DF800006088ADF88A
:105E20000C00A088ADF80E00E088ADF81000A06866
:105E30000B25059006E00E208DF8000060788DF8A7
:105E40000C000C256A4629463046079BFFF793FB5A
:105E500078E700B587B00F228DF80020ADF80C1060
:105E600000236A461946FFF786FB49E700B587B06D
:105E700071B102228DF800200A88ADF80C20498803
:105E8000ADF80E1000236A460621FFF774FB37E7D2
:105E9000102035E770B588B0064601200D46ADF8F4
:105EA0000C108DF80000014600236A463046FFF7CB
:105EB00062FB040008D12946304601F02EFA002189
:105EC000304601F057FA20463CE7F8B51C46154627
:105ED0000E46069F09F048F82346FF1DBCB2314626
:105EE0002A46009408F060FCF8BD000018B18178E3
:105EF000012938D101E010207047018842F60112D3
:105F0000881A914231D018DC42F60102A1EB02005E
:105F100091422AD00CDC41B3B1F5C05F25D06FF4BB
:105F2000C050081821D0A0F57060FF381BD11CE0CC
:105F300001281AD002280AD117E0B0F5807F14D0CA
:105F400008DC012811D002280FD003280DD0FF282B
:105F500009D10AE0B0F5817F07D0A0F58070033841
:105F600003D0012801D0002070470F2070470B2874
:105F700026D008DC1BD2DFE800F01C2025251A25DE
:105F8000292325271E0011281CD008DC0C2817D037
:105F90000D281DD00F2815D0102808D110E0822818
:105FA00009D0842810D0852810D0872812D003204B
:105FB0007047002070470520704743F20300704788
:105FC000072070470F207047042070470620704755
:105FD0000C2070474FF45050704708280DD2DFE86E
:105FE00000F00406040C0C080C0A00207047112075
:105FF000704707207047082070470320704738B566
:106000000C46050041D06946FEF7D4FA002819D1A4
:106010009DF80010607861F3020060706946681CAA
:10602000FEF7C8FA00280DD19DF80010607861F3E2
:10603000C5006070A978C1F34101012903D002298C
:1060400005D0072038BD217821F0200102E0217819
:1060500041F020012170410704D0A978C90861F3FB
:1060600086106070607810F0380F07D0A9780909A1
:1060700061F3C710607010F0380F02D160784006ED
:1060800003D5207840F040002070002038BD70B566
:1060900004460020088015466068FFF7B0FF00281E
:1060A00016D12089A189884211D860688078C007FC
:1060B0000AD0B1F5007F0AD840F20120B1FBF0F21E
:1060C00000FB1210288007E0B1F5FF7F01D90C20FA
:1060D00070BD01F201212980002070BD10B5047847
:1060E000137864F3000313700478640864F34103C5
:1060F00013700478A40864F3820313700478E4082E
:1061000064F3C30313700478240964F30413137055
:106110000478640964F3451313700078800960F310
:106120008613137031B10878C10701D1800701D5FA
:10613000012000E0002060F3C713137010BD427807
:10614000530702D002F0070306E012F0380F02D026
:10615000C2F3C20300E001234A7863F302024A70EB
:10616000407810F0380F02D0C0F3C20005E04307BA
:1061700002D000F0070000E0012060F3C5024A7081
:1061800070472DE9F04796B00D00804613D0B8F166
:10619000000F14D01221284617F0FDFE06AAFF2199
:1061A000012005F09DFE0024264637464FF4205975
:1061B0006FF4205A78E0102016B0BDE8F087072071
:1061C000FAE700BF9DF8220001280AD1BDF820009F
:1061D00048450BD010EB0A000AD001280CD0022849
:1061E0000CD0042C0ED0052C0FD10DE0012400E0C2
:1061F0000224BDF81E6008E0032406E00424BDF874
:106200001E7002E0052400E00624BDF81E10414582
:106210004AD12C74D6B30DF140094FF0000811AAF1
:10622000CDF81490CDF80880CDE903824FF0070A2D
:10623000CDE900A810234246FF21304605F0FEFEBE
:1062400010BBBDF840002A46C0B211A90AF0E8F917
:10625000D0B9AE81D7B103A90BAE4046CDF80880C6
:1062600081E84102CDE900A813230022FF2138462E
:1062700005F0E4FE40B9BDF84000F11CC01EC0B2FC
:106280002A1D0AF0CDF910B1032095E70AE0BDF808
:106290002D00E881062C05D19DF82200A872BDF8DA
:1062A00020002881002087E706A805F021FE0028AD
:1062B00088D0FFF75CFE7FE72DE9F8439846DDE9DB
:1062C000087614460D00814600D1FFDF0CB1012194
:1062D00000E0002105F1080004F0DEFC30800246F9
:1062E00000232146484602F067FC40B100973288FF
:1062F00043462146484602F0DCFCBDE8F883072C03
:1063000001D01120F9E743F20400F6E72DE9F0434C
:106310008DB00E46DDE9149805461C46174614213B
:1063200006A817F05AFE012002218DF81C108DF8E6
:1063300018008DF81D80ADF8207064B1A178C907F0
:1063400009D08DF82200E088ADF82600A088ADF8CD
:106350002400A0680A9001F0D6FE040023D06580D6
:106360000BA904A8CDE900010CAB00223146284658
:10637000FFF7A2FF002813D1049808368DE87100BA
:106380000BAA494606A80C9B05F057F8064660780C
:10639000000701D501F097FE5EB13046FFF71DFE04
:1063A0000DB0BDE8F08313212846FCF75BFB03200A
:1063B000F6E704980090BDF82C300422002128460E
:1063C00002F0EBFDECE7F0B58DB000240746099430
:1063D00006A80A94CDE904400725CDE900540794A6
:1063E00008940E460294039410232246384605F082
:1063F00025FE80B90BA8059007A90294CDE90341B9
:10640000CDE90054BDF8183000223146384605F079
:10641000F8FB002801D0FFF7AAFD0DB0F0BD05F094
:106420009DBA2DE9FC470546002600780C46B0468B
:106430000D2871D2DFE800F0B2070EAA30C853531E
:106440007188A68C970004B1FFDFA88880B201F0A4
:10645000CCFFA4E0A888042180B2814608F021FC8A
:10646000074604B1FFDF07B9FFDF494607F108001F
:1064700004F0ABFB01F047FE040008D0607840F068
:1064800008006070A4F8029001F01DFE88E013215E
:106490004846FCF7E7FA97E004B9FFDF608804217B
:1064A00008F0FFFB070000D1FFDFE888ADF800002F
:1064B000002038809DF80000010704D5C00602D5F1
:1064C000A888388005E09DF80100400667D5A888B7
:1064D00078806078022640F0080060705FE0E8880D
:1064E000ADF8000004B9FFDF9DF80100000604D5F7
:1064F0002878072806D0062828D0607840F00800C1
:1065000060704CE06088042108F0CBFB060000D1ED
:10651000FFDFA888708019E040E004B9FFDF6088E1
:10652000042108F0BEFB070000D1FFDF07F10800DF
:1065300005F04CFA90F0010F02D1E87900062ED553
:1065400060880226B880D8E704B9FFDF0226D4E7C6
:1065500004B9FFDF022661880122204601F089FF8D
:106560004FF00108C9E7A88987B204B1FFDF686866
:1065700000902889ADF8040001226946384601F0F0
:1065800093FF0CE0002CB8D1FFDFB6E704B9FFDFC2
:10659000022660880021FFF735FBAEE7FFDF9CB1E4
:1065A0006078000710D5B8F1000F0DD120781422C3
:1065B00020F00F00001D20F0F000803020702946F0
:1065C00004F1080017F0B5FC3046BDE8FC873EB585
:1065D0000C0008D06B4601AA002105F0AEFD20B1E9
:1065E000FFF7C5FC3EBD10203EBD00202080A070FE
:1065F0009DF8050002A900F00700FDF7F7FF50B96C
:106600009DF8080020709DF8050002A9C0F3C200A3
:10661000FDF7ECFF08B103203EBD9DF80800607057
:106620009DF80500C109A07861F30410A0709DF8E1
:106630000510890961F3C300A0709DF80410890654
:1066400001D5022100E0012161F342009DF8001014
:1066500061F30000A07000203EBD70B514460646F0
:106660000D4651EA040005D075B108460CF0AAF9B0
:1066700078B901E0072070BD2946304605F0B8FD25
:1066800010B1BDE8704072E454B120460CF09AF9A4
:1066900008B1102070BD21463046BDE8704096E735
:1066A000002070BD2DE9FE4F05460C46007A0A31E8
:1066B000009104F108010291904600270C31821EDE
:1066C0003E464FF0020B4FF0010A0191092A75D2A4
:1066D000DFE802F0F3F20574252577B6F400688848
:1066E000042108F0DEFA060000D1FFDF308810B187
:1066F00052270726E9E051271026002C7ED0688813
:10670000A08084F806A0A88900220099FFF7A5FFC1
:10671000002874D1A8892081288AE081F8E0B5F8A2
:106720001290072825D1E87B000622D5512709F1D0
:10673000140086B2002CE1D0A88900220099FFF74E
:106740008CFF00287AD16888A08084F806B0A889D8
:10675000208184F80EA0288A2082A4F81290A88AAA
:10676000009068884B46A969DDF8042001F0C1FA61
:10677000CEE0502709F1120086B2002C3ED0A88945
:1067800000220299FFF769FF002857D16888A0808E
:10679000A889E080287A072811D002202073288A4F
:1067A000E081E87B4B46C0096073A4F81090A88A8A
:1067B0000090688804F11202A969D7E7A7E00120D8
:1067C000ECE76888042108F06CFAB5F812A05FEADB
:1067D000000900D1FFDF09F1080005F0F7F890F09B
:1067E000010F02D1E87B000627D50AF114005127DA
:1067F00086B2002C7FD06888A08001E070E01DE0A8
:10680000A88900220099FFF728FF002816D184F8F4
:1068100006B0A88920810420A073288A2082A4F8C9
:1068200012A0A88A009068885346A969019A01F0CD
:1068300060FAA989A9F802106AE00320BDE8FE8F7A
:106840006888FAF7EBFD82466888042108F029FA87
:106850008146BAF1000F00D1FFDFB9F1000F00D17E
:10686000FFDFB9F80400A0F57F41FF3902D05127BE
:10687000142601E05027122694B36888A080502F78
:1068800006D084F806B0287B029901F042FA3FE076
:10689000287BA11D01F03DFA00219AF82300CDE9E3
:1068A00000010B46B9F8022068884946FFF72EFD23
:1068B0000028C3D12CE001E013E01FE0FE49A889C5
:1068C000C988814205D1542706264CB16888A0802A
:1068D0001EE053270CE06888A080A889E08017E0BC
:1068E00009E06888042108F0DCF900B9FFDF5527CA
:1068F0000826002CEFD1A8F800600EE056270726E6
:10690000002CF8D0A889A0800020A07100E0FFDF53
:10691000A8F800600CB12780668000208EE7E64969
:1069200000200870704730B587B00C4608F082F937
:106930000546FF2800D1FFDF0020208060804FF651
:10694000FF70A080294604F1080004F025F902AA8E
:106950002946012005F0C4FA1AE000BF9DF80B009B
:10696000000715D5BDF80E002946FFF72CFD9DF850
:106970000B00FF2340F010008DF80B00BDF80B005A
:10698000ADF80400BDF80E002946019A05F0FEFBA3
:1069900002A805F0ADFA0028E0D007B030BD0A46E5
:1069A000014602F1080004F016B970B5054604214D
:1069B00008F077F9040000D1FFDF294604F1080050
:1069C000BDE8704004F001B9F0B58FB00C46074641
:1069D000FAF724FD060005D03078222805D20820D9
:1069E0000FB0F0BD43F20200FAE70CB1A08870B11D
:1069F00001208DF81C0003208DF8200000208DF868
:106A0000210034B1A088ADF82800206803E00920F7
:106A1000E6E7ADF82800099001F075FB050007D006
:106A20006F800421384608F03CF9040007D105E0E6
:106A300013213846FCF716F80320D1E7FFDF06A93B
:106A400004A8CDE900010CAB002221463846FFF72F
:106A500033FC0028C4D104F10800049903908DE8A8
:106A6000A20096F8231006AA07A80C9B04F0E5FCE8
:106A700006466878000701D501F025FB1EB13046B7
:106A8000FFF7ABFAACE704980090BDF81830042289
:106A90000021384602F081FA4FF6FF71A1809FE78E
:106AA0002DE9FF4F87B09846DDE9159793467E881C
:106AB000DDF850A03046FAF7B1FC05460421304617
:106AC00008F0EFF8044605B9FFDF04B9FFDF08342A
:106AD000CDE90464CDE90297CDE9008ADDE907023A
:106AE00095F823105B4604F0E7F80BB0BDE8F08F93
:106AF0002DE9F04F9BB004464FF000086E48ADF80A
:106B00005880ADF83080ADF85480A0F80480ADF81E
:106B10001880ADF81C80ADF82480ADF82080007896
:106B200016460D464746012808D0022806D00328FD
:106B300004D0042802D008201BB0D7E720460BF071
:106B4000FFFED0BB28460BF0FBFEB0BB60680BF02D
:106B500042FF90BB606848B160892189884202D8B1
:106B6000B1F5007F01D90C20E6E780460BAA07A902
:106B70002846FFF78CFA0028DED168688078C0F3D9
:106B80004100022808D19DF81D0010F0380F03D0F5
:106B900028690BF017FF80B906A92069FFF72FFAC3
:106BA0000028C9D1206950B1607880079DF819008C
:106BB00000F0380002D5E8B301E011E0D0BB9DF849
:106BC000180080060ED59DF8190010F0380F03D07C
:106BD00060680BF0F7FE18B960680BF0FCFE08B1B6
:106BE0001020A9E708A96069FFF709FA0028A3D1D6
:106BF000606940B19DF8210000F0070101293BD1F7
:106C000010F0380F38D009A9A069FFF7F8F900286B
:106C100092D19DF8200080062ED49DF82400800695
:106C20002AD4A06950B19DF8250000F00701012980
:106C300022D100E020E010F0380F1DD0E06818B13C
:106C40000078C8B11C2817D20FAA611C2046FFF794
:106C500045FA0120B94660F30F27BA4607468DF87A
:106C6000520042F60300ADF850000DF13F0218A9A2
:106C7000286809F0F4FC08B107205DE79DF8600082
:106C800017A9CDF80090C01CCDE9019100F0FF0BD1
:106C900000230BF20122514614A805F066F8E8BB68
:106CA000BDF85C000E9004492A892869091D0092EC
:106CB000CDE901016B8901E010030020BDF82C2013
:106CC0002868079905F051F801007DD120784FF030
:106CD000020AC10601D480062BD5ADF80C9060697C
:106CE00050B908A907A8FFF72AFA9DF8210020F05B
:106CF0000700401C8DF821009DF820008DF852708F
:106D000040F0C8008DF8200042F60210ADF85000A7
:106D10000CA903AA0023CDF800A000E021E0CDE9F2
:106D2000012140F2032214A8089905F01EF8010081
:106D30004AD1FE484D465B468088ADF83D000FA81D
:106D4000CDF80890CDE90390CDF814904FF00709E5
:106D5000CDE900950022FF21BDF85C0004F051FF51
:106D600010B1FFF704F9E7E69DF83C00000625D5D1
:106D70002946012060F30F218DF852704FF4245002
:106D8000ADF85000ADF8105062789DF81000002367
:106D900062F300008DF810006278CDF800A0520870
:106DA00062F341008DF8100004AACDE9012540F2FC
:106DB000032214A804F0D9FF010005D1606850B384
:106DC000206970B906A900E07EE007A8FFF7B7F9CF
:106DD0006078800705D49DF8190020F038008DF800
:106DE00019008DF8527042F60110ADF8500020895C
:106DF00040F20121B0FBF1F201FB1202606815AB19
:106E0000CDF80080CDE90103002314A8069904F011
:106E1000ACFF010058D12078C00729D0ADF80C5044
:106E2000A06950B909A907A8FFF789F99DF82500BD
:106E300020F00700401C8DF825009DF824008DF8F7
:106E4000527040F040008DF8240042F60310ADF877
:106E5000500016A903AACDF800A0CDE90121002316
:106E600040F2032214A8099904F07FFF01002BD1FE
:106E7000E06868B32946012060F30F218DF8527055
:106E800042F60410ADF85000E068002302788DF857
:106E9000102040788DF81100E06804AA4088ADF811
:106EA0001200E06800798DF81400E068C088ADF841
:106EB0001500CDF80090CDE901254FF4027214A819
:106EC00004F053FF010003D00E9800F035FF33E6C5
:106ED00096480321017056B180883080BDF8540077
:106EE0007080BDF83000B080BDF85800F080002000
:106EF00022E670B501258AB016460B46012802D05D
:106F0000022816D104E08DF80E504FF4205003E013
:106F10008DF80E5042F60100ADF80C0063B100246C
:106F2000601C60F30F2404AA08A9184609F097FB17
:106F300020B107200AB070BD1020FBE704A99DF81E
:106F400020207A48CDE90021801C029000232146B0
:106F500003A802F2012204F008FF10B1FFF707F8BE
:106F6000E8E772480EB14188318005700020E1E702
:106F700070B594B0044601268DF83E6041F60100DC
:106F8000ADF83C0012AA0FA93046FFF7B2FF002867
:106F900048D12078654CC0074FF0000544D01C2133
:106FA00002A817F01AF89DF808008DF83E6040F02E
:106FB00020008DF8080042F60520ADF83C000E9543
:106FC0009DF83A00119520F00600801C8DF83A00DB
:106FD0009DF838006A4620F0FF008DF838009DF8D3
:106FE000390009A920F0FF008DF839000420ADF820
:106FF0002C00ADF830000EA80A9011A80D900FA833
:107000000990ADF82E5002A8FFF772FD002809D1B3
:10701000BDF80000E080BDF804002081401C6081C4
:107020002570002014B070BDE5802581BDF84800B2
:10703000F4E72DE9F74F3D49A2B04FF000080A7878
:10704000012A04D0022A02D0082025B04EE54A8841
:10705000824201D00620F8E723988A46824201D175
:107060000720F2E701208DF8760042F6020B00249B
:10707000ADF874B0ADF84C004FF6FF702146621CBD
:1070800062F30F21ADF84E00ADF8560007918DF870
:107090007A40FF20ADF878401EA98DF85400149175
:1070A00013A804F049FF00252E462F460DF12809AC
:1070B0000EAB4FF6FF72072113A804F040FF78B122
:1070C00082285FD1A5B39EB39DF86600ADF86C50E1
:1070D0008DF81840ADF86E601BAC012866D06DE0ED
:1070E0009DF83E002FB301285BD1BDF83C105945F7
:1070F00021D11AA8CDE904900720CDE9000402941B
:107100000394BDF83A0010230022FF2104F096FFFB
:10711000C0BBBDF86800042801D006284CD1BDF8DA
:107120002810239881423CD10F208EE710030020C5
:107130003AE0012835D1BDF83C00B0F5205F03D01E
:1071400042F6010188422CD1BAF80210BDF83A008B
:10715000814201D1012700E0002705B19EB12399AA
:1071600088421ED11AA9CDE904910721CDE9001466
:1071700005460294039410230022FF2104F05EFFD1
:1071800000B902E02DE046460BE0BDF86800022899
:1071900001D0102810D1C0B219AA0AA909F040FAEA
:1071A00050B9BDF83A8083E705204EE706A919A833
:1071B000221D09F054FA08B1032046E79DF8180093
:1071C0000023001DC2B28DF8182024980092CDE94A
:1071D00001401DA8079904F0C8FD10B902228AF8E1
:1071E0000020FEF7C4FE30E710B50B46401E88B005
:1071F00084B206AA00211846FEF770FF07A906AA66
:10720000CDE9042100200721CDE900100290039070
:1072100002460123FF21204604F0F3FC0446BDF89A
:107220001C00012800D0FFDF2046FEF7A0FE08B0BA
:1072300010BDF0B5F84F044687B038780E460328E5
:1072400004D0042802D0082007B0F0BD04AA03A986
:107250002046FEF71CFF0500F6D160688078C0F379
:10726000410002280AD19DF80D0010F0380F05D01A
:1072700020690BF0A7FB08B11020E5E7208905AADB
:1072800021698DE807006389BDF810202068039903
:1072900004F06BFD10B1FEF76AFED5E716B1BDF83C
:1072A00014003080042038702846CDE738B50C0033
:1072B000054608D000236A46FF2104F03EFF20B1B6
:1072C000FEF755FE38BD102038BD69462046FEF752
:1072D00096FE0028F8D1A078FF2100F0010328468F
:1072E000009A04F053FFEBE730B587B01446002254
:1072F0000DF10C0C06AD02928CE82C000723CDE9B1
:1073000000320A462388FF2104F07BFCBDF81810E8
:107310002180FEF72CFE07B030BD70B50D4604216C
:1073200007F0BFFC040000D1FFDF294604F108008C
:10733000BDE8704003F070BC70B50D46042107F045
:10734000B0FC040000D1FFDF294604F10800BDE8CD
:10735000704003F084BC70B50D46042107F0A1FC19
:10736000040000D1FFDF294604F10800BDE87040A9
:1073700003F092BC70B50D46042107F092FC0400A6
:1073800000D1FFDF294604F10800BDE8704003F09A
:107390008DBC0121FEF736BC2DE9F04196B04FF0CF
:1073A00000050C008046ADF818501CD0E06828B1EC
:1073B000A068C0B10188ADF8181005804046FAF702
:1073C0002DF8070011D03878222861D3404607F005
:1073D00031FC0146A07801280AD0022808D00720F5
:1073E00016B0BDE8F0811020FAE743F20200F7E79B
:1073F000208830B1401C80B207AA04F071FD50BB58
:1074000002E043F20300EBE707A804F071FD9DF8EA
:1074100026204FF45051012A09D1BDF82420A2F5AD
:107420002453023B03D1822801D0A0B901E00846D1
:10743000D6E7E068B0B106A9CDE904010720CDE99F
:10744000000502950395A2882088BDF81830FF2119
:1074500004F0D7FB10B1FEF78AFDC1E7A168BDF8C3
:10746000180008809DF81F00C00602D543F20140B5
:10747000B6E70B9818B1BDF82800022801D0032008
:10748000AEE70B98A1780078012903D0800706D4D5
:107490000820A5E7C007FBD00726022001E001264F
:1074A00003208DF83C009DF8200010F0380F00D12B
:1074B000FFDF9DF820005949C0F3C200084497F847
:1074C000231010F8010C884201D90F2088E720888A
:1074D000ADF840000421404607F0E3FB040000D172
:1074E000FFDF0DA90CA8CDE900010EAB3246214605
:1074F0004046FEF7E1FE002885D108340C9903943C
:107500008DE822010DAA07210FA80E9B03F095FF1D
:1075100010B1FEF762FD63E70C980090BDF83430BF
:1075200004223146404601F038FD59E770B5064661
:1075300015460C460846FEF7D9FC002805D12A4618
:1075400021463046BDE87040D3E470BD71E570B5AA
:107550001E4614460D0009D044B1616831B138B1FE
:107560002D494988814203D0072070BD102070BD8D
:107570002068FEF7BBFC0028F9D132462146284698
:10758000BDE87040FFF7B4BA70B515460C0006D0E0
:1075900038B121498988814203D0072070BD10206D
:1075A00070BD2068FEF7A2FC0028F9D129462046CC
:1075B000BDE870403DE670B5054686B00E461446FF
:1075C00010460BF0E1F930BB60680BF004FA10BB19
:1075D000A5F57F40FF3803D02846F9F71FFFA0B17B
:1075E000284607F027FB054630466946FEF7C9FDE9
:1075F00000280CD19DF810100F2008293FD2DFE899
:1076000001F008060606060F0F0843F2020006B056
:1076100070BD0320FBE743E0100300206AE3010094
:107620009DF80210012908D1BDF80010B1F5C05F26
:10763000EDD06FF4C052D142E9D09DF80610012977
:107640000BD1BDF80410A1F52851062905D2DFE8B9
:1076500001F0030304030303D9E79DF80A1001298D
:107660000ED1BDF80810B1F5245FD0D0A1F524519A
:107670000239CCD00129CAD0022901D1C7E7FFDFE6
:10768000606878B9002305AA2946304604F055FD04
:1076900010B1FEF76CFCBAE79DF81400800601D427
:1076A0001020B4E76188224630466368FFF71CFE6D
:1076B000ADE72DE9F043044689B0894615461046EA
:1076C0000BF062F918B1102009B0BDE8F083204634
:1076D00007F0B0FA4FF6FF770646BC4201D0FF2E06
:1076E00009D00146002307AA484604F026FD28B128
:1076F000FEF73DFCE8E743F20200E5E79DF81C00D9
:10770000C00602D543F20140DEE7002406A8CDE919
:1077100004404FF00708CDE90084029403946A887E
:107720003B463146484604F089FC070014D168689E
:107730000BF02AF968B968680294CDE90340059412
:10774000CDE900842B886A883146484604F076FCEF
:107750000746BDF8180028803846C9E739B1FA4B0A
:107760000A881B899A4202D843F20300704713E645
:1077700010B586B0F44C0423ADF81430E38843B15F
:1077800024898C4201D2914205D943F2030006B00C
:1077900010BD0620FBE7ADF810100021009101910B
:1077A000ADF8003002218DF8021005A9029104A95C
:1077B0000391ADF812206946FFF7EEFDE7E72DE9EA
:1077C000FC4781460F4608460BF0BAF888BB48468E
:1077D000F9F724FE5FEA00080AD098F80000222892
:1077E00029D30421484607F05CFA060005D103E0DE
:1077F00043F20200BDE8FC87FFDF06F1080003F05A
:1078000012FA05463878012803D0022804D0072050
:10781000F0E7A8070FD502E015F0340F0BD0B879C8
:107820003C1DC00709D0E08838B1A0680BF088F88B
:1078300018B11020DEE70820DCE73A782088002124
:1078400028B3A0F201130721112B18D20CD2DFE8C4
:1078500003F00B090D0B1D0B121D100B0B1D1D1D35
:107860001D0B1D00022A11D10846C3E7012AFBD0D7
:107870000CE0EA0600E0AA06002AF5DA06E0A0F528
:10788000C0721F2A02D97D3A022AEDD8C1B298F8F7
:107890002300CDE900017288234631464846FEF7B1
:1078A00035FDA7E72DE9FF4F8DB01E4615460C4666
:1078B0004FF000080F460D98F9F7B0FD30B1007891
:1078C000222806D2082011B0BDE8F08F43F2020052
:1078D000F9E7B00801D00720F5E7032E00D1002614
:1078E0000D9807F0A7F94FF6FF7A0690CCB1022D5C
:1078F00074D320460BF06FF830B904EB0509A9F1F9
:1079000001000BF068F808B11020DCE7AD1EAAB248
:107910002146504604F022FD39F8021C88425DD110
:10792000ADB28948B10702D50189491C00E00121A7
:107930001FFA81F9F10701D0068900E0564607AA2F
:107940004846069904F0CCFA4FF0070B4FF0000AB6
:107950000BE07888102841D808F1040108441FFA88
:1079600080F8A8453AD804EB08077FB33988494521
:10797000EFD353E09DF81F100A074FD544B304EB33
:10798000080708F104027B881FFA82F8102B25D81B
:1079900003EB0802AA4221D83A8890421ED1C806B9
:1079A0001ED50DF10C090CAA04EB08015046CDF8C8
:1079B00008A089E80700CDE900BA388800220699B6
:1079C00004F01FF928B1FEF7D2FA7CE726E005E0C3
:1079D0000CE07888BDF83010884201D00B2072E7A7
:1079E000798801EB08001FFA80F806E0C90604D583
:1079F0000699FEF7E8FC002887D19DF81F00FF23B9
:107A000020F010008DF81F00BDF81F00ADF8000039
:107A1000BDF82200009A069904F0B8FB07A804F00C
:107A200067FA18B9BDF82200B042A3D904210D9815
:107A300007F037F9040000D1FFDF22885AB1CDE901
:107A400000BA5546002321460D98FEF75FFC00283A
:107A5000BBD1258037E7002035E72DE9F04F8DB009
:107A60001E4617000D464FF000041BD0B10802D08F
:107A700007200DB028E7032E00D1002607F0DAF822
:107A80008046FF2805D07DB128460AF09BFF48B903
:107A900002E043F20200ECE73988681E08440AF06D
:107AA00091FF08B11020E4E72749B00701D54889C4
:107AB00000E00120F2074FF6FF7902D04989491E04
:107AC00000E049468EB207AA414604F009FA4FF099
:107AD000000B4FF0070A3EE09DF81F0000073AD563
:107AE00006A9CDE904B1CDF808B0CDF80CB04B46ED
:107AF00000224146CDE900AB604604F09FFA08BB86
:107B000025B3BDF818103A8821442819091D8A4266
:107B100034D3BDF8222020F8022BBDF8182020F81D
:107B2000022B06AA0592CDF808B0CDE903B0CDE945
:107B300000ABBDF82200BDF818300022414604F029
:107B40007DFA18B1032094E710030020BDF8180057
:107B50002044001D84B207A804F0CAF920B182288D
:107B600006D0FEF704FA84E7BDF822C0B445B3D9C5
:107B700034B175B13988A01C814203D20C2078E75A
:107B8000052076E722462946484604F0E7FB2919F6
:107B90000880A41C3C8000206BE710B504460AF066
:107BA000F3FE08B1102010BD6948408920800020F4
:107BB00010BD2DE9F041A4B00C4606464FF0000878
:107BC000142105A816F009FA01208DF818008DF887
:107BD000140000278DF81970ADF81C403046F9F7F5
:107BE0001DFC30B10078222806D2082024B0BDE860
:107BF000F08143F20200F9E70421304607F051F822
:107C0000050000D1FFDF0AA904A8CDE9000116ABE9
:107C1000002229463046FEF74FFB0028E6D10498A3
:107C20000835CDE90007CDE902650AAA072105A8B4
:107C3000169B03F002FC10B1FEF7CFF9D6E70498CB
:107C40000090BDF8283004224146304601F0A5F9E5
:107C500000B1FFDF21463046FDF7C6FF17A92846D1
:107C600002F0D0FF00B1FFDFBDF85C00172801D2A1
:107C7000172100E00146A14204D8172801D2172499
:107C800000E0044621463046FFF756FB05462146F4
:107C90003046FDF702FD4146304601F02BFB00B9AE
:107CA000FFDF25BB3046F9F7B9FB050000D1FFDF48
:107CB00095F822001B281AD9172C18D93A208DF8CC
:107CC0002C00ADF82E6095F82200211D884201D9C4
:107CD000241D00E00446ADF8304040F64800ADF801
:107CE000320018A90BA804F0C0FA00B1FFDF002091
:107CF0007CE7F8B51C4615460E46069F07F034F99A
:107D00002346FF1DBCB231462A46009406F04CFDC6
:107D1000F8BD70B50C4605460E21204616F03BF91D
:107D2000002020802DB1012D01D0FFDF70BD062085
:107D300000E00520A07170BD10B50C4604F09DF860
:107D400000B1FFDF2046BDE81040FEF710B900008B
:107D50001003002010B50446007896B0022805D024
:107D6000012803D043F2050016B010BDA17889297F
:107D70000AD06078892807D021B1032902D808B138
:107D8000032801D90720EFE74D208DF80000207867
:107D9000022801D0012000E000208DF80200607868
:107DA00000F0D7FDC01D8DF80300A078012815D084
:107DB00000F0CFFD10F101008DF80400607800F0B4
:107DC000C8FD8DF80500A07800F0C3FD8DF8060011
:107DD0009DF805200621102A04D005E0022000F0BD
:107DE000B8FDE9E78DF80510102801D18DF80610CF
:107DF0002078012804D19DF80300401C8DF8030071
:107E000002F0E0F8001DADF808000BA9684604F088
:107E10002CFA00B1FFDF0020A6E72DE9FF4FFF4954
:107E200091B00600D1E900010396CDE90C01507A2A
:107E3000117A9B4608441546C7B222D05FF0000471
:107E40004FF00009CDF81C900520ADF81C001F2054
:107E5000ADF81E00F2A00690CDF81490F01D8DF83C
:107E600014904FF0010A20F007008DF815A0B042E1
:107E700000D0FFDF28880399401C1FFA80F814B156
:107E800007E00124DCE708F0FF0008F06FFB00B119
:107E9000FFDF03993A4601EB0810C01C20F00301F4
:107EA000D5F8188003913CB981F800901FFA88F04A
:107EB00003F06EFE00B1FFDF0399234601EB0800DB
:107EC0000390A87A297A3A460844C1B203A800F080
:107ED0008EFD0398C01C20F003000390697A009186
:107EE0002B7AAA7A04B1002002A906F0B6FD00B1EF
:107EF000FFDFBDF8081003980DF1780808443A46F2
:107F000098E88A00C01C20F00300CDE90270CDE99A
:107F1000001304B100205B4608A906F029FF00B158
:107F2000FFDF089903980844C01D20F00700039064
:107F30001299821B002C0A603AD1BC4ABA491160DE
:107F4000111D401E086001232C220EA9B84806F01E
:107F500005FD00F00CFD00211E22084602F042F84B
:107F6000FAF7A4F900F075FFFEF7D9FCE8680CAA4F
:107F7000214620B1FBF755F830B1FFDF04E005A83A
:107F8000FBF74FF800B1FFDF05F11400FEF7F0FF3B
:107F900000B1FFDF4FF49671A64816F01EF8A54811
:107FA000022180F829A180F82A11062180F82B11DE
:107FB00015B0BDE8F08F10B59E4CA078092800D30D
:107FC000FFDF207804EB401010F8041F21F0FF01C0
:107FD0000170417821F00701C91C21F0180141709E
:107FE0000121E17010BD2DE9F04105460C46002746
:107FF0000078052190463E46B1EB101F00D0FFDF10
:10800000287A58B1012810D0FFDF00BFA8F800601F
:108010000CB1278066800020BDE8F0810227092688
:108020007CB1A889A080A87B09E00327142644B16D
:108030006888A0802869E060A88A2082287B207256
:10804000E4E7A8F80060E6E700B597B04E218DF8A8
:10805000001000780BA900F001008DF802006846BE
:1080600004F003F917B000BD00B5017897B001F036
:1080700001018DF80210417801F001018DF8031023
:108080000178C1F340018DF804104178C1F340013B
:108090008DF80510017889088DF806104178890857
:1080A0008DF8071081788DF80810C1788DF80910C7
:1080B00000798DF80A004A208DF800000BA9684667
:1080C00004F0D3F8CEE770B55A4CE078002819D008
:1080D0002078002504EB4010407900F007000119DA
:1080E00091F82801401E81F828012078401CC0B278
:1080F0002070092800D12570A078401CA07009F0DC
:10810000BAFFE57070BD4B4890F82B01002800D0F5
:1081100051E770472DE9F043464D9BB05FF00006F4
:10812000D5F8240168B1FFF7EEFF002875D02022B2
:10813000D5F8241115F0FDFEFFF7C5FFC5F8246141
:10814000EEE795F82901002867D0FFF734FF0446D1
:10815000374806F034FC606000B9FFDF606804F067
:10816000D1F888B12046F9F7C6FB6078010706D53B
:1081700020F00700401C6070FFF7A5FFD0E72C48F7
:10818000616806F025FCCBE72948616806F020FC11
:1081900001A800F0B9FC00286BD10321BDF8040050
:1081A00006F07FFD8046BDF8040006F0DDFE0746C0
:1081B000B8F1000F00D1FFDFD8F8040010B100784B
:1081C000FF2856D0FFF7F7FE0446384606F08FFA30
:1081D000606000B9FFDF606800F104090671BDF856
:1081E00004006080204600F02CFF384606F04FFB6C
:1081F00000B9FFDF47208DF81000BDF80400ADF88E
:10820000120004A805F0D9FE10A804F0DEFA607888
:10821000010711D4C00615D417E02AE070E301006D
:108220006E52463578000000000000200006024033
:10823000780500204C04002020F00700801C6070AE
:10824000FFF741FFC8F804906AE7D8F8040038B196
:108250000178491C11F0FF0101708FD1FFDF5FE74A
:1082600000221146384600F072FB002886D1FFDF5D
:1082700056E71BB0BDE8F08310B5FE4CA06008685F
:10828000E060AFF26F1001F0F6FD607010BDF949CB
:1082900000200870704730B505464FF080500C46FE
:1082A000D0F8A41097B0491C05D1D0F8A810C94344
:1082B0000904090C08D050F8A01F01F00101297031
:1082C0004168216080680EE02B208DF800000BA92A
:1082D000684603F0CAFF00B1FFDF012028700C9848
:1082E0002060BDF83400A0802878002803D0607991
:1082F00040F0C000607117B030BDF0B54FF0805451
:108300000746D4F8800097B00D462B26401C0BD1B1
:10831000D4F88400401C07D1D4F88800401C03D155
:10832000D4F88C00401C0BD0D4F880003860D4F80E
:1083300084007860D4F88800B860D4F88C0016E027
:108340008DF82C6069460BA803F08FFF00B1FFDFAA
:1083500001983860029878608DF82C6069460BA807
:1083600003F083FF00B1FFDF0198B8600298F86066
:10837000D4F89000401C0BD1D4F89400401C07D1D5
:10838000D4F89800401C03D1D4F89C00401C08D0BD
:1083900054F8900F286060686860A068A860E06882
:1083A00016E08DF800600BA9684603F05EFF00B18F
:1083B000FFDF0C9828600D9868608DF800600BA9AD
:1083C000684603F052FF00B1FFDF0C98A8600D98DB
:1083D000E86017B0F0BD30B5A74C0546D4F82401CD
:1083E00000B1FFDFC4F8245130BD3EB5054603217E
:1083F00006F057FC0446284606F0B6FD054604B9CB
:10840000FFDF606818B10078FF2800D1FFDF01AA04
:108410006946284600F09BFA60B9FFDF0AE00022B7
:1084200002A9284600F093FA00B9FFDF9DF8080082
:1084300000B1FFDF9DF80000411E8DF80010EED264
:1084400060680199884201D1002060608A4C94F8EC
:108450002A01022800D3FFDF94F82A01401CC0B291
:1084600084F82A01012803D18248407801F022FDD6
:108470003EBD70B50446A1F57F4016460D46FF3857
:1084800000D1FFDF012E01D0FFDF70BD207820F08A
:108490000F00401D20F0F0005030207000202072AE
:1084A000A5810120A07370BD70B515460C46064627
:1084B000FFF729FE90B1017821F00F01491D21F04D
:1084C000F001503101704680012101722168016183
:1084D000A18881820573BDE87040F4E53046BDE8AF
:1084E00070401321FAF7BEBA70B505460C4608462F
:1084F0000AF04AFA08B1102070BD2846F8F78EFF3E
:1085000028B1284600F0E7FE2070002070BD43F23D
:10851000020070BD2DE9F04F04465648894687B0E9
:10852000017811B1082007B043E552485349416032
:1085300020460AF029FA002875D148460AF024FAA4
:10854000002870D1637A217A5818FF287DD82088B6
:10855000FE287AD800B90A202080A06908B94FF413
:10856000B060A0616068A0B14578827805EB4505F0
:108570002A440578067905EB450502EB4502457965
:10858000C07805EB450505EB8605C0EBC000284427
:1085900009E003EB430001EB410200EB4202C1EBB7
:1085A000C10505EB830086B2C3EBC3001044C1EBE9
:1085B000C1021044084487B2208A01F0F9FC002867
:1085C000B1D101F0FFFC001D7843059001F0FAFCE9
:1085D000001D00FB06F8E168A06900F041FA5FEABF
:1085E000000AA0D1A17A607A81422ED84FF0120BF6
:1085F00008280ED8207A01280BD808F022F9054661
:1086000009F0F8FC2A1A217A607A521E0B189A4255
:1086100001DA584687E765688B460090BDB1284669
:108620000AF0D9F908B110207DE7A97868780844E4
:108630002978421800985844904206D16A792979DD
:108640001144EA781144884201D007206BE7CDF845
:108650000080CDE90176224603A90020059BFFF7A3
:10866000DCFB044D039AD9F8003068681118994270
:1086700009D805E01C0000204C040020481300200D
:10868000B2F5803F03D30420C9F800104BE7CDF8C2
:108690000080CDE90176224604A9059BFFF7BDFBCA
:1086A000DDE90301884200D0FFDF049869680844CF
:1086B0006860C9F80000FF49012028700870504622
:1086C00031E72DE9F04707460C4608460AF05CF909
:1086D00040B938460AF076F920B9F81C20F00300BA
:1086E000B84202D01020BDE8F087F3484FF00008F0
:1086F000817889B14178824600EB4115B4F8009049
:1087000015F8040F234600F00F000022294600F060
:1087100037FA060004D013E0A4F800800520E2E751
:1087200097B12188494501D90C260DE028782346C8
:1087300000F00F003A46294600F022FA060005D064
:108740000C2E01D0A4F800803046CCE79AF8010046
:108750005446401CC0B28AF80100092801D184F8AF
:108760000180A078401EA070687800F00701012900
:108770000BD0022903D0032918D0FFDFE4E7C0069D
:10878000E2D46888FFF731FEDEE7CC48696806F07E
:108790001FF994F82901401CC0B284F8290101286E
:1087A000D2D1C748407801F085FBCDE794F82B0182
:1087B000401C8AF82B01C7E770B50D4604460AF045
:1087C000BFF818B928460AF0DFF808B1102070BDCC
:1087D00029462046BDE8704007F0FFBE70B504464C
:1087E00015460E4608460AF0ABF818B928460AF0B6
:1087F000CBF808B1102070BD022C03D0102C01D092
:10880000092070BD2A463146204607F009FF00289E
:10881000F7D0052070BD70B514460D4606460AF027
:108820008FF838B928460AF0AFF818B920460AF090
:10883000C9F808B1102070BD22462946304607F01D
:108840000EFF0028F7D0072070BD10B596B0044683
:108850000AF09AF810B1102016B010BD0F208DF854
:1088600000000BA9684603F000FD0028F4D19DF834
:1088700034002070BDF836006080BDF83800A0805C
:108880000020E9E770B505460C4608460AF09AF85C
:1088900020B93CB120680AF077F808B1102070BD0B
:1088A000A08828B121462846BDE87040FEF78CB864
:1088B000092070BD70B504460D4608460AF040F820
:1088C00030B9601E1E2814D828460AF039F808B1BD
:1088D000102070BD032C01D9072070BD04B9FFDF43
:1088E000784800EB840050F8041C2846BDE870402E
:1088F0000847A4F120001F28EED829462046BDE8ED
:108900007040F9F70EBC70B504460D4608460AF0F3
:108910003BF830B9601E1E280FD828460AF010F820
:1089200008B1102070BD012C03D0022C01D0032C03
:1089300001D1062070BD072070BDA4F120001F28C2
:10894000F9D829462046BDE87040F9F76EBC05F01D
:108950006ABD892805D0032805D0022805D001204A
:10896000704710207047062070470320704710B5ED
:1089700096B003F06BFC52484178806803F064FEC7
:108980004F4801240C300178012916D13E218DF881
:108990000010C0788DF8020010B1012803D005E066
:1089A0008DF8024002E000208DF80200684605F0D4
:1089B00004FB10B10BA803F008FF02208DF82C0077
:1089C0008DF82D008DF82E000BA8FFF7C3F900B12C
:1089D000FFDF8DF82C4003208DF82D008DF82E0040
:1089E0000BA8FFF7B7F9002800D0FFDF34E72DE927
:1089F000F0410646022012B101EB4200401DC7B211
:108A00003068C01C20F0030232601BBB2A483B4682
:108A10000921243809F085FE002408E0092C11D230
:108A2000DFE804F005070509090B0B0505002648DA
:108A300004E0264802E0264800E0264809F090FEBF
:108A4000054600E0FFDFA54200D0FFDF641CE4B272
:108A5000092CE3D3306800EB07103060BDE8F081EB
:108A600038B50C00054604D0084609F069FF00BB84
:108A700002E0F62844D345E0606809F061FFC0B920
:108A8000607800F00300012803D0022801D00720FD
:108A900038BD69462046FBF78DFD0028F8D1607887
:108AA00000F0030002281CD19DF80000C8B16068E6
:108AB00012E014E0080000204C040020780500209B
:108AC0001C00002090E30100771F0000F18E0000E1
:108AD000CB9F00002103010009F074FF08B11020B2
:108AE00038BD6089F8280BD82189814208D861787F
:108AF00001F00301012905D1D73080B2A84201D984
:108B0000092038BD002038BD2DE9F04397B08146DB
:108B100046208DF82C0069460BA803F0A6FB00B197
:108B2000FFDF43F2040600246D46DFF884801FE077
:108B30002F19B87DC10706D0400704D405EB4400C7
:108B4000C08800F0B9FB98F82A0178B1B87D800799
:108B50000CD505EB4400C08800F037FA30B105EBC6
:108B600044000026C188A9F8001005E0641CE4B2A6
:108B70009DF80400A042DBD817B03046BDE8F08372
:108B80002DE9F041044600201880601E1D4616465F
:108B90000F46052800D3FFDF06482A4600EB840075
:108BA000314650F8043C3846BDE8F0411847000013
:108BB0004C04002078E301002DE9F0478A469846EE
:108BC00015460646032106F06CF80446304606F0CA
:108BD000DDF90C35AFB2002581462E4604B9FFDF22
:108BE000B9F1000F00D1FFDF04EB8A000189B9421F
:108BF00000D30125218CB94202D2BAF1060F00D36D
:108C0000012638EA050104D0817A41F0020181721F
:108C10000BE038EA060108D0817A41F00401817244
:108C200014F8220F40F00400207005EA0600BDE8A9
:108C3000F0872DE9F0478246DDE90846174604F142
:108C40000C0099460D461FFA80F80023224639464B
:108C50005046FFF7B1FF60B1A87800061BD426F894
:108C6000044C26F8029C504606F090F9060008D104
:108C700006E0072F01D01120D9E743F20400D6E720
:108C8000FFDF241D3046A1B205F0CCFA00B9FFDFAA
:108C9000504603F03DFC05EB8700062F0289A2EB4E
:108CA0000801018103D2298CA1EB0800288400204F
:108CB000BDE72DE9F8431D4617460E46DDF8208036
:108CC00006F064F9040019D03F1DB9B205F05AFA54
:108CD0002860B0B1067120466A46296805F016FD85
:108CE000009800210A460180817003F0D1FC0098B1
:108CF000C01DC8F800000020BDE8F88343F2020060
:108D0000FAE7072E01D01120F6E743F20400F3E75B
:108D10002DE9F04F0F46054687B0164650880321CF
:108D200005F0BFFF040000D1FFDF4FF000098DF810
:108D30000890A078400600D1FFDF042F53D3297894
:108D400041F30000401C06D162786B789A424AD108
:108D50002278120747D04FF0010B4FF00208142978
:108D600039DA4FF6FF7A012933D0122902D01329BC
:108D700031D11CE00C2F2ED1A17801F07F01012907
:108D800029D0207820F00F00401C20706878607097
:108D90008DF808B0A888ADF80A00E888ADF80C0096
:108DA0002889ADF80E006889ADF8100016E0062F8E
:108DB00011D1207820F00F0020707188012009F077
:108DC0007CFD8DF80880ADF80AA0A888ADF80C00ED
:108DD00004E0062F0AD09DF80810B9B17088324619
:108DE00002A9F9F73AF907B0BDE8F08F207820F032
:108DF0000F0020707188012009F05FFD8DF8088058
:108E0000A888ADF80A00ADF80CA0E7E70028EAD082
:108E1000768805A8009006AB062204213046FFF7AD
:108E200048FF00B1FFDF05980523042280F800B059
:108E300069784170A0F80280A0F804900621CDE97D
:108E4000001021463046FFF7F4FE0028CBD0FFDFAC
:108E5000C9E710B501F0B6F80021FF4B0A4600BF84
:108E600023F81120491C0829FAD3FB4A00F10C0110
:108E70001032400011805180183090804D20D080F9
:108E800011815181C1EBC100908110BD70B50C46BC
:108E9000897821F0FF01A170217821F00F01217064
:108EA000012161700021616006F070F8050000D1B9
:108EB000FFDF284605F064F9E74910318989401A37
:108EC00020852046BDE8704000F014BB70B50D460B
:108ED000032105F0E6FE040000D1FFDFA07865F372
:108EE0000600A07070BD70470146012009F0E5BC86
:108EF0003EB58DB20321284605F0D3FE040000D113
:108F0000FFDF2078002220F00F00207002208DF873
:108F100000004FF6FF70ADF80200ADF8040069469E
:108F20002846F9F79AF83EBD2DE9F84F05460C465C
:108F300000270078012192463E46B1EB101F00D079
:108F4000FFDF287A032809D0FFDF00BFAAF80060FE
:108F50000CB1278066800020BDE8F88FB5F80C8042
:108F6000702708F10A0086B2A4B16888A0806889D9
:108F70002081A4F806806888D5F8049004F10A05D9
:108F800005F0F2FF2A46072549464346009505F0BD
:108F90000BFCDBE7AAF80060DDE72DE9FC410F469A
:108FA0001C46164680460321089D05F07AFE010006
:108FB00008D033463A464046CDE90045FFF739FE32
:108FC000BDE8FC8143F20200FAE7F8B50646A0F5D9
:108FD0007F40FF3816D0304605F0C6FF040000D1B0
:108FE000FFDF204605F083FB050000D1FFDF2046B0
:108FF00029466A4605F08AFB009CB4F80500E41C8B
:10900000052801D00120F8BD0321304605F049FEB6
:10901000050000D1FFDF2079122807D120880C2815
:1090200004D1A87800F07F00022806D00023062291
:1090300004213046FFF7C0FDF8BD002306220521BC
:10904000F7E7F8B50446408805F08EFF050000D12B
:10905000FFDF6A462846616800F0CCF902460098B6
:10906000121F30F8031F458891421DD1042D1CD0DA
:10907000052D27D0062D1DD0402D15D30E46284690
:1090800000F0D4F908280FD0207820F00F00401C01
:1090900020F0F00010302070032020726581A6813E
:1090A000607840F008006070F8BD2246001D00F0B6
:1090B000C9F9F8BD636864880A46011D2046FAF7BD
:1090C000FDFEF8BD2246001DFFF722FEF8BD7FB56C
:1090D0000D460646032105F0E4FD04003AD0207851
:1090E00000F00F00012838D002A8009003AB0C223A
:1090F00005213046FFF7DDFD002829D10298122115
:109100000523017061781A46891C4170082141804D
:10911000298881806988C180A9880181E988418185
:109120000C21CDE9001021463046FFF782FD00B149
:10913000FFDFF02300223146012009F021FB2078D7
:1091400020F00F00401C20706078801C60700020B0
:1091500004B070BD43F20200FAE71120F8E77FB5D2
:109160000D460646032105F09CFD040006D020783C
:1091700000F00F00012804D00820E9E743F20200C4
:10918000E6E702A8009003AB062205213046FFF770
:1091900090FD0028DCD1029813210523017061782D
:1091A00041700221418085800621CDE900101A46D8
:1091B00021463046FFF73DFD00B1FFDF207820F06B
:1091C0000F0020700020C3E72DE9F84F0F468346BB
:1091D000032105F066FD0546584605F0D7FE80469A
:1091E0004FF0000A05B9FFDFB8F1000F58D1FFDFDB
:1091F00056E040466946002205F015F99DF800400A
:109200008146082C00D3FFDF05EB840609F1080036
:109210003189062C0144318102D2298C08442884EA
:10922000072C03D10AF1010000F0FF0AB07AC00751
:109230000DD02146284600F0DFF840B9B07A20F082
:109240000100B072584684B3032C2FD0FFDFB07AF0
:1092500081070AD502E00000A805002020F00200E6
:10926000B0722146584600F0D8F8062C18D895F868
:109270002200410714D520F0040085F822000024C4
:1092800005EB8400817A4A0706D521F0040181723A
:109290002146584600F0C1F8641CE4B2062CEFD316
:1092A0007F1EFFB2A5D2504656E602E0FAF79DFEB9
:1092B000CDE7FEF76EF8CAE710B5032105F0F1FC23
:1092C000040000D1FFDF204600F014F9A07840F040
:1092D0008000A07010BD10B5032105F0E2FC040071
:1092E00000D1FFDF00F06EFE218D0C30B1FBF0F0FD
:1092F000C0B210BD70B50D46032105F0D2FC0400CC
:1093000000D1FFDF062D00D9FFDF2946204600F0FF
:1093100073F8002805D004EB85018A7A42F0010237
:109320008A7270BD10B50446402801D2072010BDD6
:1093300000F07CF8082802D04FF4445010BD002102
:10934000774802E0491C082903D230F81120002A8E
:10935000F8D1082903D020F81140002010BD0420C6
:1093600010BD10B5402801D2072010BD00F05EF8F6
:10937000082805D06A4A002122F81010084610BDBE
:10938000052010BD2DE9FE4315460C00804606D091
:109390002DB16088402804D20720BDE8FE8310204C
:1093A000FBE7218811B300F041F8082820D002A87B
:1093B0000090228801AB07214046FFF77AFC002885
:1093C000EBD140462788019E05F0E0FD2A4607259F
:1093D00031463B46009505F020FA0298009023881C
:1093E000628807214046FFF7D8FDD6E70C20D4E776
:1093F0000520D2E705F08AB9072904D0484A10327F
:1094000032F8112000E0028D00EB810000899042CB
:1094100001D2012070470020704710B5032901D008
:10942000FFDF10BDBDE81040FAF7A5BD01460020E2
:109430003B4A02E0401C082803D232F810308B422D
:10944000F8D17047F0B50F460646014687B014467E
:109450003846FCF7B1FBC0B2082842D10020ADF875
:10946000100003906088032105F01BFC050000D16B
:10947000FFDF00212846FFF7BFFF78B96088002191
:10948000FDF769FFADF81000024603A80090608860
:1094900005AB0021FFF70DFC00B1FFDF0398059934
:1094A000CDE90010029404AB324638466168FDF7FE
:1094B000F7FAC0B205281BD2DFE800F0031A131533
:1094C0001300BDF8100000280BD003990423CDE948
:1094D0000001608800222946FFF7ABFB002800D07E
:1094E000FFDF07B0F0BD607840F010006070F8E773
:1094F000FFDFF6E710B504462021083014F06DFDBB
:109500000748002110F1100004EB810330F811200E
:10951000491C1A810629F7D9208DA08410BD0000AE
:10952000A805002030B44FF0E02001234FF4006C78
:109530000021C0F880C11D02C0F880511C06C0F88F
:109540008041E84A82F80014D21E82F80014E64AEC
:1095500082F80014E54A53609360C2F84011C2F8E3
:109560004411C2F84811C0F880C2C0F88052C0F857
:109570008042C0F800C1C0F80041136030BC7047A1
:1095800070B401204FF0E023C6024FF0000CC3F886
:1095900080610402C3F880410506C3F88051D34AB4
:1095A00050609060D24801680029FCD1C2F840C1E7
:1095B000C2F844C1C2F848C1C3F88062C3F880420F
:1095C000C3F8805270BC70474FF0E0204FF4006148
:1095D000C0F88012C910C0F880127047002804BF7C
:1095E000C4487047012804BFC3487047022804BF1D
:1095F000C248704700B5FFDF002000BD08B5BB4979
:10960000002298B101282FD002281CBFFFDF08BD1F
:109610004FF48020C1F80803C1F84803B84802603D
:10962000C1F84821B5480068009008BD4FF480306B
:10963000C1F80803C1F84803B24B1A60C1F84021D1
:10964000B14BC1031960B149C1F808034FF0E023E1
:109650000012C3F88001AE480260C1F84021C1F891
:109660000022AC48027008BD4FF40030C1F8080376
:10967000C1F84803A8480260C1F844219E48006828
:10968000009008BD70B5DFF864C2042600240125EF
:10969000B0B101284CD002281CBFFFDF70BD9F482D
:1096A0004FF48022012BC0F8401518BFCCF80823D6
:1096B000C0F8404108BFCCF80423CCF8442370BD67
:1096C000881E20F07F40CCF840054FF48030CCF865
:1096D0000803CCF84041CCF84403012B14BF00210F
:1096E00001218C4B597089490D61DFF834C2CCF8E7
:1096F00000408C4C4FF0020CC4F800C0DFF828C2C8
:10970000CCF80060DFF808C23D32CCF80020C1F888
:1097100000524FF0E0224FF4807CC2F880C2C1F8C2
:109720000403C2F800C10804804908601D7070BDC0
:109730007F4A4FF40030012BC2F8401518BFCCF817
:109740000803C2F8404108BFCCF80403CCF8440336
:1097500070BD67480068704770B5764805687749FE
:1097600075480860614CD4F84001002601280AD1F0
:10977000D4F8080310F4803F05D04FF48030C4F8CB
:109780000803C4F84061D4F8440101280DD1D4F88D
:10979000080310F4003F08D04FF40030C4F8080369
:1097A000C4F84461012007F088FCD4F8480101287E
:1097B0000DD1D4F8080310F4802F08D04FF4802086
:1097C000C4F80803C4F84861022007F076FC5C483E
:1097D000056070BD574810B5046858495648086080
:1097E0004C490878002808BF03201AD0464A4FF099
:1097F00000401060454AC00BC2F8080303124FF046
:10980000E02C0020CCF88031414B1860C2F84001B8
:10981000C2F8000208704A78002A1CBF4870002075
:1098200001D007F04AFC4648046010BD4FF0E0212B
:109830004FF08070C1F8000270474FF0E0214FF008
:109840008070C1F8800270474FF0E0214FF40010A3
:10985000C1F8000270474FF0E0214FF40010C1F84A
:10986000800270472949012008614FF0E021000281
:10987000C1F880027047410A43F609525143C0F3D0
:10988000080010FB02F000F5807001EB50207047DB
:10989000430B48F2376C03FB0CF31B0C4FEA432CD1
:1098A000C1F800C0DFF89CC003FB0C0326484CF253
:1098B000F72C5843400D10FB0CFC0CEB432303F535
:1098C00080735B1213700A6810440860704719486F
:1098D00010B5046819491848086007F087FF184850
:1098E000046010BD0BE000E018E000E000B00040B4
:1098F00004B500404081004044B1004048B1004000
:1099000048B5004040B5004008F5014000800040E7
:10991000408500402C00002044B5004008B00040C5
:1099200004850040088500401085004004F5014092
:1099300004B000401005024001000001180502407B
:1099400014050240F7C2FFFF6F0C010010B5EFF3E2
:10995000108000F0010472B6EB484178491C417058
:109960004078012801D108F0A5FB002C00D162B697
:1099700010BD70B5E44CE07848B90125E570FFF7FB
:10998000E5FF08F09FFB20B1002008F07BFB0020E2
:1099900070BD4FF080406571C0F80453F7E770B5B3
:1099A000EFF3108000F0010572B6D74C607800B973
:1099B000FFDF6078401E6070607808B908F07EFBB9
:1099C000002D00D162B670BDCF4810B5C17821B16D
:1099D00000214171C170FFF7E2FF002010BD10B5FA
:1099E000044608F06FFBC849C978084000D0012040
:1099F0002060002010BD2DE9F05FDFF80C93427865
:109A0000817889F80620002589F80710064689F82C
:109A1000085000782F4620B101280FD002280FD01F
:109A2000FFDF08F05CFB98B108F060FBA8420FD1A3
:109A3000284608F05FFB0028FAD047E00125F0E750
:109A4000FFF784FF08F03EFB0028FBD00225E8E783
:109A500001208407E060C4F80471AC490D6001077F
:109A6000D1F84412A94AC1F3423124321160A74906
:109A70004FF0020B34310860C4F804B3A060DFF883
:109A800090A2DAF80010C94341F3001101F1010876
:109A9000DAF8001041F01001CAF8001000E020BF11
:109AA000D4F804010028FAD0284608F023FB002847
:109AB000FAD0B8F1000F05D1DAF8001021F010014A
:109AC000CAF80010C4F808B3C4F8047199F8070084
:109AD0004C4670B1307860B908F0F4FA064608F0E8
:109AE000E5FC6FF0004116B1C4E9031001E0C4E9E0
:109AF000030115B12771BDE8F09F01202071BDE879
:109B0000F05F00F0DFB870B5050000D1FFDF4FF067
:109B100080424FF0FF30C2F808030021C2F8001164
:109B2000C2F80411C2F80C11C2F81011764C617021
:109B300008F0CEFA10B10120E07060702846BDE850
:109B4000704058E72DE9F0410125AF077D616E4C6B
:109B5000E079F0B1012803D0217A401E814218DA61
:109B600008F0B0FA064608F0A1FCE179012902D913
:109B7000217A491C21720EB1216900E0E168411A85
:109B8000022902DA11F1020F0EDC0EB1206100E0B1
:109B9000E060FFF7DBFE08F095FA10B13D61A570BB
:109BA00000E0257000202072BDE8F0812DE9F05F13
:109BB0005848D0F800B0574A574908321160840617
:109BC000D4F8080110B14FF0010801E04FF000088F
:109BD000D4F8000100B101208146D4F8040108B195
:109BE000012600E00026D4F80C0100B101208246D5
:109BF000D4F8100108B1012700E0002748EA090164
:109C000026EA010020EA0A00B84300D0FFDF002561
:109C1000B8F1000F04D0C4F80851012008F032FA5E
:109C2000DFF8E480B9F1000F13D0C4F8005198F8C0
:109C3000050020B188F80550002008F023FA98F8B4
:109C4000000030B108F03EFA18B1012088F8020097
:109C500020610EB1C4F80451BAF1000F0AD0C4F863
:109C60000C5198F80200464600B9FFDFB570357018
:109C7000FFF795FE37B1C4F8105198F8040008B109
:109C8000FFF760FF2349091DC1F800B033E770B545
:109C90001D4DE87808B908F011FA01208407A06189
:109CA000A87850B1D4F80C0120B9002008F022FAAD
:109CB0000028F7D10020C4F80C014FF0FF30C4F8A1
:109CC000080370BD2DE9F0411926B507C5F80863F2
:109CD0000124AC610020C5F80001C5F80C01C5F8ED
:109CE000100108F0EFF9084F10B1BC702C6100E0D2
:109CF0003C70FFF72BFE0549B87920310860C5F8A4
:109D000004636C6150E7000030000020180500403B
:109D100010ED00E0100502400100000110B5202008
:109D200000F075F8202000F07DF84449202081F8EB
:109D30000004434900060860091D42480860F7F71F
:109D4000E1FA3F49C83108603F48D0F8041341F0B8
:109D50000101C0F80413D0F8041341F08071C0F879
:109D60000413364901201C39C1F8000110BD10B59B
:109D7000202000F04CF8324800210160001D0160F5
:109D80002F4A481EE83A10602F4AC2F808032C4BAD
:109D9000C8331960C2F80001C2F860012B4908609D
:109DA000BDE81040202000F03DB825492848EC3996
:109DB0000860704722492648E8390860704770B546
:109DC0001F4A8069E83A224911601F49D1F80061B1
:109DD0000023204D1D4A5C1E1EB1A84206D300215F
:109DE0000FE0D1F8606186B1A84209D2C1F8003114
:109DF000C1F860311460BDE87040202000F012B856
:109E00001168BDE8704014F01AB9FFDF70BD00F0B2
:109E10001F02012191404009800000F1E020C0F8BC
:109E20008011704700F01F0201219140400980001D
:109E300000F1E020C0F880127047000020E000E050
:109E400000060240441300200000024000040240CB
:109E50000100000100F001004FF0E0214FF0007020
:109E6000C1F88001C1F88002384B802283F80024B9
:109E7000C1F80001704700B502460420344903E0F0
:109E800001EBC0031B792BB1401EC0B2F8D2FFDF3B
:109E9000FF2000BD41F8302001EBC00100224A71D3
:109EA0008A7101220A7100BD294A002102EBC0001B
:109EB0000171704710B50446042800D3FFDF244821
:109EC00000EBC4042079012800D0FFDF6079A1797C
:109ED000401CC0B2814200D060714FF0E0214FF0D1
:109EE0000070C1F8000210BD2DE9F0411948056865
:109EF00018491948083108601448042690F80004ED
:109F0000134F4009154C042818D0FFDF16E02178C4
:109F100007EBC1000279012A08D1427983799A427C
:109F200004D04279827157F8310080472078401C74
:109F3000C0B22070042801D300202070761EF6B233
:109F4000E5D20448001D0560BDE8F08119E000E09D
:109F5000C805002010050240010000014400002057
:109F60000F4A12680D498A420CD118470C4A1268F0
:109F70000A4B9A4206D101B508F066FAFFF715FFC1
:109F8000BDE80140074909680958084706480749DC
:109F9000054A064B7047000000000000BEBAFECA2A
:109FA00098000020040000204812002048120020E1
:109FB00018B1172802D207207047172008490880D7
:109FC0000020704706480088704770B50C4605466B
:109FD00000F0B5FB21462846BDE8704001F0B0BC5A
:109FE00046000020FE4B586019721A80C90013F019
:109FF000F4BF10B504460E2113F0CDFF17202081C9
:10A00000207B40F00A00207310BD4FF6FF720280E3
:10A01000032008F052BC7047027BD30701D192079E
:10A0200003D4408908800020704705207047027BD8
:10A03000920700D54181704701460020098847F208
:10A04000FE12114200D00120E549497A002901D0D1
:10A0500040F00800704700B50346007BC00701D000
:10A06000052000BD19811846FFF7E6FFC00703D0A1
:10A07000187B40F004001873187B40F0010018733F
:10A08000002000BD027B520700D509B1008970474E
:10A0900017207047027B61F3C302027370472DE9FA
:10A0A000F04F0E46017804464FF0010B0BFA01F019
:10A0B00047F2FF1100EA010961681D464FF6FF7380
:10A0C000088887B09646984206D0B9F1000F07D0AD
:10A0D00047F2FE12104203D0012007B0BDE8F08F16
:10A0E00040EA090008804FF0000A8DB185F800A011
:10A0F0002278002705200221102A72D2DFE802F020
:10A10000710D323B506A727C50C7C399CBFDFCFB8A
:10A1100020780B28ECD00420DFE76068B4F80C80CE
:10A12000007B80077ED5B8F1170F4BD3FFF74AFFAE
:10A130004045FAD360684089172801D3404541D192
:10A14000287820F03F00801C2870A5F801800320AB
:10A1500030806168A1F80A806068017B21F002010B
:10A16000017334E104212970A189A5F80110E18966
:10A17000A5F8031085E0A08A3188C01D1FFA80F879
:10A180004145D2D3062005F8010BA0892880E0893B
:10A190006880208AA88007200090A38AA2693EE0F8
:10A1A000082A10D008212970A189A5F80110E18999
:10A1B000A5F8031030806A1D694604F1100006F00E
:10A1C0004EFA10B1CCE01021EDE730889DF8001078
:10A1D000084456E00A202870A089A5F80100032051
:10A1E00008E006E10C212970A189A5F80110E18998
:10A1F000A5F803103080A8E0A089B6F800C00BEBEA
:10A2000040021FFA82F8C44578D3B8F1050F75D320
:10A210000E222A70CDF800B0226903EA400320899B
:10A2200080B200E079E0714600F096FAA6F800806E
:10A23000CDE06B48427A002A6FD0521E42724068CD
:10A24000227B236900EBC205AA882868D3F800C0E6
:10A250001044A0F1080240F808CC586850608DF80E
:10A2600000108DF801A028680290A888ADF80400BD
:10A2700000216846FBF758FAA5F804A0002E01D08B
:10A2800050463080A3E0287840F08001297028787B
:10A2900040F040012970E0893188C01C1FFA80F825
:10A2A00041455DD3287820F03F0012302870A18905
:10A2B000A5F80110032000902089E38980B271463F
:10A2C000226900F049FAA6F80080287841063CD5BA
:10A2D00000067CD58DF800B08DF801A03188CDE95D
:10A2E000025A091DDFF8F8800420ADF8041004902C
:10A2F00098F8080003E055E04BE02AE030E08DF8E4
:10A30000140000216846FBF70FFA074630880C302E
:10A310003080022F02D0DFB36EE047E09DF81420BA
:10A32000D8F8041098F80830404601EBC2019A4270
:10A3300016D28A88A2B9427A521C88F809200D6088
:10A3400030888880A6F800A056E06168A0898880DF
:10A350003DE0218A3288491D1FFA81F8424501D229
:10A36000042749E0297821F03F0116312970A1899D
:10A37000A5F80110E189A5F8031000902089238A2F
:10A3800080B27146626900F0E7F9A6F80080DCE768
:10A390001DE0287820F03F0018302870207B68707E
:10A3A000318014E060680188090401D4052723E0A6
:10A3B000C088A189884201D006271DE01E20287090
:10A3C000A6F800B06068018821F400410180B9F16D
:10A3D000000F11D00248002200888300032001E012
:10A3E000E8050020A16808F0CBF961682078887042
:10A3F00007E0A6F800A003276068018821EA0901A8
:10A400000180384669E62DE9F04F87B09B46119CE4
:10A410000D46030016461AD03078C10703D000F06D
:10A420003F00192801D9012100E000212046FFF753
:10A4300029FE98420BD32088A0F57F41FF3906D032
:10A440003078410601D4000603D5082045E60720F0
:10A4500043E600208DF800008DF8010030785F1E83
:10A4600000F03F0C0122981E4FF0050A4FF0020940
:10A47000B9B2BCF1200F76D2DFE80CF08C10755F1A
:10A480007569758D759E75B775BC75CA75D675E39A
:10A49000757575F375F175F075EF758C052B79D1C0
:10A4A00004208DF80000A0788DF804007088ADF8C5
:10A4B000060030798DF80100707800F03F000C281C
:10A4C00029D00ADCA0F10200092863D2DFE800F0FD
:10A4D000126215621A621D622000122824D004DC68
:10A4E0000E281BD01028DAD11BE016281FD0182800
:10A4F000D5D11FE02078800701E0207840070028B0
:10A5000048DAF0E020780007F9E72078C006F6E79F
:10A5100020788006F3E720784006F0E720780006F0
:10A52000EDE72088C005EAE72088C004E7E7208837
:10A530008004E4E720884004E1E72078800729D5FB
:10A54000032B27D18DF800A0B6F8010082E0217816
:10A5500049071FD5062B1DD381B27078012803D07F
:10A56000022817D102E0CBE0022000E010200622F2
:10A570008DF8002072788DF80420801CB1FBF0F279
:10A58000ADF8062092B242438A4203D10395ADF85A
:10A590000890A8E07AE02078000777D50721B8B2C4
:10A5A0008DF800108108ADF80410B0EB810F6DD16B
:10A5B0000295ADF8062096E02178C90666D5022BF3
:10A5C00064D381B208208DF80000707802285DD332
:10A5D000B1FBF0F28DF80400ADF8062092B24243D0
:10A5E0008A4253D1ADF808907CE0207880064DD5A2
:10A5F000092003E02078400648D50A208DF80000A5
:10A60000A088ADF80400ADF80610ADF8082069E0A8
:10A610002078000672D50B20ADF804108DF80000EC
:10A62000ADF8062002955EE02188C90566D5022BAB
:10A6300064D381B20C208DF80000707804285DD3BB
:10A64000C6E72088C00459D5012B57D10D208DF8BD
:10A650000000A088ADF8040045E021E026E016E007
:10A66000FFE72088800449D5052B47D30E208DF8BD
:10A670000000A088ADF80400B6F803005B1FADF839
:10A680000830ADF80600ADF80AA02BE036E02088CF
:10A69000400433D5012B31D10F208DF8000022E08A
:10A6A000208800042AD4B6F80100E080207B00074F
:10A6B00024D5032B22D3307800F03F001B2819D07B
:10A6C00011208DF80000208840F40040A4F800001C
:10A6D000B6F80100ADF80400DB1E0320ADF806302B
:10A6E000ADF80800039559466846FBF71DF80500CC
:10A6F00008D016E010208DF80000E9E7072510E0EB
:10A7000008250EE0307800F03F001B2809D01D28F6
:10A7100007D00320109908F0D0F8208800F40040FA
:10A720002080207B400708D52046FFF785FCC00726
:10A7300003D1207B20F0040020732846CDE400B52F
:10A7400087B0032806D18DF80000019100216846EA
:10A75000FAF7EAFF07B000BDF8B51C4615460E46ED
:10A76000069F04F013FC2346FF1DBCB231462A4667
:10A77000009404F052F8F8BD2DE9FF4F8FB0054664
:10A78000DDE91C471198DDF880B0082805D0E8699C
:10A7900001F031F950B11020CDE02088092140F0BE
:10A7A000100020808BF80010022017E0E9690120DA
:10A7B0008871EA694FF420519180E9698872E969EA
:10A7C00042F601000881E969002088732088112180
:10A7D00040F0200020808BF800100420814638785B
:10A7E0000B900A2038704FF0020A05F11800564607
:10A7F0000D9001F0A1FB4C467CE0119810280DD182
:10A80000022E0BD0AAEB0400801C80B2009021988D
:10A81000022380B206AA1F9901F0DDF8BDF81A10D4
:10A820001298814203D9F648007A109004E003D1CF
:10A830000B9808B1387031E02198CDF800A080B2B3
:10A840004FF002030DF11A021F9901F0C4F81E988F
:10A850000088811BA1EB090083B2C9F1FF00984277
:10A8600000D203460AEB090292B20DF130080292BF
:10A8700000202199CDF81480CDE903101F9910987C
:10A88000CDE9000195F82010BDF81A00002201F072
:10A89000D5FB387050B1C0B2832803D0BDF81A0080
:10A8A000288334E0022013B0BDE8F08FBDF83000FB
:10A8B000022E00EB0901CCB20CD09BF80110A14292
:10A8C00005D1BDF82410814206D0FF2C04D09BF89E
:10A8D00001401EE08BF80140C94800680178052955
:10A8E00002D1BDF81A1081800AEB04001FFA80FA29
:10A8F000301986B206AB219A10990D9801F01FFB12
:10A9000028B91E980088801BA042BFF676AF022EA1
:10A9100012D0119810280BD1AAEB0400801C80B231
:10A9200000902198022380B206AA1F9901F053F8E3
:10A930001E980680002038700020B4E72DE9F84307
:10A940009446089E02460027F06BB0B3521F94B2A3
:10A95000B6F84220A2F57F45FF3D05D08518AD88A9
:10A960002A44921D95B200E000252A19B6F84080CD
:10A970000832424522D84219BCF8010022F8020BE5
:10A98000BCF8030022F8020B98B222F8024B894669
:10A99000904604F0E9FA4FF00C0C49464246234633
:10A9A000CDF800C003F000FFA6F84250F16B002084
:10A9B0002944A41D2144088003E001E0092700E0A8
:10A9C00083273846BDE8F88310B50B88B0F84040BF
:10A9D0009C420CD9C46BE018048844B1848824F4E8
:10A9E0000044A41D23440B801060002010BD822071
:10A9F00010BD2DE9F0478AB0002590468946824671
:10AA0000ADF81C5007274DE00698068880880004A2
:10AA100048D4A8F8006008A8CDE90450CDE9007535
:10AA2000029503954FF4007300224946304601F029
:10AA300005FB04003DD1BDF81C00ADF824000699CB
:10AA400008888A88B04216D1130414D40595CDE93C
:10AA5000007522F4004202950395049542F4804368
:10AA60004A88494601F0CDF804000BD10698818848
:10AA700041F40041818006AA09A95046FFF7A4FFCE
:10AA80000400DCD00595CDE9007506980395029584
:10AA900004950088BDF820300022494601F0B1F845
:10AAA000822C06D106AA07A95046FFF78DFF0400A5
:10AAB000AAD0ADF81C5004E00698818821F400412A
:10AAC000818006AA07A95046FFF77EFF0028F3D031
:10AAD000822C03D020460AB0BDE8F0870020FAE7B8
:10AAE00030B50446C06B85B0002578B10C208DF8D8
:10AAF0000000B4F84000ADF80800E06B039101904D
:10AB000000216846FBF78DFC8DF8005044F83C5F4F
:10AB10004FF6FF70E080A58005B030BD2DE9F04113
:10AB200005460F46E96B0020069E1446002911D009
:10AB3000012B0FD1324639462846FFF75AFF00282D
:10AB400008D1002C06D0324639462846BDE8F041EF
:10AB500000F060BFBDE8F081F8B51D46DDF818C013
:10AB6000DDE907634C1DBCF800E0A4B2099FA645CF
:10AB700001D20720F8BDACF80040172403F8014BC0
:10AB800018805A80052000900B46B8B22A463146FC
:10AB900000F021FF0020F8BD70B50D4604464C21A1
:10ABA00013F01BFA04F1080044F81C0F00204FF6C4
:10ABB000FF712062E184A08425711720208514F89C
:10ABC0002C0F40F00A00207070BD4FF6FF7202801B
:10ABD000042007F072BE30B585B00D460446FFF77D
:10ABE0007FFF208F38B101208DF8000000216846DA
:10ABF0000195FBF716FC002020636063A0638BE7E0
:10AC0000F405002090F84820920703D4408808807B
:10AC1000002070470620704790F84820920701D521
:10AC2000A0F8461070470146002009880A0700D5A1
:10AC3000012011F0F00F01D040F00200CA0501D54B
:10AC400040F004008A0501D540F010004A0501D506
:10AC500040F02000090501D540F04000704700B5E4
:10AC6000034690F84800C00701D0062000BDA3F8B5
:10AC700044101846FFF7D7FF10F0760F05D093F871
:10AC8000480040F0040083F8480013F8480F40F0F3
:10AC900001001870002000BD90F84820520700D530
:10ACA00011B1B0F8440070471720704710F8482FD2
:10ACB00061F3C302027070472DE9FF4F9BB006009D
:10ACC000DDE92CB4289F1E9D2A9B25D02878C1073A
:10ACD00003D000F03F00192801D9012100E0002134
:10ACE0002046FFF7D9FFB04216D3287841060FD48B
:10ACF00000F03F011E2909D0218811F47F6F0BD18C
:10AD00003A884AB1A1F57F42FF3A05D0010606D53F
:10AD100000F03F00122802D004201FB0C4E5F8491B
:10AD20001C984FF0000908728DF818908DF83C902F
:10AD30000FAA0A602B9A4A60ADF81C90ADF85090AB
:10AD40002A789A4602F03F0C0420711F04F1180380
:10AD50004FF007084FF0030E1693BCF11F0F7DD282
:10AD6000DFE80CF07C7C107C257CA97CFD7CFC7CE5
:10AD7000FB7CFA7CFD7CF97C7C7CF87CF77C7C7C21
:10AD80007C7CF60094F84820B5F80110920701D5B4
:10AD9000032E02D08DF8180039E34FF40060ADF8AF
:10ADA000500061808DF83CE0ADF84010F1E2052ED6
:10ADB000F0D1B5F801002083ADF81C00B5F8031000
:10ADC000618300286BD0884269D80020A07220815E
:10ADD0004FF6FF706084169801F0AEF805208AF8EF
:10ADE00000000220804601900AAB5A461C99169832
:10ADF00001F0A5F898BB9DF82E00012804D002218F
:10AE00008AF80110102003E001208AF801000220D6
:10AE10000490002203A90BA805F021FCF0BB9DF8CB
:10AE20000C00049981423CD13A88801CA2EB0801B5
:10AE3000814236DB019800901FFA8BF002230DF15E
:10AE40002A02299900F0C7FD019808F10208801C28
:10AE500081B2019117AA03A90BA801E0B8E223E08F
:10AE600005F0FDFB019900911FFA8BF09DF80C3065
:10AE700017AA299900F0AFFD9DF80C000AAB08EB6A
:10AE800000011FFA81F801995A46084480B20190E6
:10AE90001C99169801F053F8002801E001E095E0B4
:10AEA000B7D0B8F1020F03D10A208DF818006DE277
:10AEB000A7F800806AE2072EFFF46CAFB5F8010036
:10AEC0002083ADF81C00B5F80310618300287DD005
:10AED00088427BD80120A072B5F8050020810020AF
:10AEE000A073E06900F087FD78B9E16901208871FD
:10AEF000E2694FF420519180E1698872E16942F67C
:10AF000001000881E16900208873F01F60841D98AA
:10AF1000A062A4F82480169801F00EF88AF8008048
:10AF20000120804602900020ADF82A002BE000BFEF
:10AF3000B8F1010F1DD0E0698079012803D1BDF877
:10AF40002800ADF80E00029800901FFA8BF007E081
:10AF50002BE2ADE13BE1DCE025E29FE076E03BE087
:10AF6000042303AA299900F036FD0298001D80B23F
:10AF70000290BDF82A00ADF80C00ADF80E0008F103
:10AF800004001FFA80F80AAB5A461C99169800F084
:10AF9000D6FF20B93988A1EB08000428C8D2B8F13F
:10AFA000010F81D0E0698079012805D0BDF8281013
:10AFB000A1F57F40FF3803D1BDF82800ADF80E00A1
:10AFC000029800901FFA8BF0042300E014E003AA1B
:10AFD000299900F000FD6BE7072E02D0152E7FF4B3
:10AFE000D9AEB5F801002083ADF81C00B5F80320F8
:10AFF000628308B1904201D90120CBE60120A07202
:10B0000000202081A073052E07D0C8B2691DE26917
:10B0100005F006FB00287FF447AF4FF6FF70608411
:10B02000299803A9029781E8010C06A814A9CDE983
:10B0300000102878002300F03F0220461C99FFF7FB
:10B040009BFB8146208BADF81C009FE1032ED4D1E1
:10B050004020ADF85000B5F801002083ADF81C0089
:10B060000DF1300C01230021CDF814C00293CDE97D
:10B0700003B1299A1C99CDE9001239880022491E92
:10B080008BB294F8201000F0D9FF8DF8180090BB17
:10B090000B208AF80000BDF8300038E0052EACD156
:10B0A0008020ADF85000B5F801002083B5F80310FA
:10B0B0006184ADF81C00B1F5007F02D98DF81880CD
:10B0C000A5E141F47C4262840DF1280800214FF093
:10B0D000010CCDE90418CDE902CB299B1C99CDE9DF
:10B0E00000133988491E8BB294F8201000F0A6FF97
:10B0F0008DF8180030B18328A7D10220D6E00000D7
:10B10000F40500200D218AF80010BDF82800401C2D
:10B110003BE1D10901EB41030EEB8301B14204D9BC
:10B1200051067FF56AAF00202FE1B5F80100ADF8B8
:10B130001C002A78520609D506228DF83C202A7870
:10B14000120605D500208DF83C0043E18DF83C80C7
:10B150004FF0030C4FF00008CDF808C0CDE903B85C
:10B16000DDE91C23CDF81480CDE90023A6EB010B0B
:10B170001FFA8BF394F82010424600F042FD8DF840
:10B1800018008DF83C80297849060DD52088C00527
:10B1900006D5208BBDF81C10884201D1C4F8288048
:10B1A00040468DF81880F0E0832801D14FF0020965
:10B1B0004FF48070ADF85000BDF81C002083A4F857
:10B1C00022B01D98A0620320A0841321DAE0052E8E
:10B1D000FFF413AFB5F80100ADF81C00B4F840203F
:10B1E0007AB3A2F57F43FE3B2CD008228DF83C2099
:10B1F0004FF0050C4FF00008CDF808C0CDE903B8BA
:10B20000DDE91C23CDF81480CDE9002389B241F497
:10B210000043B5F8032094F8201000F0F2FC8DF8FC
:10B220003C804FF400718DF81800ADF85010832861
:10B2300013D010B3B4F84010A1F57F40FE3809D008
:10B24000E5E0FFE70B228DF83C204FF6FE72A4F8F4
:10B250004020CDE7A4F84080D9E05B462A46009420
:10B2600030461D99FFF76AFB8DF8180008B1832856
:10B270004CD1BDF81C0020833FE75B462A46009472
:10B2800030461D99FFF75AFB8DF81800F0BBB4F853
:10B290004210E06B299A431801A8009780E8040C3B
:10B2A0005A88998833F8060BFFF756FC81466DE003
:10B2B00095F80180022E75D15FEA080002D0B8F13E
:10B2C000010F6FD109208DF83C0007A800908DF880
:10B2D000408094F82010434600222046FFF71EFCD1
:10B2E0008DF8410000218DF8421058B9B8F1010FD6
:10B2F00015D0B8F1000F05D1B4F84010A1F57F408A
:10B30000FF380CD0B4F8400048B100E03EE0002027
:10B310008DF83C004FF48060ADF850000EE00FA8AF
:10B320002B99FBF77EF8814600208DF83C004FF406
:10B330008060ADF85000B9F1020F06D0F8480068FF
:10B34000807928B18DF8180028E0A4F8188043E02F
:10B35000B9F1000F03D081208DF818003CE007A858
:10B36000009094F82010434601222046FFF7D6FBB8
:10B370008DF8180059462046FFF7B2FB9DF81800DB
:10B3800020B919218AF80010012038809DF83C006E
:10B3900020B10FA82B99FBF744F88146B9F1000FB3
:10B3A00032D019E016E00620F4E42078000711D529
:10B3B000012E0FD10A208DF83C00E088ADF8400046
:10B3C0005946042007F079FA0820ADF85000AAE6A3
:10B3D0005106E9D54FF004092088BDF85010084304
:10B3E0002080BDF8500080050CD5B4F84010A1F5C0
:10B3F0007F40FE3806D11D9820631E986063268723
:10B400004FF00309484688E49DF8180078B1012000
:10B410008AF8000029788AF80110BDF81C10AAF8F3
:10B4200002109DF818108AF8041005203880208832
:10B43000BDF8501088432080E4E72DE9FF4F97B016
:10B44000804601780120DDE926A488404FF20901F9
:10B450000840ADF8200021889B46A1F57F424FF0BF
:10B460000009FF3A02D028B1080703D501201BB01C
:10B47000BDE8F08F249E0020054630701999189A77
:10B480000988ADF84010A6498DF81C000A728DF8A5
:10B490002C000BA808602598486098F80000012847
:10B4A00037D0022809D003287ED1307820F03F0021
:10B4B0001D303070B8F80400E08098F800000228D1
:10B4C00004D1307820F03F001B30307094F84800F1
:10B4D000000769D513AB0020CDE904030721CDE9AE
:10B4E000001B0322CDE9022ABDF8400094F8201089
:10B4F000C01E83B2B8F80400002200F09FFD0028AF
:10B50000D2D1B8F80400A6F80100BDF84C00C01C68
:10B5100003E198F805108DF81C1098F80400012834
:10B5200006D04FF4007902282BD00328BCD171E15A
:10B530002088B8F8087010F40060ADF8200033D00F
:10B54000172F1CD3FEF73EFDB84218D3B4F84600BF
:10B55000172801D3B84212D1307820F03F00C01C28
:10B560003070A6F801700320ADF84000A4F84670D2
:10B5700094F8480020F0020084F848006CE10525AA
:10B5800085E1208808F1080700F4FE60ADF820008E
:10B5900010F0F00F1ED010F0C00F03D03888228BAF
:10B5A0009042ECD1B1B900E06BE1B878C00711D09E
:10B5B0000020B9680290CDE9030107210590CDE98B
:10B5C0000010FB88BA8894F82010388800F019FB26
:10B5D0000028D4D1BDF8200080284CD006DC1028EB
:10B5E0000DD020280BD040288AD124E0B0F5807FF0
:10B5F0006AD048457ED0B0F5806F97D1E2E0C006B2
:10B6000001D5082000E01020814605208DF82C008F
:10B61000002008A9ADF8300001AB009110AA07A8DE
:10B6200083E80508CDE9046A3B884A46072120469D
:10B63000FFF7A2F8A8E09DF81C004FF00A090028C7
:10B640009CD113ABCDE904030721CDE9001B0122F6
:10B65000CDE9022ABDF8400094F82010401E83B2C4
:10B66000208B002200F0EAFC8DF81C000B203070CB
:10B67000BDF84C001EE09DF81C004FF00C0900289E
:10B6800021D115ABCDE904030721CDE9001B01222F
:10B69000CDE9022ABDF84000628C401E83B294F8C6
:10B6A0002010208B00F0CAFC8DF81C000D2030709B
:10B6B000BDF85400401CADF8400005208DF82C006A
:10B6C000208BADF83000C7E03888B4F818C060456A
:10B6D0007FF455AF9DF81C004FF0120900281ED1D1
:10B6E000A06AB8B1B878C0073FF449AF0020B96884
:10B6F000029000E016E0CDE9030107210590CDE9B5
:10B700000010FB88BA8894F82010604600F079FA9F
:10B710008DF81C00132030700120ADF840009BE034
:10B72000F4050020B7F800C0208B8445D0D19DF8E7
:10B730001C004FF016090028E06B06D0F0B3002083
:10B74000ADF808004FF6FF7729E078B1B978C9075E
:10B75000BED1B4F8421010AACDE9002BCDE9026A9F
:10B7600043185A88998833F8060B0BE0B878C0075D
:10B77000BAD010AACDE9002BCDE9026ABA88F988BF
:10B780006046BB68FFF7E8F9050065D0072D79D062
:10B790007DE00F4605AA02A92046FFF715F9B4F887
:10B7A0004220BDF808108A4201D00028F1D0B4F838
:10B7B0004210E26B00201144088000E04CE0A4F845
:10B7C000427049E09DF81C004FF0180940B1208BF1
:10B7D000D0B13888208351462046FFF781F93BE0FD
:10B7E00004F118000090237E94F8201001222046D6
:10B7F000FFF794F98DF81C000028ECD11920307067
:10B800000120ADF84000E6E7052551462046FFF748
:10B8100067F93CE0208800F40070ADF8200048454E
:10B820002FD1B4F84000A0F57F41FE3990D1D8F86F
:10B8300008004FF0160958B1E063B8F80C10A4F8EE
:10B8400040104FF6FF71A4F842100021018003E080
:10B850004FF6FF70A4F84000BDF8200030F47F617F
:10B860001AD0782300225146042006F089FF98F868
:10B87000000020712088BDF82010084320800EE0D1
:10B8800000E007252088BDF820108843208020880C
:10B8900010F47F6F1DD03EE02188814321809DF808
:10B8A0002C0028B16F4841680BA8FAF7BAFD05468D
:10B8B0009DF81C000028EAD086F801900120307025
:10B8C000208B70809DF81C0030710520ADF8400081
:10B8D000DDE7208FF8B119990988ADF84010DDE94E
:10B8E000242302A9059481E80C0410AACDE9002BB9
:10B8F000D4E90C231899FFF7DFF9054601208DF8EC
:10B900002C0000210BA8CDF830A0FAF78AFD00B179
:10B9100005460020208794F8480040070AD52046B5
:10B92000FFF781F910F0760F04D114F8480F20F0DA
:10B93000040020701998BDF840100180284696E553
:10B9400000B585B0042807D102208DF800000191D0
:10B9500000216846FAF765FD05B000BD10B5414A03
:10B9600003781168012B02D0022B2BD112E00B7847
:10B970000BB1052B01D104230B70136881889980CA
:10B980001168C388CB8013680189198111684089C7
:10B9900048810FE083888B801168C388CB8013684F
:10B9A00001891981136841895981116883898B81C3
:10B9B00000690861D2E90001FAF733FD022803D0DB
:10B9C000002800D0812010BD832010BDC06B00284E
:10B9D00000D001207047F8B51C4615460E46069F5C
:10B9E00003F0D4FA2346FF1DBCB231462A46009428
:10B9F00002F013FFF8BD8178012909D10088B0F564
:10BA0000205F03D042F60101884201D10020704737
:10BA100007207047F0B589B0002415460E4607464A
:10BA2000ADF8184011E0079801882980811D029423
:10BA3000CDE9034107210594CDE9001483884288AC
:10BA40000088314600F0DDF830B907AA06A938466B
:10BA5000FEF7BAFF0028E6D0822800D1002009B006
:10BA6000F0BD0000F405002010B58B7883B102789A
:10BA70009A4205D10B885BB102E08B79091D4BB16D
:10BA80008B789A42F9D1B0F801300C88A342F4D1F6
:10BA9000002010BD812010BD072826D012B1012A38
:10BAA00027D103E0497801F0070102E04978C1F3AA
:10BAB000C20105291DD2DFE801F00318080C1200AD
:10BAC0000AB1032070470220704704280DD250B1FC
:10BAD0000DE0052809D2801E022808D303E00628BD
:10BAE00003D0032803D005207047002070470F20A3
:10BAF00070478120704710B513880B800B781C06A7
:10BB00001FD5F64CA47A844204D843F01000087084
:10BB1000002010BD94682478C44064F304130B70B3
:10BB20001378D17803F0030341EA032140F20123A3
:10BB3000B1FBF3F403FB1411926800FB0120401CDD
:10BB400010BD906810BD37B5BDF8041011809DF888
:10BB5000045029061BD5E14901239468897A814262
:10BB600009D8FE280FD1E80602D58B405B1E00E005
:10BB70000023237007E0217883409943C5F3001325
:10BB8000834019432170107820F0100010703EBDE2
:10BB90002DE9F0410746C81C0E4620F00300B042D4
:10BBA00002D08620BDE8F081082A01D90E20F9E7ED
:10BBB000CA4D002034462E60AF802881AA72E880EA
:10BBC0001AE0E988491CE980810614D4E17800F084
:10BBD000030041EA002040F20121B0FBF1F201FB39
:10BBE0001201206800F021FB2989084480B22881D5
:10BBF000381A3044A0600C3420784107E1D400208A
:10BC0000D0E72DE9FF4F87B01646DDE9147A80466C
:10BC1000994623F4404500F0F8FA04000BD0207850
:10BC200000060AD5AD48817A0898814205D8872058
:10BC30000BB0BDE8F08F0120FAE7224601A9089871
:10BC4000FFF759FF834600208DF80800072F1BD00F
:10BC5000012221463846FFF71FFF0028E8D120784F
:10BC6000400611D502208DF80800BDF80400ADF89B
:10BC70000C80ADF80E00ADF810601698ADF81250BB
:10BC8000CDF818A0ADF814005FEA094004D50025EE
:10BC90002E46A84601270CE02178E07801F0030148
:10BCA00040EA012040F20122B0FBF2F1804602FBA3
:10BCB00011875FEA494009D5B84507D1A1782079B5
:10BCC00001F0030140EA0120B04201D3BE4201D994
:10BCD0000720ADE7A8191FFA80F9B94501D90D2051
:10BCE000A6E79DF8080020B102A8FAF798FB002803
:10BCF0009ED1B84507D1A0784FEA192161F3010020
:10BD0000A07084F80490199800B10580189850EA42
:10BD10000A0028D0189830B10BEB06002A46189973
:10BD200012F0C2F80FE017980BEB060880B25746E6
:10BD3000169E03F019F92B46F61DB5B23946424658
:10BD4000009502F031FD224601A90898FFF7D3FEC5
:10BD50009DF80400224620F010008DF8040001999F
:10BD60000898FFF7F0FE002062E72DE9FF4FDFF8AB
:10BD70006C9182461746B9F80610D9F8000001EB1D
:10BD8000410100EB810440F20120B2FBF0F187B0E9
:10BD900000FB11754E46DDF854802946089800F0E6
:10BDA00044FA316832898B46611A0C3101441144DE
:10BDB000B38889B28B4201D8842039E70899CEB282
:10BDC000310603D5B10601D5852031E7B9F806C0A3
:10BDD0000CF1010C1FFA8CFCA9F806C0169909B1E8
:10BDE000A1F800C0B10602D5C4F8088007E01044ED
:10BDF00080B2A9F80800191A01EB0B00A0602246D6
:10BE0000FE200899FFF79FFEE77025712078390A18
:10BE100061F301002A0AA17840F0040062F30101F5
:10BE2000A17020709AF802006071BAF80000E080FA
:10BE300000252573300602D599F80A7000E0012725
:10BE4000B00601D54FF000084E4600244FF0070918
:10BE50000FE00295CDE903580595CDE90095F088EE
:10BE60002146149B0A9AFFF7CCFE0028A5D1641C3A
:10BE7000E4B2BC42EDD30020DAE62DE9F04780467B
:10BE800000F0C3F9070005D000264446134D40F2E8
:10BE9000012916E00120BDE8F087204600F0B5F941
:10BEA0000278C17802F0030241EA0222B2FBF9F300
:10BEB00009FB1321006800F0B8F93044641C86B215
:10BEC000A4B2E988601E8142E7DCA8F10100E880A5
:10BED0002889801B288100203870DCE700060020BC
:10BEE00020B1401E108091700020704701207047E3
:10BEF00010B5D54904460088CA88904201D38220F3
:10BF000010BD096800EB400001EB80025079A0727F
:10BF1000D08820819178107901F0030140EA012056
:10BF2000A081A078E11CFFF7E6FD20612088401C7D
:10BF30002080E080002010BD0121818270472DE922
:10BF4000FF4F83B04FF6FF780546A3F800804068A6
:10BF50001F4680788DF8060068680088ADF80400F8
:10BF600000208DF80A00A88A2C88A04200D304463D
:10BF7000AC8242E0A88A401CA882701D6968FFF765
:10BF800073FDC0BB3988414501D1601E3880688887
:10BF9000A04237D3B178307901F0030140EA01299A
:10BFA00001A9701DFFF760FD28BB698941452ED0AE
:10BFB000002231460498FFF76FFDE0B969894945D1
:10BFC00019D10598D5F810B0B5F80CC0D6F808A06E
:10BFD00080B2CDF800C002F0C7FFDDF800C05946BE
:10BFE0000CF1070C1FFA8CFC52464B46CDF800C0F2
:10BFF00002F09DFB58B1641CA4B2204600F005F984
:10C000000600B7D1641EAC82822007B011E67C80A6
:10C010007079B871F088B8803178F07801F0030158
:10C0200040EA01207881A7F80C90287A324607F17F
:10C030000801FFF760FD38610020E6E72DE9FF4FBA
:10C0400087B01C46DDE9158B91460F46DDF864A0EC
:10C05000079800F0DAF8050008D02878000607D520
:10C060007948807AB84203D88720E1E50120DFE5EE
:10C07000C9F309062A4601A93846FFF73CFD0746E1
:10C08000149807281BD000222946FFF705FD002839
:10C09000EBD12878400612D501208DF808000798CA
:10C0A000ADF80C00BDF80400ADF80E00ADF810605E
:10C0B000ADF8124002A8FAF7B2F90028D5D12978D4
:10C0C000E87801F0030140EA0121AA78287902F01A
:10C0D000030240EA02204E4507D0B1F5007F04D9A3
:10C0E000611E814201DD0B20A2E5864201D90720B5
:10C0F0009EE5801B85B2A54200D92546BAF1000F06
:10C1000001D0AAF80050189818B1B9192A4611F0B0
:10C11000CBFEB8F1000F0ED017983E4480B24446D3
:10C120005F4602F033FF2146FF1DBCB232462B466C
:10C13000009402F072FB00207AE52DE9F0411D46E3
:10C1400017460E4600F061F8040008D0207800067B
:10C1500007D53D48807AB04203D8872022E50120E8
:10C1600020E5224639463046FFF7C5FC65B1217807
:10C17000E07801F0030140EA0120B0F5007F01D82A
:10C18000012000E00020287000200BE52DE9F0419F
:10C190001D4617460E4600F038F8040008D02078F7
:10C1A000000607D52848807AB04203D88720F9E4F2
:10C1B0000120F7E4224639463046FFF7C4FCFF2D44
:10C1C00014D02178E07801F0030240EA022040F226
:10C1D0000122B0FBF2F302FB130015B900F20120BB
:10C1E00080B2E070000A60F3010121700020D9E400
:10C1F00010B50C4600F009F828B1C18821804079BB
:10C20000A070002010BD012010BD0F49CA888242D5
:10C2100009D340B1096800EB40006FF00B0202EB5C
:10C2200080000844704700207047C0B2820609D4DD
:10C23000000605D50448807A4843401C80B2704708
:10C2400008467047002070470006002010B506F031
:10C250001BFD05F088FFF6F7D7FD10F011FE06F084
:10C26000EBFBBDE8104006F09DBC10B50C4601F09C
:10C27000A4FE80B3204600F0A8FA68B322780F2A03
:10C2800009D0102A07D0022A05D0032A03D0142A85
:10C290002ED0FFDF1DE0A0781E282DD00EDC0C284C
:10C2A00024D008DC092827D2DFE800F0132617265F
:10C2B000261E1E1A1C0012281ED11BE0302819D081
:10C2C0001ADDA0F13A00032816D2DFE800F01115BC
:10C2D0000B00002010BD13E010E043F20200F9E76C
:10C2E0000420F7E70D20F5E70F20F3E70820F1E73A
:10C2F0001120EFE70720EDE70320EBE7FFDFE8E79A
:10C30000FFDFE6E700F061BA70B5034600200246A1
:10C310006FF02F050EE09C5CA4F130060A2E02D3CC
:10C320004FF0FF3070BD00EB800005EB4000521C69
:10C330002044D2B28A42EED370BD30B50A240AE05E
:10C34000B0FBF4F304FB13008D18303005F8010C3A
:10C35000521E1846D2B2002AF2D130BD30B50023A9
:10C360004FF6FF7510E0040A44EA002084B2C85C6E
:10C370006040C0F30314604005EA00344440E0B27A
:10C380005B1C84EA40109BB29342ECD330BD0000AA
:10C3900010B50AF04CF8042803D00AF048F8052834
:10C3A00002D108F05FFD50B90AF0FEF8032803D06F
:10C3B0000AF000F9032804D107F0EFFC08B10120CE
:10C3C00010BD002010BD70B50C460546062102F0D8
:10C3D00068FC606008B1002006E00721284602F0F2
:10C3E00060FC606018B101202070002070BD022048
:10C3F00070BD2DE9FC470C4606466946FFF7E3FF92
:10C4000000287DD19DF8000050B107F022FCB04219
:10C410007CD0214630460DF020F9002873D115E07C
:10C4200008F039FAB04271D0214630460BF0CAFF0D
:10C43000002868D1019D95F8C000503518B9687E74
:10C4400008B1012000E00020804603E0019D95F83E
:10C45000698050354FF0010A95F835004FF000091A
:10C46000A0B195F83600800710D584F8019084F8C3
:10C4700000A084F80290A68095F83710A171298F4A
:10C480002181698F618185F835903CE0304602F06A
:10C490007DFD070000D1FFDF384601F078FF10F086
:10C4A000FF0008D084F801900D212170A680E08063
:10C4B00084F802A027E0304602F056FD070000D1C4
:10C4C000FFDFB8F1000F21D0384601F0F0FFB8B11E
:10C4D0009DF8000038B90198D0F8E4004188B142D5
:10C4E00001D180F80090304607F075FA84F8019089
:10C4F0000A21217084F80290A680A97EA17100E033
:10C5000004E085F819900120BDE8FC870020FBE7D6
:10C510001CB56946FFF757FF00B1FFDF684601F021
:10C52000A0FDFF4900208968A1F8C2001CBD2DE9CB
:10C53000FC4104460E46062002F05EFB054607203D
:10C5400002F05AFB2844C7B20025A8463E4417E033
:10C550002088401C80B22080B04202D34046A4F81C
:10C56000008080B2B84204D3B04202D20020BDE8BD
:10C57000FC816946FFF727FF0028F8D06D1CEDB25B
:10C58000AE42E5D84FF6FF7020801220EFE738B5B5
:10C590004FF6FF70ADF800000DE00621BDF8000079
:10C5A00002F091FB04460721BDF8000002F08BFB6E
:10C5B0000CB100B1FFDF00216846FFF7B8FF00288B
:10C5C000EBD038BD2DE9F041D6A00679076807F019
:10C5D0006FFA0EF047FCD54C4FF004081020A4F879
:10C5E000388060874FF6FF70A4F85600002584F865
:10C5F0005850A4F85A0084F8315004F8345BCB4901
:10C6000004F8065C25702572C4F809703D31667324
:10C61000481E0CF051F8A5731B2020824FF4A47122
:10C620006182A082E1820A21217684F819800321A7
:10C63000A176E1760E212177072161770621A17786
:10C64000E1772084BDE8F08170B5B54C0D4660609F
:10C65000217007F0A8F9FFF79AFFFFF7B3FF2078E2
:10C6600009F099FC08F03CFA217860680BF043FF70
:10C6700020780DF0A9FF28460AF04EFB07F029FBB1
:10C68000217860680DF094F8BDE870400EF0EABBC8
:10C6900010B501240AB1002010BD21B1012903D039
:10C6A0000024204610BD02210FF030FEF9E72DE9ED
:10C6B000F047040000D1FFDF9C4D002695F83100C3
:10C6C00058B166701420207095F83200A07095F86B
:10C6D0003300E07085F8316068E0287840B12C22A2
:10C6E000A91C204611F0E0FB0F2020702E705DE0A9
:10C6F00095F82E0060B10120E07095F82F00A07031
:10C7000095F8300060701020207085F82E604DE0A4
:10C71000864802215A308246FFF709FF00B1FFDF49
:10C72000B5F85A90062002F067FA0746072002F093
:10C7300063FA3844C7B2781C00F0FF08B5F85A0015
:10C74000B84212D1204608F039F850BB95F83400B1
:10C7500078B36670122020702021A01C11F01BFC01
:10C760000220A07085F8346020E040451AD12046B0
:10C7700007F044FAE8B12078122817D1A0783C28B5
:10C7800014D1A088072102F08CFA050000D1FFDF48
:10C79000288807F020F9A088072102F094FA00B158
:10C7A000FFDF03E02146FFF724FE10B10120BDE8C2
:10C7B000F087FFE702215046FFF7B9FE18B9B5F838
:10C7C0005A104945BAD10020F1E770E710B509F0D9
:10C7D0005FFB00B1FFDF0BF08CFE00B1FFDF08F064
:10C7E00049F90AF082FA00B1FFDF0CF0DFFF00B177
:10C7F000FFDF07F038FA00B1FFDF0DF0DFFE00B118
:10C80000FFDFFFF7C4FEFFF7DDFE07F0B5F802F02B
:10C810009AFB0EF027FB454800210171012141716F
:10C820000222C270017010BD10B5404C207828B1B2
:10C830000A21BDE810400F2001F0D8BBFFF7A8FD8A
:10C8400008B10C2002E00EF053FB00202071012003
:10C8500060710A21E170207010BD70B5334D04463F
:10C86000287828B1BDE8704032210F2001F0BEBB0E
:10C87000207818B1012801D0122010E001F0C3FB8C
:10C8800020B10EF080FC08B10C2008E0207801F007
:10C89000A2FB04F11703E21D611C0EF081FB28715D
:10C8A000012068713221E970287070BD70B51F4C8D
:10C8B0000546207828B1BDE870400B210F2001F01B
:10C8C00095BB287818B1012801D012200EE0FFF79F
:10C8D0005FFD08B10C2009E0287801F07CFB691CA1
:10C8E0000EF0CDFA08B1002000E0072020710120F1
:10C8F00060710B21E170207070BD10B50B4C217878
:10C9000029B13021BDE810400F2001F06FBB008835
:10C910000EF03CFC302158B10020207109E00000ED
:10C9200048000020FFFFFFFF1F0000000C06002052
:10C93000217101206071E170207010BD70B5FF4C55
:10C940000546207828B1BDE8704031210F2001F064
:10C950004DBB01F058FB08B10C2005E0287800F031
:10C9600001000EF00DFC00202071012060713121CA
:10C97000E170207070BD10B5F04C207828B13421E2
:10C98000BDE810400F2001F031BB01F03CFB20B1AD
:10C990000EF0F9FB08B10C2002E00EF058FB00206D
:10C9A0002071012060713421E170207010BD10B53C
:10C9B000E24C217829B13621BDE810400F2001F06A
:10C9C00015BB0378411CA21D18460EF041FC08B1AE
:10C9D000002000E002202071012060713621E1700A
:10C9E000207010BD70B5D54C0546207828B1BDE843
:10C9F000704037210F2001F0F9BA287801F0EBFAE6
:10CA0000691C0EF0D1FB022508280AD00EF00FFD9C
:10CA100038B10168C4F80610808860810020207158
:10CA200000E02571012060713721E170207070BD38
:10CA3000C248017819B10F21084601F0D7BA002188
:10CA400001710F218170C170FF2181714FF6FF715B
:10CA50000181BB4949680A7882728A888281498843
:10CA6000C1810121417101707047B4490A781AB13E
:10CA700047210F2001F0BABA0088A1F85600012022
:10CA800081F8580000220A7148714722CA70087064
:10CA9000704710B5A94C207828B12B21BDE8104073
:10CAA0000F2001F0A3BA0821A01D05F0F5FB00201E
:10CAB0002071012060712B21E170207010BD70B5D4
:10CAC0009E4C217829B1BDE870403F210F2001F034
:10CAD0008DBA90F90000042816D0032814D098B11C
:10CAE000011D11D010F1080F0ED010F10C0F0BD05A
:10CAF00010F1100F08D010F1140F05D010F1280F0D
:10CB000002D01220207103E0002506F0DEF9257125
:10CB10003F20E07001206071207070BD10B5874C1F
:10CB2000217829B12A21BDE810400F2001F05EBA1A
:10CB3000A31D012200F110010FF097F800202071D1
:10CB40000F20A0702A20E07001206071207010BDBD
:10CB50002DE9FF41794C207828B146210F2001F0C2
:10CB600045FABDE8FF814FF0000884F80680B4F86C
:10CB70005600ADF8040002A9FFF725FC20B1002102
:10CB800001A8FFF7D4FCE8BBBDF80400ADF8000035
:10CB900002A980B2FFF717FC00B1FFDFBDF800006B
:10CBA00002F0F4F9050000D1FFDF2846039F01F0F1
:10CBB00085FC80F0010697F86950BDF8000002F08E
:10CBC000D3F9070000D1FFDF384601F070FC80F098
:10CBD000010255EA020019D0A179BDF8000004EB6A
:10CBE000410108815549A3791831585C65F300006B
:10CBF0005854A37962F341005854A27966F3820035
:10CC0000505400E00DE0A079401CA071002168465E
:10CC1000FFF78DFC28B9BDF80000BDF8041088426C
:10CC2000B6D1012084F8048060714621E170207043
:10CC300097E770B5414C0546207828B1BDE87040B3
:10CC400042210F2001F0D2B909F0F1FB052804D0F0
:10CC5000284609F08DF9002000E00C202071012009
:10CC600060714221E170207070BD10B5334C2078A6
:10CC700028B10E21BDE810400F2001F0B7B9A11D69
:10CC8000002006F029FF00202071012060710E2194
:10CC9000E170207010BD70B5284C0546207828B191
:10CCA000BDE8704040210F2001F0A0B901F0ABF9C0
:10CCB00038B10C202071012060714021E17020709A
:10CCC00070BD2946002006F0F4FE0020F2E770B5A2
:10CCD0001A4C0546207828B1BDE870403E210F204F
:10CCE00001F084B909F0C4F910B90AF0EBFA68B19F
:10CCF00028780AF060F8287808F0EBF80020207116
:10CD0000012060713E21E170207070BD0C20F6E7BB
:10CD100070B50A4C0546207828B1BDE8704017214F
:10CD20000F2001F063B901F06EF958B10C202071A9
:10CD3000012060711721E170207070BD0C06002089
:10CD4000480000202946012006F0B3FE0020EEE74F
:10CD500038B5FF4D0446287828B1BDE838404A214F
:10CD60000F2001F043B9227961798A4215D0A07968
:10CD7000E379984211D01F2A0FD81F290DD800221D
:10CD8000114610F0D7FB40B90022E079114610F0AF
:10CD9000D1FB10B9207A072801D9122015E04FF6EF
:10CDA000FF70ADF8000009F0FFFBA8B909F002FC24
:10CDB00090B909F03CFB78B900216846FFF7B7FB52
:10CDC00050B1204605F09AFF0020287101206871BB
:10CDD0004A21E970287038BD0C20F6E72DE9FC47A0
:10CDE000DB4C054694F82E0028B12821102001F0D4
:10CDF000FDF8BDE8FC87282084F83000012184F884
:10CE00002E10A8784FF000091A2825D00EDC16281D
:10CE100031D2DFE800F03030303030213030303087
:10CE20003030303030303030302121212A2822D0AB
:10CE30000BDCA0F11E000C281DD2DFE800F01C1C4A
:10CE40001C1C1C1C1C1C1C1C1C0D3A38042812D257
:10CE5000DFE800F0110211022888B0F5706F0AD2E5
:10CE60001F20884684F82F0028886946FFF7ABFA10
:10CE700018B1022019E0122017E09DF80000019F70
:10CE8000002806D007F1F607019E05D106F1DD0660
:10CE900004E007F1DC07F7E706F1F706684601F062
:10CEA000D5F808B1387818B10C2084F82F00A0E725
:10CEB00087F80080A878307084F82F90684601F0D9
:10CEC000D0F896E77CB5A24C0546207820B1252104
:10CED0000F2001F08BF87CBD28886946FFF773FAB4
:10CEE000002160B102202071A1602173E1800F2038
:10CEF000A0702520E0700120607120707CBD019A37
:10CF00001046503282F83E108368A360037B23737F
:10CF100092F83E30002BF5D12888E080E7E710B585
:10CF200040B10478406813B1B0F8440003E0B0F8B1
:10CF3000460000E0FB201B2908D3814206D8B2F549
:10CF4000A47F03D340F64800824201D9122010BDCD
:10CF5000002010BD70B57E4C0546207828B1BDE894
:10CF600070404C210F2001F041B8012666711F204E
:10CF700020710F20A0704C20E0702670EA88A988EC
:10CF800033460020FFF7CBFF30B900236A88298899
:10CF90001846FFF7C4FF08B12071CEE604F8426FCF
:10CFA000A888E080E8882081288860806888A08040
:10CFB0000020207004F83E0CBFE67CB5644D0446AA
:10CFC000287820B13A210F2001F010F87CBD01260D
:10CFD0006E711F2028710F20A8703A20E8702E7003
:10CFE00020886946FFF7EFF908B102200DE0A2881A
:10CFF000618801236846FFF792FF30B9A2886188F3
:10D0000000236846FFF78BFF08B128717CBD9DF8AF
:10D0100000100020002901990988E98028710199F0
:10D0200018D081F81961019A6188A2F81E11019A3D
:10D03000A188A2F82011019A6188A2F81A11019A18
:10D04000A188A2F81C11019981F81861019981F851
:10D0500019017CBD81F8F160019A6188A2F8F6108F
:10D06000019AA188A2F8F810019A6188A2F8F2103A
:10D07000019AA188A2F8F410019981F8F060019951
:10D0800081F8F1007CBD70B5314C0546207828B19F
:10D09000BDE870403C210F2000F0A8BF012666715A
:10D0A0000F20A0703C20E07026706A8829883346E3
:10D0B0000020FFF734FF30B900236A88298818461A
:10D0C000FFF72DFF08B1207137E604F8426F28887A
:10D0D00060806888A0802888E0806888208100209F
:10D0E000207004F83E0C28E670B5194D287828B158
:10D0F000BDE870403B210F2000F078BF95F842005A
:10D100002C1D00B1FFDFB5F848006080B5F84A007B
:10D11000A08001206070002121700F21A9703B21A7
:10D12000E970287009E670B5094D287828B1BDE886
:10D1300070403D210F2000F059BFFB262C1DEE80D2
:10D14000304600F04FFFA080E680304602E000004D
:10D150000C06002000F046FF2081012060700021B5
:10D1600021700F21A9703D21E9702870E5E52DE9B6
:10D17000FC41FC4C064694F82E0028B110210846CC
:10D1800000F034FFBDE8FC811F2084F82F00102040
:10D1900084F83000012784F82E7030886946FFF744
:10D1A00012F978B9684600F051FF58B1019D9DF819
:10D1B000000050350028019806D000F585700178F0
:10D1C00041B904E0022006E0D0F8E400F7E795F862
:10D1D000351019B13A2084F82F00D3E795F83610AE
:10D1E00089070CD1042101709DF8000020B9019934
:10D1F0003088D1F8E4104880684600F032FF002003
:10D2000084F82F0085F83570BCE72DE9F041D54C46
:10D210000546207828B1BDE8F0411D210F2000F01F
:10D22000E5BE1F202071012060711D21E17020707A
:10D2300009F0FDF80C2604283CD005283AD0A9793D
:10D240001220012904D019B1022901D0032926D1C5
:10D25000297809B1012922D1E97929B1012903D01D
:10D26000022901D003291AD1698843F6FD720B1FE8
:10D270003020934213D2AB881B1F93420FD22187D9
:10D28000A88860870027A87907F05DFD90B1E8794C
:10D2900007F0B0FD2878012804D030B10CE02071EF
:10D2A000BDE8F0810021022001E00021012007F00B
:10D2B000D0FD08B12671F3E72771F1E770B5A94CED
:10D2C000217829B1BDE870401E210F2000F08EBEEC
:10D2D0001F212171012161711E22E27021700278EB
:10D2E0001221012A00D01AB9407818B1012801D0C2
:10D2F000217122E500260C25012A08D009F097F8B3
:10D30000052802D008F071FD40B1257115E507F040
:10D3100031FD618F208F08F0B8FEF5E726710CE52E
:10D320002DE9F0478F4C0746B0F84600B4F844505A
:10D330000E46854200D3054600F054FE0146B4F87F
:10D340004600814203D8B7F8460000F04BFE804605
:10D35000A146B4F84840B7F84400844200D30446DC
:10D3600000F040FE0146B9F84A00814203D8B7F800
:10D37000440000F037FE4FF4A4721B2C01D0904201
:10D3800003D11B2D08D0904506D0F580A6F8088063
:10D390007480B08001203070BDE8F0872DE9FC5F1B
:10D3A0000546AFF680216F4ED1E900A196F82E0018
:10D3B000884628B1BDE8FC5F2121102000F016BE90
:10D3C0001F2086F82F00212086F830004FF0010B37
:10D3D00086F82EB0284600F052FE002811D109F040
:10D3E00026F805280CD009F022F8042808D096F871
:10D3F000340028B907F04FFAA0F57F41FF3901D07A
:10D400000C20D0E0062101A801F01CFC04007DD016
:10D4100003210EF061FAB6F85400A4F84400B6F8FF
:10D420005400A4F8460096F84D000090B6F8541049
:10D4300096F84C3020880A4601F0E1FC04287CD0A4
:10D4400000B1FFDF208806F0C5FA04F10D07B4F83B
:10D4500000900421384604F01FFF494638460EF07C
:10D4600078FB41A03F1D006800900321684604F04E
:10D470009EFE002069460A5C3A54401CC0B2032854
:10D48000F9D3288A6080688AA080A88AE08096F80C
:10D490004F2096F84E1020460EF0FFFC0146204625
:10D4A0000EF034FD4FF0000984F8569084F8579040
:10D4B0004F46687900F08FFD6076D5F80600C4F815
:10D4C0001A006889E083C4F808A084F80C8084F806
:10D4D000ECB004F1F0012046FFF722FF8DF8007058
:10D4E0000121684604F063FE9DF8000000F007018A
:10D4F000C0F3C1021144C0F3401008448DF800008D
:10D50000401D2076092804D2083001E013E014E021
:10D510002076002120460EF0DFF9287B07F013FC6F
:10D5200098B107F027FC69792879AA1D07F06DFCEE
:10D5300007001BD027E0092035E02088062101F0F4
:10D54000C2FB00B1FFDF07202DE0208806F043FA80
:10D550002088062101F0B7FB00283FF451AFFFDF20
:10D560004EE700000C060020112233002146032064
:10D5700007F06FFC070006D16A882988204608F06A
:10D5800036FD07000CD0208806F025FA20880621F9
:10D5900001F099FB00B1FFDF86F82F70BDE8FC9F1A
:10D5A000484684F8E09086F82F00F7E738B5FE4C3F
:10D5B000207820B122210F2000F018FD38BD1F2057
:10D5C0002071012565712220E070257094F83400E7
:10D5D00010BB08F02CFF052805D007F05CF9A0F57A
:10D5E0007F41FF3918D000202071684608F083FD84
:10D5F0000028E3D10098008806F0EDF90098062194
:10D60000008801F060FB00B1FFDFE84884F8345087
:10D610000078FCF74FFC38BD0C20207138BD2DE997
:10D62000F041E14D044695F82E0028B1BDE8F041E7
:10D630002321102000F0DABC1F2085F82F002320C2
:10D6400085F83000012085F82E00618840F67B4384
:10D650008A1F30209A4251D2A288961F9E424DD2F4
:10D6600091424BD8E188B1F5FA7F47D2218940F643
:10D670007746A1F10A03B34240D2B1EBD20F3DD9B4
:10D680006189A289914239D84FF00008208806218B
:10D6900001F007FB06004FF0020707D000F0C8FCBE
:10D6A00020B1D6F8E400017839B902E085F82F708E
:10D6B000F6E5D6F81011097809B13A201EE00521E7
:10D6C0008171D6F8E4004146A0F80880D6F8E4203D
:10D6D000A0885081D6F8E420E0889081D6F8E42034
:10D6E0002089D081D6F8E400028943899A4204D87F
:10D6F0008279082A01D89A4203D3122085F82F0094
:10D70000CEE522884280D6F8E400077085F82F1015
:10D71000C6E52DE9FE43A44C0646207830B103B09F
:10D720002421BDE8F0430F2000F060BC01256571A5
:10D730002420E070257030460EF02DFA08B100204C
:10D7400000E01220207100282CD184F83C50306871
:10D75000C4F83D00307984F841004FF0000884F8A7
:10D760003C806946062001F028FA00B1FFDF6846D8
:10D7700001F001FAA0B9BDF8047000BFBDF80400C3
:10D78000062101F08EFA060000D1FFDF86F8EC508A
:10D79000684601F0F0F918B9BDF80400B842EDD1BF
:10D7A00084F80480BDE8FE8370B57F4D064695F889
:10D7B0002E0028B1BDE870402621102000F016BCD4
:10D7C0001F2085F82F00262085F83000012085F8DD
:10D7D0002E003088062101F064FA040007D000F022
:10D7E00027FC20B1D4F8E400017831B901E002202F
:10D7F0000CE0D4F81011097809B13A2006E00521AF
:10D800000170D4F8E41030884880002085F82F009B
:10D810005AE46548017819B106210F2000F0E6BBF3
:10D82000002202710F2181700621C170C0F806200C
:10D83000C0F80A20F1218171012141710170704706
:10D840002DE9F041584D064695F82E0028B1BDE867
:10D85000F0412C21102000F0C9BB1F2085F82F00BB
:10D860002C2085F83000012085F82E003088062114
:10D8700001F017FA040007D000F0DAFB20B1D4F869
:10D88000E410087830B901E0022026E0D4F8100155
:10D89000007808B13A2020E08C200027005D10F0CD
:10D8A000010F19D0D6F802004860D6F8060088604B
:10D8B00054F8E40F718910228181206806F10C016F
:10D8C0000E3010F0F1FA21680320087021683088CA
:10D8D000488085F82F70E3E40C2085F82F00DFE402
:10D8E00070B5314D04460C26287828B1BDE870404B
:10D8F00018210F2000F07ABB08F056FE03284BD009
:10D9000008F058FE032847D0A07908B101282DD18E
:10D91000607928B1012803D0022801D0032825D13D
:10D92000A07B28B1012803D0022801D003281DD1F3
:10D93000607BD8B1C00819D162884FF48040824220
:10D9400002D82188814203D9207901280ED118E01C
:10D95000207930B1012814D0022805D0032805D140
:10D9600002E0202A0BD30CE0A0290AD22079042857
:10D9700005D12088202802D36188884201D9122647
:10D980000AE0607906F010FA30B1207985F83600A7
:10D99000204606F073FA064601202E7168711821A0
:10D9A000E9702870A5E400000C0600204800002063
:10D9B00010B5FE4C217829B11A21BDE810400F2086
:10D9C00000F014BB01781F2902D91220207106E053
:10D9D000002121710278411C104606F0C6FA012090
:10D9E00060711A21E170207010BD10B5EF4C2178E4
:10D9F00029B12021BDE810400F2000F0F7BA0178CE
:10DA00001F2902D91220207106E00021217102781D
:10DA1000411C104606F098FA012060712021E17047
:10DA2000207010BD2DE9FC41E04C217829B1BDE802
:10DA3000FC411B210F2000F0D9BA012767710C218E
:10DA4000217100780026012804D0002879D0122006
:10DA5000207190E006F072F9002819D006F0B7F9AD
:10DA600094F83600A8B1012813D0042811D008F08A
:10DA7000A1FD00287FD108F097FD18B108F094FDB2
:10DA8000022878D1002009F099F900B1FFDF267152
:10DA900071E008F089FD00286DD108F08BFD0028A9
:10DAA00069D106F0D6F8A0F57F41FF3963D107218F
:10DAB00001A801F0C7F8BE4905468860280000D1DA
:10DAC000FFDF032128460DF00BFE284606F081FB00
:10DAD00034F8540FA5F8440034F80409A5F84600BA
:10DAE000E278A17828460EF043FA01460022284643
:10DAF0000EF077FA6078009014F8043B288834F828
:10DB000054190A4601F07BF980B1042800D0FFDFE8
:10DB10002888072101F0D7F800B1FFDF0720207126
:10DB200005F58C712846FFF7FBFB24E0288805F0FB
:10DB300051FF284609F042F900B1FFDF2671EFE7F7
:10DB4000FFE708F031FD032803D008F033FD032878
:10DB500011D108F02CFD0546002009F052F850B90B
:10DB6000267145B1288805F036FF2888072101F085
:10DB7000AAF800B1FFDF1B20E0702770BDE8FC8130
:10DB80002DE9F041894C0646207828B1BDE8F041E6
:10DB90002D210F2000F02ABA3088072101F081F8EA
:10DBA00005004FF0010720D095F8F90040B995F82D
:10DBB0005C00112801D0122802D195F8360150B12D
:10DBC0000C2020710F20A0702D20E0703088E080A4
:10DBD000677127706CE51022B11C05F1FA0010F096
:10DBE00063F985F8F9700020EBE70220E9E770B5EA
:10DBF0006E4C0546207828B1BDE870402E210F20DC
:10DC000000F0F4B92888072101F04BF8022178B11F
:10DC100090F8F9202AB990F85C20112A04D0122A31
:10DC200002D00C20207104E080F8F9100020F9E700
:10DC300021710F20A0702E20E0702888E080012044
:10DC400060712070E4E52DE9FC47584C06462078C9
:10DC500028B138210F2000F0C9F9BDE8FC87708891
:10DC60004BF68032122190420AD848B14FF000089A
:10DC700030886946FEF7A7FB20B10220207110E032
:10DC800021710EE0019800F15009851C2F887288DF
:10DC9000394648460DF01AFD2888B842F6D184F876
:10DCA0000480012060713821E1702070D5E77CB5D7
:10DCB0003E4C0546207820B145210F2000F096F912
:10DCC0007CBD28886946FEF77EFB38B102202071B2
:10DCD000012060714521E17020707CBD01987F2298
:10DCE000014680F8582080F85920002280F85A20F8
:10DCF000A87801F8280FE878487028798870227190
:10DD0000E6E71CB5294C217821B113210F2000F042
:10DD10006DF91CBD00886946FEF755FB08B102206D
:10DD200005E0019890F82810012902D00C202071FC
:10DD300006E0582100222271095C21720088E080EF
:10DD4000012060711321E1700F21A17020701CBDB2
:10DD50002DE9F041154C0546207828B1BDE8F04189
:10DD600043210F2000F042B9A87808B1012803D15F
:10DD7000A888B0F5FA7F01D91220207128880721E0
:10DD800000F08FFF0126C8B1002780F8F070A98845
:10DD9000A0F8F21080F8CC60A978012900D0002109
:10DDA00080F8F01090F8CD0030B103E00C060020B0
:10DDB0004800002009F04EF9277101E0022020718F
:10DDC00066714320E070267072E42DE9F041CF4C7B
:10DDD0000546207828B1BDE8F04148210F2000F029
:10DDE00005B92888072100F05CFF012358B3828819
:10DDF0006D88C688418803EB4207BD4217D342F2C3
:10DE000010777E43BF107943B6FBF1F1491E89B20A
:10DE10004FF4FA76B14200D931468D4200D22946FC
:10DE2000491C521CB1FBF2F15143491E8AB290F8D1
:10DE3000221101B90284E280002020716371482020
:10DE4000E070237034E40220F7E770B5AF4C05466C
:10DE5000207828B1BDE8704041210F2000F0C6B8FD
:10DE600008F0A2FB08B10C2017E0297889B10A2933
:10DE70000FD014290DD01E290BD0282909D0322902
:10DE800007D04B2905D0642903D0FF2901D01220E7
:10DE900003E0284609F04FF800202071012060714E
:10DEA0004121E1702070B3E498490A781AB14D21FC
:10DEB0000F2000F09BB8427862B1827852B1C278EC
:10DEC00042B1027932B1C2881B2A03D303781BB155
:10DED000012B01D0122007E0A1F854200278D0F8DD
:10DEE000010042B1086500200871012048714D22EF
:10DEF000CA7008707047C864F5E770B5834C054672
:10DF0000207828B1BDE870404E210F2000F06EB897
:10DF1000287800F0010008F019F9287800F00100D5
:10DF200009F061F800202071012060714E21E1703C
:10DF300020706DE470B5754D0446287828B1BDE8B1
:10DF400070404B210F2000F051B800F05CF808B190
:10DF50000C200DE0601C0DF063FA207800F0010049
:10DF600005F031FF207800F0010006F0FFFE0020F0
:10DF70002871012068714B21E970287048E470B560
:10DF8000624C0546207828B1BDE8704049210F2039
:10DF900000F02CB808F008FB10B908F00BFB08B132
:10DFA0000C2003E0287805F0F0FF0020207101200C
:10DFB00060714921E17020702AE410B501784F2981
:10DFC00007D2534A52F8211019B1801C884701200A
:10DFD00010BD002010BD18B1022801D001207047EB
:10DFE00000207047C000703080B27047474A92F8F6
:10DFF0003130002B06D182F8320082F83310012034
:10E0000082F83100704710B508F011FA04280DD0DD
:10E0100008F00DFA052809D008F0C6FA032805D043
:10E0200008F0C8FA032801D0002010BD012010BD5F
:10E0300090F8691041B990F8C01029B190F8C0006B
:10E04000042801D001207047002070470178406803
:10E0500021B190F8690010B100207047E8E7012075
:10E0600070470178012909D1406890F8CD10002946
:10E0700004D0002180F8CD1008F0ECBF704710B537
:10E08000038843F6FD711A1F8A4223D24288141F67
:10E090008C421FD29A421DD8C28940F67B43911F01
:10E0A000994217D2018A8C1F9C4213D28A4211D8FE
:10E0B000428AB2F5FA7F0DD2828A40F67744A2F105
:10E0C0000A03A34206D2B2EBD10F03D9C18A028B55
:10E0D000914201D9302010BD017911B1012910D12F
:10E0E00007E0417929B1012903D0022901D0032990
:10E0F00007D1007B38B1012805D0022803D00328BE
:10E1000001D0122010BD002010BD00000C06002020
:10E110009CE301003F3070470844C01D424301F1B9
:10E120003F00104480B2704770B51D460446A818E1
:10E13000049BC01D00FB03F205F13F00104486B2B2
:10E14000B14238BFFFDF1E2120460FF024FFA6F1A9
:10E150001E0080B2A5756080B0F5004F88BFFFDF5C
:10E16000608805F13B01884238BFFFDF6088401BB3
:10E17000A0F13B011B2934BF1B203B38208070BD20
:10E18000408870472DE9F04F0D46C188044600F1E4
:10E190001E08008921F4004320F4004221F40046C7
:10E1A00020F400474FF0010A4FF000099A4208D1CD
:10E1B00000F4004001F4004188421CBF0020BDE88B
:10E1C000F08FB7420BD9A17DB81B401AC01F854202
:10E1D0001BDC08EB06000021058041801EE0608802
:10E1E000A17D801B401AB0F1070B0ED4BBF11B0FB1
:10E1F000B8BFFFDF5D45D4BF29461FFA8BF1681A0F
:10E200000204120C18BFBA4204DD84F814900020F6
:10E21000BDE8F08F08EB06000180428084F814A06E
:10E22000BDE8F08F2DE9F041044600F11E02C088E0
:10E2300020F40043207D002808BFBDE8F081D018FD
:10E240000288438813448B423CBF0020BDE8F08124
:10E25000002791429CBF0180478013D9891A0D0481
:10E260002D0C45800ED0E088A61D20F4004085428C
:10E2700088BFFFDF30884FF4004121EA00002843C7
:10E28000308009E0A27D0088D31D1044C01D81B2FA
:10E290006288A01D00F044FB27750120BDE8F081D5
:10E2A00030B4B0F804C0C488034600F11E052CF455
:10E2B00000402844A44503D10020188230BC704798
:10E2C000B3F80CC00488A44509D34088ACEB040C17
:10E2D000A0EB0C0084B20CEB0500C01E06E0A4EB22
:10E2E0000C049D7DA4B2AC446044001DB1F800C094
:10E2F000A44588BF0C80B3F80CC0BCF1000F0CBF64
:10E300004FF0010C4FF0000C82F800C00988198210
:10E3100030BC70472DE9F041044600F11E018088B1
:10E3200020F400404518208A002808BFBDE8F0818D
:10E33000A189084480B2A08129886A881144814259
:10E3400038BFFFDF28886D88A289411900279142D4
:10E3500019D175B1A088261D20F40040A84238BF0D
:10E36000FFDF30884FF4004121EA0000284330806D
:10E3700008E0A27D1044C01D81B2D31D6288201D1B
:10E3800000F0CEFAA78127820120BDE8F0812DE9B7
:10E39000F0474189B0F804800027044600F11E0AC6
:10E3A000414518BF4FF400493AD000BF21F4004066
:10E3B000504446886EB1608904F10A0520F400409B
:10E3C000B04238BFFFDF288829EA000030432880A8
:10E3D00021E0A37D008803F1070C18446389C01D68
:10E3E00023F400456288284480B204F10A01904277
:10E3F0000BD2121A92B20CF11B0C62452CBF03F423
:10E40000004229EA030004D204E0801A80B229EA1B
:10E41000030210430880781C618987B24145C5D149
:10E420003846BDE8F0872DE9F047B0F808800B4684
:10E43000044600F11E01B0F80A90808828F4004CD0
:10E4400001EB0C05804504BF0020BDE8F087002AE1
:10E450001CBF281D106023B1A27D291D18460FF096
:10E4600023FD2F886D888DB1E81987B2208904F1CA
:10E47000080620F40040A84238BFFFDF30884FF480
:10E48000004121EA00002843308009E0A07D628835
:10E49000C119C91DC31D89B204F1080000F040FA7A
:10E4A000C84504BF208960813846BDE8F08781886F
:10E4B000C08881420CBF01200020704781880089FC
:10E4C00088420CBF01200020704730B48488C28885
:10E4D00000F11E0324F4004C22F4004163449442F2
:10E4E0001BD08289048A15191C885A88A3189D425A
:10E4F00016D312B18A4210D212E0837D0CF1070CC0
:10E500001A196244408892B2801A80B2223398422B
:10E5100001D211B104E08A4202D130BC0020704720
:10E5200030BC012070472DE9F007B0F806C004891F
:10E5300000F11E0702462CF400457E1924F4004920
:10E540002CF4004A002024F400434FF00108D14588
:10E550000AD104F400440CF4004C644504D0508209
:10E56000BDE8F00700207047AB4207D992F816C00B
:10E570005B1BA3EB0C03DC1F002308E0B2F802C016
:10E58000947DACEB050CACEB040CACF10704002C57
:10E59000E5DBB2F80EC0BCF1000F0DD0B6F800C03C
:10E5A00075884DB15B1B50758B42D8DBD0893844E0
:10E5B000A0EB0C00C01E09E0A4EB0C0450758C42CB
:10E5C00008DB907DD38918443044001D5182BDE89A
:10E5D000F00770478B42A8BF82F81580E6DABEE7E5
:10E5E0002DE9F05F044600F11E0AC088934620F42E
:10E5F00000400AEB0005608A894608B1484502D20E
:10E600000020BDE8F09FE089002804BF4FF000081B
:10E61000464607D0B5F800806E8808EB06018842B0
:10E6200018BFFFDF607D4FF0000750EA060101D000
:10E6300048B332E0E08938B1A17D01444819B4F80B
:10E6400017108180617E8171E18908EB09004944DE
:10E65000E18128806F80BBF1000F0BD0A07D29885D
:10E66000C31D0144C91D89B26288A01D00F058F97C
:10E67000E78137E0A07DE189084428448188A4F837
:10E68000171080792DE0E089B4F817105044A0EB02
:10E69000080020F8031D617E817006EB090086B238
:10E6A000E089BBF1000F4844E081A5F800806E804E
:10E6B0000ED0E088A51D20F40040B04238BFFFDF37
:10E6C00028884FF4004121EA000030432880CFE73A
:10E6D000E0895044A0EB080030F8031DA4F817109F
:10E6E00080786076678227750120BDE8F09F01463B
:10E6F0001E308A88CB8822F4004C60449A4203D0B2
:10E700008989002908BF70470020704700F11E0367
:10E71000807D01F1040C604410600888002804BF6B
:10E72000D81E106008884988084480B270472DE9D7
:10E73000F04115460A4600F11E061C46807D131D59
:10E74000034410885788069900281CBFC01C80B25B
:10E7500026D088429CBF081A80B213D9401AA04222
:10E76000A8BF20461FFA80F85818424629460FF0E5
:10E770006FFB002818BFBDE8F0814544A4EB0800FA
:10E7800084B2002001198F423CBF4FF0FF30BDE83A
:10E79000F081304422462946BDE8F0410FF058BBD5
:10E7A000FA1C97B2F61ED4E72DE9F04100F11E07DE
:10E7B0001D46807D0B1D0344164608880024B1F8D1
:10E7C0000280069A00281CBFC01C80B21FD0904255
:10E7D0009CBF101A80B20DD9801AA842A8BF284643
:10E7E00084B29918224630460FF05EFB281B85B292
:10E7F000264400204119414506D839182A4630469A
:10E800000FF052FB601984B22046BDE8F08108F198
:10E8100003011FFA81F8FF1ED9E72DE9F0411646E2
:10E820000A4600F11E071D46807D131D0344108813
:10E830000024B2F80280069900281CBFC01C80B2D8
:10E840001FD088429CBF081A80B20DD9401AA84236
:10E85000A8BF284684B25818224631460FF024FB40
:10E86000281B85B2264400204119414506D838446A
:10E870002A4631460FF018FB601984B22046BDE8E5
:10E88000F08108F103021FFA82F8FF1ED9E770B584
:10E89000044600F11E01C288808820F40043194418
:10E8A000904205D0A289002A04BF228A002A01D002
:10E8B000002070BDB1F800C04D8885B1261D20F440
:10E8C0000040A84238BFFFDF30884FF4004121EA02
:10E8D00000002843308000202082012070BDA07DF0
:10E8E0000CF10701C31D084481B26288201D00F0AD
:10E8F00017F8F0E70021C181417541820175704729
:10E9000003881380C289002A04BF00207047C28890
:10E9100000F11E0322F400421A440A60C0897047C5
:10E9200010B4B0F800C02CF40044214489B24FF474
:10E93000004491420AD2521A92B21B339A422CBF1F
:10E940000CF4004224EA0C0104D204E0891A89B2D2
:10E9500024EA0C021143018010BC70472DE9F041FC
:10E9600088464FF6FC7102F103021E46040002EADB
:10E97000010509D00027E01C20F00300A04200D0D0
:10E98000FFDF201D01210CE00127F4E702462844A7
:10E990002FB9B14201D2034600E000231360491CA5
:10E9A000C9B2B142F2D9011BC8F80010002F04D13E
:10E9B0000EB1201D00E000202060BDE8F08102467D
:10E9C00000201168002902D00846096811607047CC
:10E9D00002680A60016070474FF6FC73C91C194059
:10E9E000101A001F90FBF1F0C0B270474FF6FC7395
:10E9F000C91C1940001D01FB02007047F8B5D24D3B
:10EA000004460E46A878A04200D8FFDF05EB860733
:10EA1000B86A50F8240000B1FFDFB868FFF7CFFFF5
:10EA200005000DD0B86A062E40F824500AD0082EF2
:10EA300000D3FFDFC548294650F8262020469047DE
:10EA40002846F8BDC048C24B7A30A0F12E02009093
:10EA50002946204609F0A0FCF2E72DE9F84F804650
:10EA6000DDF828901E4603EB090093468A46C4B29F
:10EA70005FEA080707D00025FF2800D9FFDFBAF1B9
:10EA8000000F03D101E00125F6E7FFDF08F10300E5
:10EA900020F00301414500D0FFDFCB4500D9FFDF67
:10EAA00065B9A94A00204C324FF6FF7110705180B1
:10EAB000A74A1070A44A7A3210705180A24880F898
:10EAC00000B046708470C4700471447180F8069080
:10EAD000DFF878B2C67100260BF1400B8146FF1CAF
:10EAE00027F003000746002D02D109EB860188605C
:10EAF0003BF8162019F8063001D04FF000006946A7
:10EB0000FFF72CFF0098761CF6B20744082EE6D3D8
:10EB1000FF1C27F003002346064675B100200222A1
:10EB20006946FFF71BFF00983118002003464E4648
:10EB3000C91C21F003021DB110E0C9F84800EEE73E
:10EB400006EB80070021BA6206E000BFD7F828C0B4
:10EB50004CF82130491CC9B2A142F7D3401CC0B2C5
:10EB600002EB84010828E3D3A1EB0800AAF8000017
:10EB70000020BDE8F88F10B5044603F005FF08B18A
:10EB8000102010BD2078704A618802EB80009278D6
:10EB90000EE0836A53F8213043B14A1C6280A180A1
:10EBA000806A50F82100A060002010BD491C89B285
:10EBB0008A42EED86180052010BD70B505460C462E
:10EBC000084603F0E1FE08B1102070BD082D01D306
:10EBD000072070BD25700020608070BD0EB56946AD
:10EBE000FFF7EBFF00B1FFDF6846FFF7C4FF08B196
:10EBF00000200EBD01200EBD10B50446082800D32C
:10EC0000FFDF5148005D10BD3EB505460024694652
:10EC1000FFF7D3FF18B1FFDF01E0641CE4B26846E0
:10EC2000FFF7A9FF0028F8D02846FFF7E5FF001BF3
:10EC3000C0B23EBD44498978814201D9C0B2704713
:10EC4000FF2070472DE9F0410C460546062901D00A
:10EC5000072C10D13C4FB86CFFF7B1FE02004FF605
:10EC6000FF7604D00221B86CFFF7B6FE00E0304614
:10EC70002880B04202D10020BDE8F0812146FFF794
:10EC8000BDFE040002D1288800F050F82046F3E7CA
:10EC9000A0F57F42FF3A01D0082901D30020704738
:10ECA000ACE6A0F57F42FF3A0BD0082909D2264AEC
:10ECB0009378834205D902EB8101896A51F82000DB
:10ECC0007047002070472DE9F04104460D46A4F539
:10ECD0007F4143F20200FF39CED0082D01D3072037
:10ECE000CAE719494FF000088A78A242C4D901EB5B
:10ECF00085072146BA6A52F82460002EBCD0134A18
:10ED000008462032314652F825209047B96A062D30
:10ED100041F8248001D0072D02D1204600F006F8EA
:10ED20003146B868FFF754FE0020A5E710B5064C41
:10ED3000C2B20221A06CFFF759FE0146A06CBDE8EB
:10ED40001040FFF745BE000068060020D8E401002F
:10ED50005400002001469F48002200680260037AA8
:10ED600000EB830040F80C2F8180114600F022B99F
:10ED70002DE9F05F9846DDF830B0DDF828A01546A3
:10ED8000894604004FF0000623D00027E01C20F045
:10ED90000300A04200D0FFDF65B30120FFF7BAF9FE
:10EDA00000FB05620AEBCB0016180120FFF7B2F951
:10EDB00000FB05620B9805EB450108EBC000104411
:10EDC00000EB4100143000EB850000EB850617B125
:10EDD00010E00127DAE77F48A6EB8507A900046069
:10EDE000257204F10C000C3F60600FF0F6F8B8B229
:10EDF000FFF7B0FF0020C9F80060BDE8F09F2DE9E3
:10EE0000FF4F744C814681B020689A468B4600B90A
:10EE1000FFDF2068027A4A4503D9426852F8291078
:10EE200021B143F2020005B0BDE8F08F006800B9DF
:10EE3000FFDF01210E9A0398FFF76EF9C61C4FF60B
:10EE4000FC752E40584601215246FFF765F9C01C5B
:10EE500000EA050808EB0600001D85B25D480027A2
:10EE60000068046801E027460446206838B1A1889C
:10EE7000A942F8D13946204600F0A4F813E005F184
:10EE80000800A18880B2814229D33946204600F08B
:10EE900099F8A0880022411B6019026081803946E0
:10EEA00000F088F8A580A08860802680251D0E9F30
:10EEB0000123039A314628460097FFF735F9208849
:10EEC000414628445A460123CDF800A0FFF72CF90B
:10EED000404800684168002041F82940A3E7042029
:10EEE000A1E770B53B4C0546206800B9FFDF2068FC
:10EEF000017AA94210D9426852F8250060B14188D0
:10EF0000002342F8253003608180194600F052F852
:10EF1000216800200A7A08E043F2020070BD4B68C5
:10EF200053F820306BB9401CC0B28242F7D80020A1
:10EF300002E08A88104480B209680029F9D1FFF7FD
:10EF400009FF002070BD70B5224D286800280AD046
:10EF5000002404E02046FFF7C4FF641CE4B22868E4
:10EF6000007AA042F6D870BD70B51A4E054600244E
:10EF7000306800B9FFDF3068017AA94204D94068DF
:10EF800050F8250000B1041D204670BD70B5114E2B
:10EF900005460024306800B9FFDF3068017AA942D5
:10EFA00006D9406850F8251011B131F8040B441807
:10EFB000204670BD19B10A680260086070470549B3
:10EFC0000968F8E7006809B10860704701490968F5
:10EFD000FAE700005C00002070B5044600780E4699
:10EFE00001281AD0072802D00C281AD115E0A068F1
:10EFF000216905780B2D0CD0052003F05EFC052D52
:10F000000FD0782300220520D4F8101003F0B8FBAD
:10F0100007E0782300220620F8E70520216903F0A5
:10F020004CFC31462046BDE8704001F0A7B910B550
:10F0300000F13902C3799478411D64F00304234040
:10F04000C371DB070DD04B79547923404B710B7999
:10F05000127913400B718278C9788A4200D9817085
:10F0600010BD00224A710A71F5E74178012900D0EC
:10F070000C21017070472DE9F74F86B000208C6994
:10F080000D468DF8040009780127FA4816464FF01E
:10F09000070A4FF011094FF00A0B2A2978D2DFE84E
:10F0A00011F02A00110352036903A803B303CC0330
:10F0B000FA030F043B04620481049A04D504E604B5
:10F0C000050510053005540577059C05C605E005C6
:10F0D000EE050F062706300663068506D6060D07E1
:10F0E0001B074B076A0779078A07C407FB0727082E
:10F0F000E407E807ED0714B120781D2829D0D5F8DA
:10F1000008805FEA080043D001208DF80400686A97
:10F11000059003208DF808008DF809B0286A039047
:10F12000A8880028EFD098F8001091B10F2910D2CC
:10F130007ED2DFE801F07D144CDCFDFCFBFAF9F82F
:10F14000F7089FF6F500022822D124B120780C2878
:10F1500001D0002770E302208DF80400ACE1062006
:10F16000696A03F0AAFBA8880728EDD1204601F0C0
:10F1700000F9022809D0204601F0FBF8032808D93D
:10F18000204601F0F6F8072803D20120207005E0A0
:10F1900011E2002CB7D020780128D5D198F80400CE
:10F1A000C11F0A2903D300BF85F81CB089E2A070F3
:10F1B000D8F80010A163B8F80410A18798F80600E9
:10F1C00084F83E00012028700320207046E00728C4
:10F1D000BAD1002C97D020780D28B5D198F803101B
:10F1E00094F83B20C1F3C000C2F3C002104201D02A
:10F1F0000E2000E00F20890707D198F80510014282
:10F20000D2D198F806100142CED194F83D2098F85A
:10F21000051020EA02021142C6D194F83E2098F867
:10F22000061090430142BFD198F80400C11F00E0CE
:10F2300045E20A29B8D2617F814201D90620C2E3A2
:10F24000D8F800106160B8F80410218198F8060021
:10F25000A072012028700E20207003208DF8040079
:10F26000686A059004F139000290601D0390173020
:10F27000049067E2412890D1204601F07AF80428F2
:10F2800002D1E078C00704D1204601F072F80F28BF
:10F290009ED1A88CEF6880B24FF0400AD4F8248049
:10F2A000FFF762FE39460827424653460097FFF7AC
:10F2B0007BFA0E208DF80400686A0590606A02905F
:10F2C000002101A8FFF788FE2078042806D0A07F3F
:10F2D00038B1012805D0032806D0AEE30520207000
:10F2E0000BE284F8009034E71220207066E01128C9
:10F2F000C1D1204601F03DF8042802D1E078C007D2
:10F3000019D0204601F035F8062805D1E078C0076D
:10F3100011D1A07F02280ED0204601F02AF808E083
:10F32000AFE07DE09AE16EE14EE106E1E5E0CBE0A1
:10F330001CE011289FD1102208F1010104F14800BE
:10F340000EF0B2FD607801280DD012202070E07818
:10F35000C00703D0A07F88B301282FD085F800B064
:10F360008DF804B0F0E384F800A027E011288FD1D5
:10F37000204600F0FEFF082804D0204600F0F9FFE8
:10F38000132885D12869D8B16869C8B104F178001B
:10F39000102208F1010107460EF086FD20780828AA
:10F3A00012D014202070E078C0070FD0A07F022870
:10F3B00018D06178022912D00328CFD10420FDE3B0
:10F3C00000208DF80400F6E00920EBE70B20287000
:10F3D000296901204870206CC1E9010792E208B157
:10F3E000012870D10B202870296981F801A0606A7A
:10F3F0004860206AC1E9020778E2206CE278006880
:10F40000C2F34402521ED04000F0010040F08000E0
:10F4100000E000200874E06A48617CE20746F9E3F6
:10F420001128D0D1204600F0A4FF0A2802D1E078AC
:10F43000C00704D1204600F09CFF1528C3D110223C
:10F4400008F1010104F148000EF02EFD20780A2891
:10F4500012D01620207012202870296909204870C7
:10F4600004F158004860203088601038C860206C73
:10F470000861ACE314E601000B202070E4E2287080
:10F48000D9E102289FD1204600F073FF042804D35D
:10F49000204600F06EFF082809D3204600F069FFDF
:10F4A0000E2890D3204600F064FF12288BD2A07F54
:10F4B000022888D18DF80490686A059098F80100B8
:10F4C0008DF80800FBE36CE20228AAD1204600F088
:10F4D00050FF00286FD0204600F04BFF0128F9D0E4
:10F4E000204600F046FF0C28F4D005208DF80800D7
:10F4F00098F801008DF8090065E71128FCD1002C6F
:10F50000FAD020781728F7D16178E06A022912D062
:10F510005FF0000101EB4101182606EBC10110224A
:10F52000405808F101010EF0BFFC0520696A00F0A7
:10F5300013FF26700DE60121ECE70B28DCD1002C2F
:10F54000DAD020781828D7D16178E06A02292CD047
:10F550005FF0000101EB4101102202EBC1014158B3
:10F56000B8F8010008806078E16A022820D0002005
:10F5700000EB4002142000EBC2000958404650F84E
:10F58000032F0A60406848600520696A00F0E4FEC5
:10F590006078022810D04FF000002044407A20F01C
:10F5A00001000CD14FF001010BE04FF00101D1E758
:10F5B0004FF00100DCE77FE24FF00100EDE74FF094
:10F5C00000012144487279E3112895D1002C93D091
:10F5D0002078192890D16078E16A022811D00020A3
:10F5E00000EB40021C2000EBC2001022085808F17A
:10F5F00001010EF059FC0520696A00F0ADFE1A20E9
:10F60000F5E00120ECE7082898D1002C98D020786C
:10F610001A2893D1E06A98F80120017862F3470133
:10F620000170E16AD8F8022041F8012FB8F806000D
:10F6300088800520696A00F08FFE6078022807D074
:10F640004FF000002044407A20F002012BD033E03C
:10F650004FF00100F6E7204441722FE31128B4D1A6
:10F66000002CB4D020781B28AFD16178E06A022941
:10F670001CD0002101EB4101202202EBC10110222C
:10F68000405808F101010EF00FFC0520696A00F0F6
:10F6900063FE607802280CD04FF000002044407ACE
:10F6A00020F0040108D14FF00100D4E74FF0010130
:10F6B000E0E74FF00100F1E74FF00000CBE785F8FD
:10F6C0001CA0FAE33078012884D11C2204F11C002C
:10F6D00071680EF02EFCE079C10894F83B0001EA55
:10F6E000D001E07861F30000E070217FF1BB217868
:10F6F00003290AD0C0073FF4F9AD032028708DF824
:10F7000004B0686A059041209EE3607FA17888423A
:10F710003FF694AD02272771E179204621F0E00100
:10F72000E171617A21F0F0016172A17A21F0F001BA
:10F73000A172FFF77CFC2F708DF804B0686A059009
:10F740008DF808A0F2E33078112888D18DF804A054
:10F75000696A0591B1680391ADF808A0084661682F
:10F76000016021898180A17A817100E06AE0042032
:10F770002070A4E230781128A6D18DF804A0686A20
:10F780000590301D02AB07C883E807004120ADF8A3
:10F79000080008460C210170A88CD6F80C8080B2B5
:10F7A0004027D4F82090FFF7F1FB41464FF00808BE
:10F7B0004A463B46CDF80080FFF72FF8002101A80C
:10F7C000FFF70AFCE07820F03E00801CE070207813
:10F7D000052801D00F200AE0A07F00283FF4C3AD28
:10F7E0000128FBD003287DD184F80080B1E420708B
:10F7F000AFE430780328A8D170680168A16640683A
:10F80000E0660520287035E2317803299DD17168C2
:10F810000A68226749686167216C51B9A17F19B1F3
:10F82000012901D0062029E185F800A02064606448
:10F8300001E085F800A00327F3E33178022984D1A1
:10F84000317909B1297737E1A17F022910D0032945
:10F85000EFD16178012910D0A17994F83A200129DB
:10F860000FD02064E178C90713D0012A0ED010E030
:10F87000B0680028E7D020640BE0A27994F83A1031
:10F88000EDE7B1680029DED02164EBE7F0680028DD
:10F89000D9D06064CDE78DF804B0696A0591E1784C
:10F8A0005846C90709D06178022903D1A17F29B13F
:10F8B000012903D0A17F032900D00820287012E27B
:10F8C00030781128BFD1B068286209202870E0780C
:10F8D0002969C0070FD081F801A0206A4860606ADA
:10F8E000886000E0ABE004F16800C860A07F0228F7
:10F8F0007FF48FAD81E501204870206C486004F1F1
:10F900006800886004F13800C860201D0861206B21
:10F910004861606B88611FE2E1783078C90701D0E7
:10F92000062100E00A2188428DD12078072817D0CF
:10F9300084F800908DF804A0686A0590286A039006
:10F94000ADF80890032100F8011B102271680EF039
:10F95000ABFA002101A8FFF73FFB00202862C2E4B8
:10F9600008202070E6E730781128ABD18DF804A08C
:10F97000686A0590B0680390ADF80890042100F81B
:10F98000011B102204F168010EF08EFA002101A87B
:10F99000FFF722FB2078092801D0132027E784F8FD
:10F9A00000B016E0E1783078C90701D0062100E008
:10F9B0000A21884286D1102204F1480071680EF0B5
:10F9C00047FA10B104202877A2E3207809283FF4F1
:10F9D000C5AC0C2053E5E078C10735D0A17F0129E3
:10F9E00002D002291BD02CE00D202870296981F853
:10F9F00001B06078012809D0206A4860606A886098
:10FA000004F16800C8601030086104E5606A48606D
:10FA1000206A886004F17800C8601038F4E7C0F309
:10FA2000440114290DD24FF0006101EBB0104FEAF0
:10FA3000B060E0706078012801D0102055E4062005
:10FA4000D5E6607801288AD00E2018E5307809289C
:10FA50008BD185F800B010208DF80400686A0590FD
:10FA600070680290002101A8FFF7B6FAE9E7E07894
:10FA7000C00706D0A07F01281FD10F2028700420C6
:10FA8000F8E015202870296902204870206C486031
:10FA90006078012805D004F1780088601038C860CB
:10FAA0005AE104F1680088601030F8E730780228E5
:10FAB000CED1307908B1287728E3102028700F20A4
:10FAC000D8E030781328F7D185F80090296908200C
:10FAD000487070684860607801280DD004F16800B3
:10FAE00088601030C860206B0861606B486104F169
:10FAF00058008861A06A21E004F17800886010381D
:10FB0000F0E730780728D7D1607801281AD1A0789B
:10FB1000A16A0A18C0F1100110460EF03CFA12203A
:10FB2000287029690920487004F158004860203085
:10FB300088601038C860206C086141E0C861E06AE4
:10FB4000086209E11320C9E0CBE030780828B3D17E
:10FB5000102204F1480071680EF07AF908B10B2008
:10FB600031E720780B28EDD02046FFF760FAA07827
:10FB7000A16A0A18C0F1100110460EF00CFA162006
:10FB8000287008208DF80400686A0590002049E07C
:10FB90003078112890D1B068286214202870296923
:10FBA0000920487004F15800486010308860103017
:10FBB000C860606C08616078012800E09EE006D0B3
:10FBC00004F139004861206B8861606BB6E7601D05
:10FBD0004861606B8861206BB0E73078082892D16B
:10FBE0008DF804A0686A0590286A0390ADF8089023
:10FBF0000D2100F8011B102271680EF055F900214B
:10FC000001A8FFF7E9F9002028626178012902D0F4
:10FC10001520ECE569E21621297008218DF8041001
:10FC2000696A05910290A0788DF80C007EE1307829
:10FC30000B288CD1162028706078022802D120462B
:10FC4000FFF7F5F9A07871680A18C0F110011046A5
:10FC50000EF0A1F908208DF80400686A059070681C
:10FC6000E0E730780F2895D1E079C0077BD01720E6
:10FC7000287009208DF80400686A059056E13078F4
:10FC8000102887D11422311D04F11C000EF051F907
:10FC9000E16A208DA1F80900E16AA078C871E179D4
:10FCA000E26A01F003011172E16A627A0A73E16AA1
:10FCB000A07A81F824006078012876D0B3E13EE292
:10FCC0006078022801D0012000E000202044407A22
:10FCD000C0070BD0E078C00708D1192028708DF834
:10FCE00004B0686A05908DF808901FE11E2071E647
:10FCF0003078112874D1B06828621A202870052045
:10FD0000B8E7307803286BD16078E26A022801D026
:10FD1000012000E0002000EB4001142000EBC101B5
:10FD20005158726813680B6052684A601B21297031
:10FD3000D5E9041205234B70636A4B606778E36A68
:10FD4000022F01D0012700E0002707EB470700EB57
:10FD5000C7001858C1E90202686A4862069800F0B4
:10FD600024FBFFF75BBB87E130780E2838D1607841
:10FD7000E26A022801D0012000E0002000EB4000F0
:10FD8000102101EBC00002231058093271680CF0F9
:10FD90006DFC1C202870296904204870206A486086
:10FDA000E06A09308860F84879E65AE130780D2831
:10FDB00016D16178E06A022901D0012100E000211A
:10FDC00001EB4101182707EBC101A2784058716887
:10FDD0000EF06AF86178E06A022902D0012101E0A0
:10FDE000A9E0002101EB410107EBC1014058A178D6
:10FDF0000844C1F110010EF0CEF88DF804A0686A35
:10FE00000590286A0390ADF8089006210170627889
:10FE1000E16A022A01D0012200E0002202EB420244
:10FE200007EBC202401C895810220EF03DF8002159
:10FE300001A8FFF7D1F8002028621D2028708DF856
:10FE400004B0686A05900B208DF808006EE03078E9
:10FE5000112870D18DF804A0686A0590B0680390ED
:10FE60000B20ADF80800039880F800A06278E16AE2
:10FE7000022A01D0012200E0002202EB42021023FC
:10FE800003EBC20289580988A0F801106178E26A80
:10FE9000022901D0012100E0002101EB41031421DE
:10FEA00001EBC30151580A6840F8032F49684160CB
:10FEB000002101A8FFF790F818E729E160780228EF
:10FEC00001D0012000E000202044407A800701D5C5
:10FED0001F2003E721207DE5307811282BD18DF8F4
:10FEE00004A0686A0590B0680390ADF808900827F0
:10FEF00007706178E26A022901D0012100E0002147
:10FF000001EB41031C2101EBC301401C515810229D
:10FF10000DF0CAFF002101A8FFF75EF8202028702D
:10FF20008DF804B0686A05908DF80870314601A814
:10FF3000FFF752F815E775E03078112872D18DF887
:10FF400004A0686A0590B06803900820ADF8080026
:10FF5000039809210170E169097849084170E16954
:10FF600051F8012FC0F802208988C180002101A822
:10FF7000FFF732F8AEE76078022801D0012100E0F7
:10FF800000212144497A490701D52220A6E601280B
:10FF900049D068E03078112844D1B0682862232025
:10FFA0002870296904204870206A4860E06A093096
:10FFB0008860764873E530780D2833D16178E06A3F
:10FFC000022901D0012100E0002101EB410120279D
:10FFD00007EBC1011022405871680DF065FF8DF8E4
:10FFE00004A0686A0590286A0390ADF8089080F82C
:10FFF00000B06278E16A022A01D0012200E000220A
:020000040001F9
:1000000002EB420207EBC202401C895810220DF09D
:100010004BFF002101A8FEF7DFFF00202862607877
:10002000B5E791E037E02420D4E4607802280BD0D3
:1000300000202044407AC10702D0E178C90705D0EA
:10004000810705D51920A9E40120F2E71720A5E4CE
:10005000400701D51B20A1E41C20207060780128F6
:1000600001D01820B6E42720B4E4282028700B2003
:1000700000E63078122849D12920ABE42078012805
:1000800044D00C2842D02046FEF7EFFF0C208DF81C
:100090000400686A059039E030784FF0260811288E
:1000A00005D012203070032785F800804CE08DF8D1
:1000B00004A0686A0590B06803900220ADF80800BB
:1000C000039805210170297F4170002101A8FEF7E6
:1000D00083FF0B208DF80400686A0590314601A863
:1000E000FEF77AFF074685F80080012F0ED02BE03F
:1000F00001208DF80400686A059004208DF808003E
:10010000287F8DF809000020287712E0287F80B131
:100110001D202070252028708DF804B0686A059095
:1001200002208DF80800314601A8FEF755FF07466A
:100130000AE00CB1FE2020709DF8040020B10021DF
:1001400001A8FEF749FF0AE409B03846BDE8F08F80
:100150002DE9F04F0C4601274E69097885B090468D
:10016000BA464FF00209072021B101294ED00229D9
:100170001FD1C8E0217901290AD0022915D003290D
:1001800010D0042915D11BE00CE6010028E5010080
:10019000707801280CD10620616A02F067FB002804
:1001A00007D11AE01D20307017E07178022901D0C4
:1001B000052796E031780C2927D18DF804000EE050
:1001C0003078011F042902D30E3803281DD2B07FD6
:1001D00002281AD12089022817D38DF8049084F8B8
:1001E00000A020899DF80410884203D20A208DF8CF
:1001F00000003FE01121083488F8001094E80E0058
:10020000C8E901120327C8F80C306AE098F800101A
:10021000112966D18DF80000616A0491D8F8085060
:10022000029521794FF00B0B012906D0022929D024
:10023000032911D0042954D15AE0ADF8049085F86F
:1002400000B0207E4F4600F01F0068700021684615
:10025000FEF7C2FE377043E0ADF804900520287029
:10026000207E68704E4600216846FEF7B5FE267077
:100270008DF800B0606A049041466846FEF7ACFE17
:1002800007462EE0ADF8040085F800A0207F6870D6
:10029000607F00F00100A870A07F00F01F00E870F0
:1002A000E17F2971C0071FD094F8200000F00F00F3
:1002B000687194F8210000F00F00A87100216846D1
:1002C000FEF78AFE2868B063A888B087A87986F808
:1002D0003E00A069407870772879B0700D203070AA
:1002E0000027384605B031E70020A8716871E5E7BE
:1002F000ADF804900E202870207E687000216846BA
:10030000FEF76AFEECE7FE2030708DF800A0606A10
:10031000049004208DF80400207E8DF80500EDE7A0
:1003200000B50023012285B005280FD006280BD187
:1003300002208DF8002004918DF804008DF805301E
:1003400000216846FEF748FE05B000BD8DF800208C
:1003500004918DF80420F1E770B50C46054602F0D3
:10036000ACFA21462846BDE870407823002202F00E
:1003700007BA08B1007870470C20704770B50C00C0
:1003800005784FF000010CD021702146F3F727FAD1
:1003900074482178405D884201D1032070BD02205D
:1003A00070BDF3F71CFA002070BD027B032A05D054
:1003B00000220A704B780B2B02D003E00420704718
:1003C0000A770A62027B9300521C0273C150032019
:1003D0007047F0B585B00F4605460124287B05EB34
:1003E000800050F8046C7078411E0C290AD25D49D7
:1003F0003A46123101EB8000314650F8043C284661
:10040000984704460CB1012C11D1287B401E10F0F6
:10041000FF00287301D00324E0E70D208DF80000D1
:10042000706A0490002101966846FFF7A7FF032C2D
:10043000D4D005B02046F0BD70B515460A46044636
:1004400029461046FFF7C5FF064674B12078FE28FE
:100450000BD1207E30B100202870294604F10C0019
:10046000FFF7B7FF2046FEF700FE304670BD70472D
:1004700070B50E46044688210DF0AFFD0225012E11
:1004800003D0022E04D0052070BD0120607000E072
:1004900065702046FEF7E9FDA577002070BD28B104
:1004A000027E1AB10A4600F10C01C5E7012070472F
:1004B00030B5044687B00D46062002F0FEF9294605
:1004C000052002F0FAF92078FE2806D000208DF8E9
:1004D000000069462046FFF7E2FF07B030BD7FB558
:1004E0000E4600218DF80C1041780B2903D00C2901
:1004F00003D0002405E0846900E044690CB1217E4A
:1005000091B16D4601462846FFF74FFF032809D1F8
:10051000324629462046FFF78FFF9DF80C10002930
:1005200000D0042004B070BD04F10C05EAE710B55A
:1005300090B00C4607900B480421801E08900A4892
:100540008DF8191009900F92694606A8FFF7C7FFAA
:10055000002805D11022204601990DF0A5FC0020AD
:1005600010B010BD2EE501000CE6010070B50D467F
:10057000040011D085B1210128460DF00CFD102298
:100580004E4928460DF090FC4C4801210838018066
:1005900044804560002070BD012070BD70B5474E9D
:1005A00000240546083E10E07068AA7B00EB0410AA
:1005B000817B914208D1C17BEA7B914204D10C221C
:1005C00029460DF045FC30B1641C30888442EBDBD9
:1005D0004FF0FF3070BD204670BD70B50D4606006F
:1005E00006D02DB1FFF7DAFF002803DB401C14E032
:1005F000102070BD314C083C20886288411C91421B
:1006000001D9042070BD6168102201EB0010314651
:100610000DF04AFC2088401C20802870002070BD0E
:1006200070B514460D0018D0BCB10021A17002288D
:1006300002D0102811D105E0288870B10121A170E5
:10064000108008E02846FFF7A9FF002805DB401CC2
:10065000A070A8892080002070BD012070BD70B5F9
:10066000054614460E000BD000203070A8780128F3
:1006700008D005D91149A1F108010A8890420AD988
:10068000012070BD24B1287820702888000A50709D
:10069000022008700FE064B14968102201EB0011DC
:1006A000204610390DF000FC287820732888000AB5
:1006B000607310203070002070BD000068000020C2
:1006C0002DE9F041FE4C207EE17D884208BFBDE867
:1006D000F0810126FB4D0027E07D215C01EB8102CA
:1006E00005EB8200037C052B18D0037C062B23D05E
:1006F000037C072B34D0437C002B08BFFFDF29D0BD
:100700004774E07D16280EBF0020E07D401CE07598
:10071000481CC0B255F8222007211AE00674E07D7B
:1007200016281ABFE07D401C0020E075481CC0B2AE
:1007300055F8222002210CE00674E07D16281ABF2D
:10074000E07D401C0020E075481C55F82220C0B216
:1007500003219047207EE17D8842BDD1BDE8F08134
:100760000674E07D16281ABFE07D401C0020E0756D
:10077000481CC0B255F822200821EAE770B5D24DD6
:100780000C2085F82900A5F53B70002480F8CD41A8
:1007900080F8CC4100F5F4700476C47505F12C00A6
:1007A0000CF0C0FDA5F58E70047585F82B40601E19
:1007B0002C60A86085F8254085F8224085F8234004
:1007C00085F8244085F82140C048A5F1E80104706F
:1007D0004470002000EB800201EB82021474401C84
:1007E000C0B20B28F6D30120F8F708FF0020F8F775
:1007F00005FF012085F82600F9F72EFBB448F9F72C
:100800003AFBB44C2070B448F9F735FB6070BDE892
:100810007040F8F787BE10B5F8F7B2FEAD4C2078FF
:10082000F9F742FB6078F9F73FFBA74C94F82800F2
:10083000002808BF10BDF9F7B2F8002084F828009E
:1008400010BD0B20704770B59F4C94F8260000280F
:100850001CBFFFDF70BD94F82B00002808BFFFDF2E
:10086000F8F777FF62690025811A6FF07F43B1F5D1
:10087000800F24BFA2EB000CBCF5800F0DD38B4280
:1008800003D2991A0844411C07E0634528BFFFDFE3
:1008900005D2181A1044401C4142002900DBFFDF3A
:1008A000012684F8266084F82B5094F8291004203F
:1008B000844A01EB810102EB81010874A068B0F168
:1008C000FF3F04D0B01EA0600120F8F797FE002083
:1008D000F8F794FEF8F778FE25600CF0C7FEF8F7FD
:1008E000C1FF7E48056005604FF0E0214FF40040F5
:1008F000C1F88002F2F7E5FA74480078022804D0C3
:10090000032805D194F8230010B184F8226001E097
:1009100084F82250BDE87040F8F788BF0346694963
:100920000B2000BF00EB800201EB820212F8042CC6
:1009300022B1401E10F0FF00F4D1704700EB80029E
:1009400001EB8201012241F8143C01F8042C7047AC
:10095000012804D0032808BF002926D000E021B3D5
:10096000594B4FF0000C83F821C0584A0028907072
:1009700014BF022882F803C00BD0072915D2DFE884
:1009800001F01404060C0E1012001B2000E03A20A7
:10099000D070012083F8210070475820F8E77720B5
:1009A000F6E79620F4E7B520F2E7002070474748C5
:1009B00010B54078F8F75FFF80B210BD30B5421E29
:1009C0004049002500EB800001EB80040A2A02D890
:1009D00014F8040C00B9FFDF14F8040C012818BF48
:1009E000FFDF04F8045C30BD70B53D4C94F8CD01D8
:1009F00094F8CC1188420CBF01250025F8F7A9FE18
:100A0000F8F739FF94F8CD1194F8CC2191420CBF3E
:100A100001210021A942E9D170BD30B50D46314A0E
:100A200044190021101A71EB010038BFFFDF2E4876
:100A30008542C8BFFFDF2D488542B8BFFFDF2C4885
:100A40008442A8BF2B4804DA002CAABF20462848BD
:100A500030BD201830BD70B51A4900EB800001EBA5
:100A60008004254A54F8101D607A002852F820208E
:100A700011440CBF04200220084420F07F40F8F706
:100A8000FAFE94F90850174A44190021101A71EB24
:100A9000010038BFFFDF14488542C8BFFFDF13489D
:100AA0008542B8BFFFDF12488442A8BF114804DA6C
:100AB000002CAABF20460E4870BD201870BD000053
:100AC000DC080020F8080020E00900207A0000205F
:100AD0002D26010078000020C106010000F500402D
:100AE000F4060020FF7F841E0020A10700E05EF8CE
:100AF0000080841E00807BE170E501002DE9F04F4D
:100B00000646FF4885B00068C005C00D11D01038FA
:100B100040B20028B8BF00F00F0000F1E020B4BFE1
:100B200090F8140D90F80004400908BF4FF0010A36
:100B300001D04FF0000A307800281FBF01280020A4
:100B400005B0BDE8F08F307900280CBF04210221E8
:100B5000EC4ABAF1000F52F8200001EB000903D172
:100B6000E949002081F827006C4602AA2146B068B6
:100B7000F8F78EFE9DF90820F068211D104401222F
:100B8000C01C1F28B8BF019208DB03AAF8F780FE3B
:100B90009DF80C0010B10198401C0190DDE9001097
:100BA0000844401D20F07F400190A1EB090020F097
:100BB0007F40009070798DF80A0000980390F8F754
:100BC000C8FD009A019B121A181AD04922F07F42E0
:100BD00020F07F40B2F5800F26D2814224D3CA484C
:100BE00090F82950009CCA4F181B20F07F486FF0E6
:100BF0007F40001BAB4604900C2D24D005EB8500F4
:100C000007EB80026FF07F435068011BB1F5800F46
:100C100012D3A4EB000CBCF5800F0DD38B4205D290
:100C200004990844411C07E000205FE0634509D2B5
:100C3000191A0819401C41420029BCBFAB46957CDB
:100C4000DADB00E0FFDF5D4525D00BEB8B0007EB27
:100C500080026FF07F4091680B1BB3F5800F12D3B9
:100C6000A4EB010CBCF5800F0DD3984203D204987D
:100C70000844431C07E0604528BFFFDF0BD2431A3E
:100C80001819401C4342002B05DD9DF80A00927B99
:100C9000904228BF0C460C2D18BF9DF80A1010D0AA
:100CA00005EB850007EB80004268121B22F07F42B3
:100CB000424506D2827B914228BF8468857C0C2DF8
:100CC000EED10098A04205D004EB080020F07F4050
:100CD0000094019000990398814206D001EB09002D
:100CE00020F07F40F8F7C7FDB0600120864991F8F9
:100CF0002710002904BF05B0BDE8F08FBAF1000F3E
:100D00003FF42EAF05B0BDE8F08F2DE9F04F064659
:100D100087B00C467F480CF00DFB4FF0010800280F
:100D200035D07D4F387D002818BFFFDF3E74207915
:100D3000794D05F10C022872607968722946A06825
:100D4000F8F7A6FD95F90C000F2804DD1F3828736D
:100D50002868401C286095F90C00E1682E1D0844A5
:100D6000C01C1F28B8BFC6F8008009DB6A463146A0
:100D7000F8F78EFD9DF8000010B13068401C30601F
:100D80002078A87287F8148007B0BDE8F08F634D13
:100D900095F8CD0116281ED095F8CD0195F8CC1107
:100DA000401C884200D1FFDF55480068C005C00DD7
:100DB0001AD0103841B20029BDBF01F00F0000F178
:100DC000E02090F8140D01F1E020A8BF90F8000495
:100DD000400909D104E095F8CC010028E4D1E2E70C
:100DE0002078002818BFFFDF4C4890F8CD1101EBA8
:100DF000810100EB810006742078012800F04A810F
:100E0000022843D0454890F8CD1101EB810100EB59
:100E10008105207928726079687205F10C022946F3
:100E2000A068F8F735FD95F90C000F2804DD1F3890
:100E300028732868401C286095F90C10E0682E1D66
:100E40000844C01C1F28B8BFC6F8008009DB6A46EA
:100E50003146F8F71DFD9DF8000010B13068401CC8
:100E600030602078A8722D4890F8CD1116290EBF59
:100E7000002190F8CD11491C80F8CD1125480CF0C7
:100E80006FFA07B0BDE8F04FF8F7D0BC234890F8F0
:100E9000CD1101AA01EB810100EB81076946E068F1
:100EA000F8F7F6FC9DF904000F28CCBF01200020C4
:100EB00000993D1D08440190A068C01C1F28B8BFC0
:100EC000C5F8008009DB6A462946F8F7E1FC9DF881
:100ED000000010B12868401C28600220B8726079B8
:100EE00078722079387200280CBF04210221054A4B
:100EF00052F82000014403917A68481D10440FE025
:100F000004ED00E070E50100E0090020FFFF3F0074
:100F1000F80800200C0A0020C4080020F406002075
:100F20000199009008440399401A0590FD4C002057
:100F300084F82700F8F70DFC3860019980460844D2
:100F400020F07F40F86094F829000C287ED02146DC
:100F500091F8290000EB8002A1F1E80000EB820289
:100F60005668009A324422F07F42029297F809B004
:100F700091F829503446111B21F07F4A6FF07F41D0
:100F8000891BA94604910C2D23D0E74805EB850168
:100F900000EB81026FF07F435068011BB1F5800FB9
:100FA00024BFA4EB000CBCF5800F0BD38B4203D203
:100FB00004990844411C05E0634509D2191A08192F
:100FC000401C41420029BCBFA946957CDBDB00E008
:100FD000FFDF4D4524D0D44809EB890100EB8103A4
:100FE0006FF07F429868011BB1F5800F12D3A4EB1C
:100FF000000CBCF5800F0DD38A4203D20499014442
:10100000491C07E0624528BFFFDF09D2121A1119F7
:10101000491C4942002903DD997B8B4528BF0446C2
:101020000C2D18BFC04910D005EB850001EB8000E6
:101030004268121B22F07F42524506D2827B9345C2
:1010400028BF8468857C0C2DEED100E01BE0A64211
:1010500005D004EB0A0020F07F4026460290029A59
:10106000A6EB080020F07F40A2EB0802059922F0D1
:101070007F42B0F5800F06D2914204D303983044EA
:1010800020F07F403860A74890F8270000287FF4C0
:101090004DAFE8E6A548851915F8010C002818BFE2
:1010A000FFDF05F8018CADE60020F8F797BA0120C4
:1010B000F8F794BA9E48007870472DE9F0419A4EAF
:1010C00000274FF00308012506F1E80450B301287A
:1010D0005BD0022800F0E98003281CBFFFDFBDE8D9
:1010E000F08194F829000C2808BFFFDF84F82670EF
:1010F00084F82B5094F8290000EB800006EB800068
:1011000080F81080F8F799FB94F8290094F82910DA
:10111000401CC0B201EB810156F82120BDE8F0412E
:101120000521104794F829000C2808BFFFDF84F838
:10113000267084F82B5094F8290000EB800006EB11
:10114000800080F81080F8F778FB207F002818BF17
:10115000FFDF84F825500020F8F750FAA168B1F1BC
:10116000FF3F04D0012300221846F8F78BFA94F8C9
:10117000290094F82910401CC0B201EB810156F8F7
:101180002120BDE8F0410121104794F829000C28E6
:1011900008BFFFDF84F8267084F82B5094F82900EC
:1011A00000EB800006EB800080F81080F8F745FB2C
:1011B0000120F8F723FA94F8250000281CBFA06846
:1011C000B0F1FF3F0DD094F8290094F82910401C8D
:1011D000C0B201EB810156F82120BDE8F0410621A3
:1011E0001047207F012815D002281FD0032833D0B4
:1011F00004281CBFFFDFBDE8F08194F82010606870
:101200000123411A00221846F8F73CFA94F8280006
:10121000B8BB37E094F8240028B184F82470F8F7BC
:1012200013FB84F823502777BDE8F08194F8280059
:1012300018B9F8F78BFB84F8285094F8290094F833
:101240002910401CC0B201EB810156F82120002179
:1012500090472777BDE8F081217B60680123411A20
:1012600000221846F8F70EFA94F8240028B184F802
:101270002470F8F7E9FA84F8235002202077BDE8BB
:10128000F08103E0F8F762FB84F8285094F8290015
:1012900094F82910401CC0B201EB810156F82120BE
:1012A000002190472577BDE8F08121480078BDE80E
:1012B000F041F8F7FFBD10B51A4C94F829000C283E
:1012C00008BFFFDF94F8290094F82910401CC0B231
:1012D000154A01EB810152F82120BDE8104004219C
:1012E00010472DE9F84F8046087C104C401EC6B2CE
:1012F0000D46A05D01281DD0022825D0297CDFF8ED
:1013000028A0481EC4B204EB84020AEB8206371DF3
:101310000A2821D801EB81000AEB800010F8040CA8
:10132000D8B919E0E0090020F8080020D40900200D
:1013300078000020A87A012814BF02200020A055C0
:1013400018BFBDE8F88FD9E7A87A012818BFFFDFDA
:101350000021A972A155D1E7FFDF307CDFF8289486
:1013600007280BD11720009099F8172009F11803CE
:10137000494620460BF02AFD01203074307C0128BC
:1013800004D0A87A012818BFFFDF02D0A87A01286C
:101390004BD1FE4B307C022818D099F81800162843
:1013A00072D099F8180099F81710401C884200D1A3
:1013B000FFDF0120707499F8180009F8004099F8CF
:1013C0001800162800F09E8100F093B9F04A92F8B8
:1013D00029000146A04207D0014600EB810003EB43
:1013E0008000807CA042F7D192F829C084450CD1BE
:1013F00092F8291001EB810103EB8101897C82F8CD
:101400002910012182F82A1009E000EB800203EB89
:10141000820201EB810103EB8101927C8A7400EB73
:10142000800003EB80000C218174287AD9490028C0
:1014300051F820A02968A1EB0A010CBF042002206A
:10144000081A20F07F423A60D5E90001084420F0F4
:101450007F407860A87A022818BF287B1ED0387297
:101460007868401D20F07F407860687AB872287AEA
:1014700006257872032872D2002870D000F022FE70
:1014800000286DD0A1E0FFE799F81700002890D15F
:101490008EE700BF89F81800BDE8F88F287A002889
:1014A0000CBF0420022000EB0A036868591D00EB02
:1014B000010BB9484078504503D9B54991F823103C
:1014C00011B10BF1060003E0A0EB0A005844801DA7
:1014D000AF4991F829C0BCF10C0F25D091F829C073
:1014E0000CEB8C0EA1F1E80C0CEB8E0CDCF804C0BC
:1014F000624519D0DFF8A4C291F8291001EB8102EE
:10150000A24901EB82014A688968A2EB080222F035
:101510007F42A1EB080121F07F41904298BFB2F5D4
:10152000800F9DD28C459BD34044A0EB0B0020F054
:101530007F4139601944E86821F07F410A1A6FF051
:101540007F4CB2F5800F24BF431AB3F5800F11D33F
:10155000944506D2ACEB00000844421C0AE034E09B
:101560002FE09C4528BFFFDF1DD2ACEB01010844F2
:10157000401C4242002A16DD0520307499F81800FC
:10158000162819D099F8180099F81710401C8842AD
:1015900000D1FFDF99F8180009F8004099F8180009
:1015A00016287BD0A5E03868ABF10501084420F08F
:1015B0007F407860002052E799F817000028E9D1B1
:1015C000E7E7CAF138054FF0320A7348017801297C
:1015D00018BF03290AD14078504507D96C4991F8C2
:1015E0002310002904BFA0EB0A0005446B4B3868A8
:1015F000A0EB0802786822F07F41A0EB080020F001
:101600007F4C8D4298BFB1F5800F1BD2634519D333
:101610005F4991F829300C2B30D091F829504FF0C8
:101620000C0BDA46594905EB850301EB8303D3F82C
:1016300008C0ACEB080C944531D8AB469D7C0C2D12
:10164000F0D193E00520307499F81800162810D0D6
:1016500099F8180099F81710401C884200D1FFDF54
:1016600099F8180009F8004099F81800162849D090
:101670003FE099F817000028F2D1F0E7022030741B
:1016800091F829000C2818BF91F82900B07481F84E
:101690002940012081F82A00BDE8F88F32E00C2DA6
:1016A0001CBFAA46002261D00AEB8A0301EB830328
:1016B000D3F804C0ACEB080C84452CD29A7B97F885
:1016C0000AC0944520D30520307499F818001628D4
:1016D00013D099F8180099F81710401C884200D1CF
:1016E000FFDF99F8180009F8004099F8180016284B
:1016F00008D099F81800401CCCE699F8170000288B
:10170000EFD1EDE70020C5E693F812A00122BAF16F
:101710000C0FC9D103E0002A08BFAA4626D02F46E5
:101720001A4807EB870100EB8108062288F8102091
:1017300099F81800162838D099F81800411C99F823
:101740001700814200D1FFDF99F8180009F80070F6
:1017500099F8180016280EBF002099F81800401CB0
:1017600089F8180098F81270BA45D9D10220074FAD
:10177000307407F1E80090F82910A9421AD186F8D0
:1017800012A080F829400BE0DC080020F8080020B7
:10179000E009002070E501007A000020FFFF3F0013
:1017A000012180F82A10BDE8F88F99F81700002869
:1017B000CAD1C8E70C2D0CD0BBF10C0F08BFFFDF5E
:1017C0000BEB8B0007EB8000847486F812A0BDE859
:1017D000F88FBBF10C0F08BFFFDF0BEB8B0007EBA3
:1017E000800084740C20B074BDE8F88F2DE9F04FB0
:1017F00083B0F7F7AEFF05464FF00C0BFE4C94F8A4
:1018000029100026A4F1E8094FF001080C292FD077
:1018100094F82920214602EB820209EB8202127C15
:10182000042A25D091F8292002EB820209EB8202DA
:10183000127C032A04BF03B0BDE8F08F2A4620695A
:101840006169801A491BED4B20F07F4021F07F41F8
:1018500006283CBF03B0BDE8F08FB0F5800F24BF71
:1018600003B0BDE8F08F8B423CBF03B0BDE8F08F02
:10187000A068B0F1FF3F18BFFFDF84F8256094F83F
:101880002900DF4F0C2809D094F8290000EB8000D4
:1018900009EB8000007C042808D01AE094F82100AD
:1018A000B8B1F8787870B878387012E094F829B048
:1018B0000BEB8B0009EB800080F8108094F8290076
:1018C00000EB800009EB8000807C84F8290084F81C
:1018D0002A80DFF830A39AF8CD019AF8CC1188421B
:1018E00019D000BF9AF8CC0100EB80000AEB800110
:1018F0002846FFF7F6FC9AF8CC0116280EBF002008
:101900009AF8CC01401C8AF8CC019AF8CD019AF8DB
:10191000CC118842E6D1DFF8F0A29AF8140028B181
:1019200051462846FFF7DDFC8AF81460BBF10C0F26
:1019300006D00BEB8B0009EB8000017C01292BD03A
:1019400094F829000C2800F0ED8094F82A00002873
:1019500000F0F78084F82A6094F8290000EB8001F9
:10196000AA4800EB8102A0F50173D2E90101D26817
:10197000C3F80423C3E9BF01607E00280CBF4FF009
:1019800004094FF00209A249022811F8201021731E
:1019900018BF012834D123E007210174DFF874A2B5
:1019A0009AF81800162816D09AF818009AF8171006
:1019B000401C884200D1FFDF9AF818000AF800B0F6
:1019C0009AF8180016280EBF00209AF81800401C3C
:1019D0008AF81800B4E79AF817000028ECD1EAE773
:1019E00020690844421B22F07F42382A08D903218B
:1019F0003238617620F07F4020613220207309E088
:101A0000322907D294F8280058B9F7F79FFF84F8D5
:101A1000288006E094F8280018B1F7F7C0FF84F892
:101A200028607B7884F8203094F80CA03878062160
:101A3000A3EB0A02012818BF032804D184F82480EC
:101A4000002AC8BF911D94F822B0BBF1000F18BF47
:101A5000891C206901905044484420F07F40606018
:101A6000BAF1000F14BF02200020207794F8240060
:101A7000002808BFBBF1000F37D060480090D4F8B1
:101A800010E0D4F814C0AEEB050E2EF07F4EACEB98
:101A9000050C20462CF07F4C714598BFBEF5800F99
:101AA0001FD2009961451CD3002A0FDD0199BAF1BC
:101AB000000FA1EB020101611944494421F07F416B
:101AC00041600CBF0121032121770EE004DA002BD5
:101AD0000CBF02210421F7E7BBF1000F08BFFFDFB5
:101AE00003E080F8246084F82260207F40B1206900
:101AF000012300EB090100221846F7F7C3FD02E0BD
:101B00000120F7F77BFD94F82900012300EB800109
:101B10003E4800EB8100616890F90C200020F7F747
:101B2000B1FD0EE00120F7F769FD0020F7F766FD33
:101B3000F7F74AFD94F8280018B1F7F730FF84F85A
:101B4000286094F8220028B1F7F77EFE84F823601D
:101B500084F8226094F8210018B1F8787870B87889
:101B6000387094F8240030B184F823603878002865
:101B700008BF84F824602748017EC07D814203D0DD
:101B800025484078F8F796F984F8278003B0BDE837
:101B9000F08F70B5184C054682B094F829000C28D7
:101BA00008BFFFDF94F8290000EB8000174E06EB1A
:101BB0008000007C032818BFFFDFA068B0F1FF3F62
:101BC00018BFFFDF94F8290001AA00EB800006EBA4
:101BD0008000694690F90C002844F7F759FE9DF9FA
:101BE00004000F28CCBF0120002000990844616840
:101BF000084420F07F4111E0E0090020FFFF3F0092
:101C00007A000020F4060020C4080020F808002014
:101C100070E50100DC08002078000020A16094F845
:101C20002500002804BF02B070BD012302B00022CD
:101C3000BDE870401846F7F725BD744A0B1A02F14B
:101C4000010CB3EB9C0F3CBF1846704710B5441A0B
:101C5000B4EB9C0F3CBF184610BD9A4203D2101A39
:101C60000844401C10BD94429EBFFFDF002010BD01
:101C7000511A0844401C404210BD01230022014675
:101C80000220F7F7FFBC0220F7F7B8BCF7F761BDF9
:101C90002DE9F0415E4C054682B094F82B000028F7
:101CA00008BFFFDF642D50D35A480022401B72EB5F
:101CB00002004AD3584890F8CD1190F8CC018142E7
:101CC00043D15648007D00283FD194F82900DFF821
:101CD000508100EB800008EB8006206801AA2844B0
:101CE0006946F7F7D5FD9DF90400002802DD00984C
:101CF000401C0090B168009872680F18BA1A22F060
:101D00007F42B2F5800F20D2B27C0C2A09D002EBC0
:101D1000820208EB82025268511A21F07F4181420F
:101D200013D3A068B0F1FF3F05D00120F7F766FCA0
:101D30004FF0FF30A06020682844206027F07F40EB
:101D4000606102B00120BDE8F08102B00020BDE872
:101D5000F0812DE9F8430646401EC7B2304807EB34
:101D6000870100EB8104207C002808BFFFDF2A4A9E
:101D700092F8CC1192F8CD0181420DD001EB810394
:101D800002EB83031B7CB34210D016290CBF002149
:101D9000491CC9B28142F1D120484FF0170800F127
:101DA0001805017D29B3007CB04222D10020BDE896
:101DB000F883207C05281FBF207C0628207C07286C
:101DC0000AD184F81090CDF80080EA7D05F118035F
:101DD000144938460AF0FAFF607C68B16674CDF8A1
:101DE0000080EA7D05F118030E4938460AF0EEFF3F
:101DF00002E04FF001090026207C012804BF607C2E
:101E00000028D6D10120BDE8F8830000FF7F841EA2
:101E1000E0090020FF1FA107F4060020C4080020ED
:101E2000F8080020DC080020F0B5734AD2F8003230
:101E3000724D002401212E7856B9714E3460704FD6
:101E400003263F1D3E606E4F04260C373E6029700E
:101E5000C2F80042D1601160694C4834D1642568F1
:101E60008542FBD35160D160C2F80032F0BD2DE94C
:101E7000F041044680074FF000054FF0010604D5FD
:101E800060480560066024F00204E0044FF0FF376C
:101E900005D55D484660C0F8087324F4805460009E
:101EA00003D55A48056024F08044E0050FD5524818
:101EB000C0F80052C0F8087351490D60091D0D604B
:101EC0004F4A04210C321160066124F48074A0048E
:101ED00009D54F484660C0F80052C0F808734D4815
:101EE000056024F40054C4F38030C4F3C031884248
:101EF00000D0FFDF14F4404F14D047484660C0F8CC
:101F0000087346488660C0F80052C0F80873444918
:101F10000D600A1D16608660C0F808730D601660BB
:101F200024F4404420050AD53E4846608660C0F847
:101F30000873C0F848733C48056024F400640BF053
:101F40006FFB3A48044200D0FFDFBDE8F08170B576
:101F5000202500224FEA020320FA02F1C90719D016
:101F600051B201F01F060124B4404E09B60006F13B
:101F7000E026C6F88041C6F88042002906DA01F062
:101F80000F0101F1E02181F8143D03E001F1E021AE
:101F900081F80034521CAA42DED370BD70B5174CD4
:101FA0000D466060FFF763FF6068FFF7D0FF2846CB
:101FB000F7F7A9FD0AF064FF00F0D5F80BF030FB4D
:101FC0000BF07BFAF7F748FFBDE870400BF006B85E
:101FD00010B50A4C6068FFF74AFF6068FFF7B7FF6B
:101FE0000BF01EFBF7F753FE0020606010BD0348A6
:101FF0004068704702207047008000408000002049
:1020000004850040FC1F004000C0004004E5014082
:1020100000D0004004D5004000E0004000F0004047
:1020200000F5004000B0004008B50040FEFF0FFC86
:1020300070B51F490A68BAB100231D4601244A68D9
:10204000521C4A60092A00D34D600E7904FA06F248
:102050000E6816420AD072B60B6893430B6062B6E4
:1020600049680160002070BD052070BD5B1C092B14
:10207000E5D3FFDFF8E74FF0E0214FF48000C1F82F
:1020800000027047EFF3108111F0010F72B64FF0AC
:10209000010202FA00F20648036842EA0302026003
:1020A00000D162B6E7E70248002101604160704755
:1020B0008800002001208107086070470120810707
:1020C0004860704712480068C00700D00120704780
:1020D0000F48001F0068C00700D0012070470C485F
:1020E00008300068C00700D0012070470848103051
:1020F0000068704706490C310A68D20306D50968A2
:1021000001F00301814201D1012070470020704796
:102110000C040040C84911F8210F4978884201D3C6
:10212000401A02E0C1F121010844C0B27047C2491F
:10213000233111F8210F4978884201D3401A02E077
:10214000C1F121010844C0B27047BB49463111F8C2
:10215000210F4978884201D3401A02E0C1F12101E0
:102160000844C0B27047B54910B5802081F800041A
:10217000B1490020233101F8210F4870AE4901F820
:10218000210F4870AC49463101F8210F4870AC4826
:102190000BF0C8F8AA48401C0BF0C4F8F0F7A4FEF6
:1021A000BDE8104000F03DB920207047B2E770B59F
:1021B0000C4605460026FFF7ADFF01469E48A142AA
:1021C00012D30022641EE4B20DD390F82210435CB7
:1021D000491CC9B205F8013B80F822102129F1D130
:1021E00080F82220EEE7012600F01BF9304670BD92
:1021F000202070479BE770B50C4605460026FFF788
:1022000096FF01468C482330A14212D30022641E5F
:10221000E4B20DD390F82210435C491CC9B205F812
:10222000013B80F822102129F1D180F82220EEE72D
:10223000012600F0F6F8304670BD20210170002024
:10224000704710B50446FFF780FF2070002010BDD6
:1022500070B50C460546FFF778FF014676484630D4
:10226000A14213D30022641EE4B20DD390F82210D1
:10227000435C491CC9B205F8013B80F822102129B2
:10228000F1D180F82220EEE7002401E042F20704B9
:1022900000F0C7F8204670BD70B50C4605462129F0
